:020000040800F2
:1000000000200010459C020829F40108FDE80008C2
:1000100025F4010821F401081DF401080000000086
:1000200000000000000000000000000019F40108BA
:1000300015F401080000000011F40108F1D20008D5
:10004000AD9C0208AD9C0208AD9C0208AD9C020864
:10005000AD9C0208AD9C02081DE6000849E70008B7
:100060000DE70008D1E6000895E6000861CD00081C
:1000700051CD000841CD000831CD000821CD000848
:100080000DCD0008F9CC0008AD9C0208AD9C02081B
:100090001DF80108AD9C0208AD9C020859E6000855
:1000A00031EF00088DEF000821EF0008B1EF0008E4
:1000B00081EF000871EF000861EF0008AD9C0208B5
:1000C000AD9C0208AD9C0208AD9C0208AD9C0208E4
:1000D000AD9C02081DD40008A1D3000825D3000858
:1000E000E1E50008AD9C020801F40108AD9C02089E
:1000F00041EF0008AD9C020851EF0008AD9C0208DA
:10010000000000000000000000000000AD9C02089C
:10011000AD9C0208AD9C0208554D0208394D0208FD
:10012000E5CC0008D1CC0008BDCC0008A9CC000863
:1001300095CC0008AD9C0208000000000000000003
:10014000AD9C0208AD9C0208AD9C020800000000B6
:10015000000000000000000000000000000000009F
:100160000000000000000000AD9C0208AD9C0208E9
:10017000AD9C02080000000000000000000000002C
:0801800000000000AD9C020824
:100188002DE9F04FB0F908502DED028B0D81EDB23D
:10019800442D8FB00C4600F02D85804642D9812D24
:1001A80000F0838400F29380542D00F0C88040F260
:1001B80034846E2D00F05984802D40F0E780664B22
:1001C80093F8009009F1020919F0FF0900F09280F4
:1001D800624B634F634EDFF8B0A1994403F1010805
:1001E8000A2516E0322D02F00C80A5F13C00C0B2C1
:1001F800132842F20D8000232268511C21601570DB
:100208002268C84502F101012160137072D018F804
:10021800015B0A2DE6D1BAF80030FF2BA8BFFF23F7
:10022800DBB2E9E7052D00F0D2841AD8022D7ED082
:1002380040F2E083032D00F0BD84042D40F0A68039
:100248002A46494920460CF09DF8002120460CF02A
:10025800C9F822680021531C012523602B46117020
:100268002EE0242D5BD040F27B83282D00F065849E
:10027800382D40F08B800A683C4B0125511C2160C9
:1002880015702268052150192060117022680A2112
:1002980050192060117022680021501920601170D7
:1002A80022681978501920601170226859785019FD
:1002B8002060117022689978531923602B461170B9
:1002C800284663810FB0BDEC028BBDE8F08FA02DEE
:1002D80013D040F26483B82D00F06984FE2D55D107
:1002E800234D05F1080635F8021B20460CF07AF874
:1002F800AE42F8D101252B46E2E71E4B08461968A5
:100308000CF058F81C4B204619680CF053F81B4B9E
:100318002046196801250CF04DF82B46D0E7184BFC
:100328001968204601250CF045F82B46C8E7042239
:100338001449204601250CF025F82B46C0E70B6828
:1003480000215A1C22601970226801255319236064
:100358002B461170B4E700BF7554002008C5020889
:10036800676666667C230020E3590020BD6700208D
:1003780098540020ACF7FF1FB0F7FF1FB4F7FF1F1A
:100388005C3C0020CCEB0208A4230020A5F10A0362
:10039800E72B00F2EA80DFE813F06006E800E800E7
:1003A800E800E800E800E800E800E800E800E80005
:1003B800E800E800E800E800E800E800E800E800F5
:1003C800E800E800E800E800E8004106E800E80086
:1003D800E8003006E800E800E8002606E800E50541
:1003E800E800E800E800E800E800C605E800B8060C
:1003F800E800A306E800E800E8005A048904E800D9
:100408009F06E800E8009606E8007306E800E800A2
:10041800E8004D04E800E800E800E8004E08E800BD
:100428002C08E8001A08F607E800E800E800E800E9
:10043800E800E800E800A907E8007E07E8004D07A3
:10044800E800DE06E8001409E800E800E800E80033
:10045800EB082509ED077C086A08E800E800AD0804
:10046800BC05E80082056505E800E800E800E8004A
:100478005905E800E8003705E800E800E800260527
:100488000D05FC04E800E800E800E800EB04E800DB
:10049800E8009F04E800E800E800E800E800E80059
:1004A800E800E800E800E800E800E800E800E80004
:1004B800E800EB08E800E800E800E800E800E800E9
:1004C800E800E800E800E800E800E800E800E800E4
:1004D800E800E800E800E800E800E800E800E800D4
:1004E800E800E800E800E800E800E800E800E800C4
:1004F800E800E800E800E800E800E800E800E800B4
:10050800E800E800E800E800E800E800E800E800A3
:10051800E800E800E800E800E800E800E800E80093
:10052800E800E800E800E800E800E800E800E80083
:10053800E800E800E800E800E800E800E800E80073
:10054800E800E800E800E800E800E800E800E80063
:10055800E800E800E800E800E800E800E800E80053
:10056800E800E800E8009204C004742D00F06C82F2
:10057800772D00F05882292DD8F8006000F04383C9
:10058800392D01F07687212D01F04D87D8F8042008
:100598000B3D931BEF2D01F2918501A151F825F038
:1005A80043170008C5200008C5200008C52000081A
:1005B800C5200008C5200008C5200008C52000087F
:1005C800C5200008C5200008C5200008C52000086F
:1005D800C5200008C5200008C5200008C52000085F
:1005E800C5200008C5200008C5200008C52000084F
:1005F800C5200008C5200008C5200008C52000083F
:10060800CB160008C5200008B1160008C520000850
:100618008F160008C5200008C5200008C52000085E
:1006280063160008C52000083D210008C520000801
:10063800C5200008C5200008C5200008C5200008FE
:100648002D210008C5200008CF200008C52000087B
:1006580081200008C5200008C5200008C520000822
:10066800C5200008FD020008C5200008E521000893
:10067800C5200008C5200008C9210008C5200008B9
:10068800931E0008C5200008C5200008C5200008E2
:10069800C5200008C5200008C5200008C52000089E
:1006A800C5200008471E0008C5200008291F0008AB
:1006B800C5200008C5200008EB1E0008C52000085A
:1006C800C5200008C5200008C5200008C52000086E
:1006D800C5200008C5200008AD1F0008C520000877
:1006E800B31D0008C5200008051D0008C520000826
:1006F800511C0008C5200008DF1B0008BF1B0008AC
:10070800C5200008C5200008C5200008C52000082D
:10071800C5200008C5200008C5200008C52000081D
:10072800C5200008C5200008C5200008C52000080D
:10073800C5200008C5200008C5200008C5200008FD
:10074800C5200008C5200008C5200008C5200008ED
:10075800C5200008C5200008C5200008C5200008DD
:10076800C5200008C5200008C5200008C5200008CD
:10077800C5200008C5200008C5200008C5200008BD
:10078800C5200008C5200008C5200008C5200008AD
:10079800C5200008C5200008C5200008C52000089D
:1007A800C5200008C5200008C5200008C52000088D
:1007B800C5200008C5200008C5200008C52000087D
:1007C800C5200008C5200008C5200008C52000086D
:1007D800C5200008C5200008C5200008C52000085D
:1007E800C5200008C5200008C5200008C52000084D
:1007F800C5200008C5200008C5200008C52000083D
:10080800C5200008C5200008C5200008C52000082C
:10081800C5200008C5200008C5200008C52000081C
:10082800C5200008C5200008C5200008C52000080C
:10083800C5200008C5200008C5200008C5200008FC
:10084800C5200008C5200008C5200008C5200008EC
:10085800AB1A0008C5200008951A0008C520000832
:10086800C5200008C5200008C5200008C5200008CC
:10087800C5200008C5200008C5200008C5200008BC
:10088800C5200008C5200008C5200008C5200008AC
:10089800C5200008391A0008C5200008FB190008FF
:1008A800C5200008111B0008DB1A0008F51A00080B
:1008B800C5200008E1190008C5200008B71900087C
:1008C800C520000857190008C52000082F1900087E
:1008D800C5200008C52000080D190008D91800080F
:1008E8006B1800083D180008C52000081B180008F0
:1008F800C5200008C5200008C5200008C52000083C
:10090800C5200008C5200008C5200008C52000082B
:10091800C5200008C5200008C5200008C52000081B
:10092800C5200008C5200008C5200008C52000080B
:1009380001180008C5200008C520000897170008FE
:10094800C5200008C5200008C5200008C5200008EB
:10095800C5200008C5200008C52000087D1700082C
:10096800202D7FF413AD0B68BD4D591C6A782160AA
:100978001A7023682A78591C21601A702368AA788B
:10098800591C21601A70298920460BF02BFD236819
:100998006A79591C21601A702268A9795BE4822D52
:1009A8007FF4F4AC0B68AF4AAF4D1178AC4A581CD1
:1009B80020601970118920460BF014FDAB4B22689A
:1009C8001B88FF2B02F10101A8BFFF2321601370D0
:1009D800A96881F3100189B220460BF003FD29684C
:1009E80001F30F0189B220460BF0FCFCA04B2268F2
:1009F800197830E4012D7FF4C9AC0B680022591C2A
:100A080021601A7023685A1C22601D7022682421F4
:100A1800531C23602B46117052E4522D7FF4B6AC60
:100A28000A68002117E4D8F80030D8F804209A4260
:100A38001EBF5A1CC8F8002019788E4A08BF00212A
:100A4800204623F083F855E4D8F80030D8F804207D
:100A58009A421EBF5A1CC8F800201978864A08BF57
:100A68000021204623F072F844E4804B0A681B8872
:100A78007D4DFF2BA8BFFF23511C21601370A9686F
:100A880081F3100189B220460BF0ACFC7B4B204669
:100A980019880BF0A7FC296801F30F0189B22046D9
:100AA80001250BF09FFC2B460AE4754B1E78033694
:100AB80016F0FF063FF41EAC724B734F1E4403F151
:100AC80001094FF00A0820E0B8F1500F01F09683B1
:100AD800B8F1320F01F0B283A8F13C00C0B213287C
:100AE80041F2B0830025294623685A1C226020461B
:100AF80083F800800BF076FC294620460BF072FC48
:100B08004E453FF4F7AB19F8018BB8F10A0FDBD16A
:100B18005E4B9D68196805EB85054FF6FF736D0000
:100B28009D42A8BF1D469942A8BF194625EAE5750A
:100B380021EAE171ADB289B2D6E70B68DFF86881C6
:100B4800534E591C022221601A70236806275A1C2A
:100B580022601F7023680A22591C21601A702368BA
:100B680001255A1922601D70B8F8001020460BF0B4
:100B780039FCB8F8021020460BF034FC23685A19E7
:100B880022601F7023685022591921601A70236847
:100B98000022591921601A70318820460BF022FC76
:100BA800718820460BF01EFC2B46FFF789BB394B9A
:100BB800FFF7B6BB0B685A1C0A601D700B6802224F
:100BC800591C21601A7022680021FFF744BB0B22D0
:100BD800314920460BF0D6FB0822304920460BF05D
:100BE800D1FB012507222E4920460BF0CBFB2B46D3
:100BF800FFF766BB002A3FF47DAB2A4B1360012543
:100C08002B46FFF75DBB731CC8F8003033780A2BFE
:100C180001F07484502B41F05C8140460BF0A0FB3E
:100C28001B4E308040460BF09BFB012570802B4605
:100C3800FFF746BB236800255A1C22602946204638
:100C48001D700BF0B7FB294620460BF0B3FB0021C3
:100C5800204601250BF0AEFB2B46FFF731BB00BF4A
:100C68006C5A00205A550020204500204455002089
:100C780078430020352E0208153A0208583A002019
:100C88007554002018C50208742300203023002062
:100C980064230020A4430020D4EB0208E0EB020800
:100CA800ECEB020839E800082C3C002022680121FE
:100CB800531823600D460B461170FFF701BB9C4D7E
:100CC8002046E9890BF08EFBA989204601250BF007
:100CD80089FB2B46FFF7F4BA2368964F591C3A78DC
:100CE80021601A703B78002B3FF404AB0025EEB26C
:100CF800304621F0B1F823684278591C216030460B
:100D08001A7021F0A9F8018920460BF06BFB3B789B
:100D180001359D42EBDBFFF7EDBA874B03F1700518
:100D280022681978501C2060117022685978501C6C
:100D38002060117022689978501C20601170226818
:100D4800D978501C2060117022681979501C2060D5
:100D5800117022685979501C2060117022689979A5
:100D68000733501CAB4220601170D9D1FFF7C2BACB
:100D7800724D2046298A0BF035FB698A20460BF014
:100D880031FBA98A204601250BF02CFB2B46FFF7E7
:100D980097BA23686A4A6B491078654A5D1C2560D2
:100DA800187023689278581C20601A702268897815
:100DB800FFF751BA2268644B64491878551C2560BE
:100DC800107022685878551C2560107022689B782E
:100DD800501C20601370C988204601250BF002FBC7
:100DE8002B46FFF76DBA594D204629880BF0FAFAC1
:100DF800698820460BF0F6FAA988204601250BF0F1
:100E0800F1FA2B46FFF75CBA514D05F16006A98847
:100E180020460BF0E7FAE98820460BF0E3FA298927
:100E280020460BF0DFFA2368AA7A591C21601A7051
:100E38002368EA7A591C21601A7055F80C1B204661
:100E48000BF0B8FAB542E2D1FFF754BA4149522340
:100E58002268501C2060137011F8013F002BF7D155
:100E6800FFF748BA3C4D00232268286803EB43018A
:100E7800561C405C266010702A6820680A44461C8C
:100E88005278266002702A6820680A4401339278F2
:100E9800411C0A2B21600270E6D1FFF72BBA2F4DB7
:100EA80023682A68591C127821601A702B682268F6
:100EB8009978531C2360002311702A6821681A440A
:100EC80001335279481C032B20600A70F5D123683E
:100ED8002A68591C127A21601A7023682A68591CDA
:100EE800D27821601A7023682A68591C1279216007
:100EF8001A702B68204659890BF074FA23682A68FF
:100F0800591C527A21601A702B6822685978FFF7A9
:100F1800A2B9002120460BF04DFA002120460BF023
:100F280061FAFFF7E7B90E4B2268597DFFF793B9CD
:100F38003C3C00207554002054330020C04B002056
:100F4800F04E00204C3C0020343C0020742F002040
:100F580060320020D8C40208EC590020D02B0020B1
:100F680030530020A74D23682A7A591C21601A7033
:100F7800A98B20460BF036FA298B20460BF032FA63
:100F8800698B20460BF02EFA2368EA7C591C2160F5
:100F98001A70A98C20460BF025FAE98C20460BF034
:100FA80021FA2368AA7F591C21601A70236895F8D2
:100FB8002020591C21601A70698C20460BF012FA07
:100FC8002368EA7A591C21601A70E96820460BF0F8
:100FD800F1F923682A7C591C21601A70226895F857
:100FE8002110FFF738B9884B22681978501C206007
:100FF800117022685978FFF72EB9844D2046298848
:101008000BF0F0F9A98820460BF0ECF92989204665
:1010180001250BF0E7F92B46FFF752B97C4D05F196
:101028005006287822F0E6FD2368027A591C2160D0
:101038001A7023686A78591C21601A702368AA7884
:10104800591C21601A702368EA780435591CAE428D
:1010580021601A70E5D1FFF74DB96E4D284628F08A
:101068002FF900287FF746A92B460544226813F874
:10107800011B501C9D4220601170F7D1FFF73AB94F
:101088002368614A614D1178634A581C20601970C1
:10109800116820460BF08EF923685A4A591C127AB7
:1010A80021601A70298820460BF09CF9A9882046EF
:1010B8000BF098F9298920460BF094F90021204675
:1010C8000BF090F929E708224E49204601250BF03C
:1010D80059F92B46FFF7F4B8504B2268997885E701
:1010E8004F4D504E05F1300795F902104E4B93F9CC
:1010F80006208A4203F1080301F0BD809E42F6D122
:101108000835AF42F0D1FFF7F5B8484B03F15A055F
:1011180022685979501C2060117022681978501C77
:101128002060117022685978501C20601170226864
:101138009978501C206011702268D978501C206062
:101148001170226819790633501C9D422060117075
:10115800DED1FFF7CFB8002120460BF043F900217C
:1011680020460BF03FF9002120460BF03BF923689D
:101178002F4D00265A1C22601E7023682A68591CAD
:1011880092F82C2021601A7023682A68591C92F85A
:10119800362021601A7023682A68591C92F8372073
:1011A80021601A7023685A1C22601E7023685A1C1A
:1011B80022601E7023685A1C22601E702B6820460D
:1011C800598F0BF00FF92B682046198F0BF00AF98D
:1011D8002A68236892F82E20591C21601A70236807
:1011E8005A1C22601E702B682046598E0BF0FAF8A4
:1011F8002B682046998E01250BF0F4F82B46FFF753
:101208005FB800BF305300207C3C00208C43002096
:10121800803C0020183C00205C3C0020583C00200A
:1012280008590020BC5300208C530020B0430020F4
:10123800EC590020BC4E23687279BC4D591C2160C2
:101248001A702B682046198C0BF0CCF82B682046B6
:10125800D98B0BF0C7F8718920460BF0C3F8B18918
:1012680020460BF0BFF82B682046598C0BF0BAF8D3
:101278002B682046998C0BF0B5F8F18920460BF0C5
:10128800B1F8318A20460BF0ADF82B68226893F844
:101298002610FEF7E0BFA44FFB78002B01F0098170
:1012A80023680822591C21601A70236801229918A2
:1012B80021601A7023689E4D591C2A7921601A7082
:1012C8002368AA78591C21601A70298820460BF0D7
:1012D80089F8E98920460BF085F82368FA79591CC2
:1012E80021601A702268E978FEF7B5BF25F08AFEFA
:1012F800FF28064601F0EA800EA9002501F82E5DB8
:101308000DF109008DF809501FF0ACFD0EA800F88A
:101318002D5D1FF09BFD0EA800F82C5D1FF08AFDC7
:101328000EA820F8245D25F04DFE23685A1C226083
:101338001E7023689DF80920591C21601A702368C3
:101348009DF80A20591C21601A7023689DF80B200B
:10135800591C21601A7023689DF80C20591C2160C3
:101368001A70BDF81410204601250BF03BF82B46E7
:10137800FEF7A6BF10226F49204601250BF002F8A0
:101388002B46FEF79DBF23686B4E01255A1C226031
:101398001D702368B278591921601A7017F07CFE05
:1013A8002368664A66495F1927601870B1F900100A
:1013B800B2F900000BF090F923685A1922601870EE
:1013C800318820460BF00EF82B46FEF779BF2368CC
:1013D80000255A1C22601D7023685A1C22601D704B
:1013E80023685A1C226029461D7020460AF0E2FF35
:1013F8002DE4544E3378002B3EF47CAF524F002539
:10140800B846236817F81520591C21601A7098F8F7
:10141800011001EB810101EB810101F2EE2189B29A
:1014280020460AF0DFFF337801359D4208F10208B3
:10143800E7DBFEF75FBF2368444D591C2A7921601A
:101448001A7023686A79591C21601A702988204605
:101458000AF0C8FF2368AA79591C21601A706988A4
:1014680020460AF0BFFF2268E979FEF7F4BE354E40
:101478003378002B3EF43EAF354F002537F8021F76
:1014880020460AF0AFFF337801359D42F6DBFEF7C0
:1014980031BF304D304EDFF8D080DFF8D0909FED6F
:1014A8002F8A05F120070EE0FCEEE77ACDED017AF0
:1014B800BDF80410204604350AF094FFBD4206F139
:1014C80018063EF417AF717C0029F3D098F8003065
:1014D800D5ED007A012BE7D1D9F80030DB0440F1D3
:1014E800DB87F5EE407AF1EE10FA41F0228040F207
:1014F800DC51DFE71A4D204629880AF073FF698816
:1015080020460AF06FFFB5F904301649DA1781FB57
:101518000313C2EBA30399B2204601250AF062FF28
:101528002B46FEF7CDBE00BFF04E0020EC59002040
:10153800C04B00205C3A0020EC6800209C3A002058
:101548009E3A0020605A0020E03400208C2F0020B2
:10155800006700206C3A0020004B00200000404249
:10156800D859002067666666E44B00209851002031
:101578000DF1140900220592DFF850A3BE4B039227
:101588000492C9F80420904601214FF6FF7B07E03A
:1015980008F10108B8F10B0F00F08B861AF9011F4A
:1015A8004F1C4BFA08F2F3D0D607F1D51A8842FA45
:1015B80008F2D007ECD5484601930BF0E9F8019BF7
:1015C800E6E72368AD4AAE49D078AE4A5D1C25608F
:1015D800187023685279581C20601A702268C978DC
:1015E800FEF739BEA84B9B8AB3F5006F00F25E8701
:1015F800B3F5806F00F28887B3F5007F34BF012709
:101608000227A24D05F10C0655F8041B91FBF7F1D2
:10161800204689B20AF0E6FEAE42F5D19C4D9D4FB8
:1016280005F10C06B5EC010AD7ED087A80EE270A19
:1016380028F082FD81B220460AF0D4FEAE42F1D1F4
:10164800954D05F10C0655F8041B204689B20AF0A1
:10165800C9FEAE42F7D1FEF74DBE731CC8F8003084
:101668008E4930780870D21A002A7EF743AEB31C30
:10167800C8F800307378003318BF012301254B7078
:101688002B46FEF71DBE40460AF06AFE844E3060C7
:1016980040460AF065FE706040460AF061FE01258A
:1016A800B0602B46FEF70CBE7E4E002333604046EA
:1016B8000AF03EFE33680125034333602B46FEF7EC
:1016C800FFBD731CC8F800303578132D00F2F6847E
:1016D800B31CC8F80030707822F072FA002800F0C5
:1016E800ED84714B027803F82520F21CC8F800201D
:1016F80003EB8505B2786A70321DC8F80020F278CD
:10170800AA70721DC8F800203279EA7003F15001FE
:1017180003E004338B4200F098871A78002AF8D146
:101728009878DA789042F4D20123604A83F0010372
:10173800012513702B46FEF7C3BD5D49102B4FF0F2
:10174800000228BF10230A604A608A60CA600A74CF
:10175800002B3EF4CFADD8F80020013913440132F4
:10176800C8F8002012F8010C01F8010F9342F6D1D5
:10177800FEF7C0BD4F4B1B78DB0700F19F840125A6
:101788000DF0EEF80DF016FF2B46FEF799BD731C11
:10179800C8F8003033780F2B00F29084B21CC8F8D8
:1017A8000020C3EBC303444A7178D154F11CC8F834
:1017B80000101344B2785A70321DC8F80020F2782D
:1017C8009A70721DC8F800203279DA70B21DC8F814
:1017D800002072791A71F21DC8F80020B2795A7186
:1017E80006F10802C8F80020F2799A71012512F072
:1017F80077FB2B46FEF764BD40460AF0B1FD1F4E4D
:10180800F08140460AF0ACFD0125B0812B46FEF779
:1018180057BD40460AF0A4FD284E308240460AF0E3
:101828009FFD708240460AF09BFD0125B0822B4641
:10183800FEF746BD3346721CC8F80020204A13F84C
:10184800021B1170C8F800300C4A73789370F31CAF
:10185800C8F800300A4BB2789A7001252B46FEF77B
:101868002FBD184B184918684E2201252AF057FD3C
:101878002B46FEF725BD00BF5A3200203C3C002015
:101888004C3C00201048002090590020C8590020E6
:101898008C510020044F0020A42F00207C3C002005
:1018A8008C4300205C3C0020803C0020441B00202E
:1018B800183C0020D05A002054330020C04B002090
:1018C800F04E0020EC59002050CD020828C502082F
:1018D8003246731CC8F80030CA4B12F8021B197044
:1018E800C8F8002072785A70F21CC8F80020B27844
:1018F8009A7040460AF034FDC34B0125D8802B4628
:10190800FEF7DEBC40460AF02BFDBF4E3080404655
:101918000AF026FD708040460AF022FD0125B080BD
:101928002B46FEF7CDBCB94F3B78002B3EF4E2AC1A
:10193800B74E002540460AF013FD12F067FF3B78CA
:10194800A6EC010A01359D42F4DBFEF7D3BC0D2B52
:1019580040F0B483731CC8F800303578072D00F2C6
:10196800AD83AC4F40460C260AF0FAFC06FB05F6A0
:10197800BD19A88040460AF0F3FCE88040460AF00A
:10198800EFFCD8F8003028811A46591CC8F8001016
:1019980012F8021BA972C8F800205B78EB72404667
:1019A8000AF0C6FC0125B8512B46FEF789BC731C0A
:1019B800C8F800303078060600F16F86964B1B7821
:1019C800DD073EF597AC032828BF002001250CF061
:1019D800ABFF2B46FEF774BC8F4B1B78D8073EF540
:1019E80089AC01250DF090F80DF0E4FD2B46FEF7CB
:1019F80067BC8A4B1868F31C02462136991EC8F842
:101A0800001013F8031C1170591EC8F8001013F8C1
:101A1800021C5170C8F8003013F8011C9170033390
:101A28009E4202F10302E9D112F0C0FDFEF762BC4A
:101A3800C3F34705122D00F24183BDB10EAB0DF182
:101A4800120703EB45093E46A9F1260940460AF06C
:101A580087FC26F8020FB145F8D1714B37F8022FF1
:101A680023F8022FBE42F9D1112D09D86D4A6B0017
:101A7800023B13440021223223F8021F9A42FBD171
:101A8800694A01231D461370FEF71ABC674E0023EE
:101A9800404633600AF04CFC012530602B46FEF7C7
:101AA8000FBC3346721CC8F8002013F8025BC8F854
:101AB8000030F31C7078C8F80030B178002D00F0C1
:101AC8002386012D7EF416AC23F04EF92B46FEF743
:101AD800F7BB514B1B78D9073EF50CAC544B4FF470
:101AE800C87201251A802B46FEF7EABB4A4B1B78C1
:101AF800DA073EF5FFAB4F4A1378012543F004039C
:101B080013702B46FEF7DCBB092B40F3D7824A4FF4
:101B18003346721C3D68C8F8002013F8022B2A705F
:101B2800C8F800307378AB70F31CC8F80030B3788D
:101B3800642BA8BF6423321D6B71C8F80020F378AA
:101B4800642BA8BF6423721DAB71C8F800203379D9
:101B5800EB71B31DC8F800307379642BA8BF6423F8
:101B6800F21D2B72C8F80020B379EB7006F1080358
:101B7800C8F80030F3792B7140460AF0F1FBD8F829
:101B88000420D8F800306881D11A00290DDD591CCD
:101B98003868C8F80010521A002A1978417204DD12
:101BA8009A1CC8F800205B784370012510F090FB60
:101BB8002B46FEF785BB184B1B7813F0010140F04C
:101BC8007D82731CC8F800303078012523F01CF89A
:101BD8002B46FEF775BB3346721CC8F80020174A1F
:101BE80013F8021BD170C8F80030154A7378537186
:101BF800F31CC8F80030134BB278DA7001252B4675
:101C0800FEF75EBB343C0020742F00207554002082
:101C1800CC2E002060320020D05A0020EC59002041
:101C2800DE2F0020E02F002004300020A4430020F5
:101C3800666A0020CC3F0020D02B00203C3C0020CE
:101C4800104800204C3C002040460AF089FB4046E2
:101C58000AF086FB40460AF083FB40460AF08CFBFC
:101C6800D8F80030C24D1946581C2A68C8F8000038
:101C780011F8020B82F82C00C8F80010597882F885
:101C88003610D91CC8F800109B7882F837304046C7
:101C98000AF072FB40460AF06FFB40460AF06CFB04
:101CA80040462E680AF05CFB708740462E680AF0B2
:101CB80057FBD8F80030D8F804203087D11A01290A
:101CC8000DDD591C2A68C8F800101B7882F82E30E0
:101CD80040460AF051FBD8F80030D8F80420D31A4F
:101CE800032B09DD40462E680AF03AFB7086404611
:101CF8002E680AF035FBB086286895E6731CC8F88C
:101D080000309B4D9B4F33787B7140462E680AF01C
:101D180027FB308440462E680AF022FBD8F80420BE
:101D2800D8F80030F083D11A072915DD40460AF0AB
:101D380017FB788140460AF013FBB88140462E68AD
:101D48000AF00EFB708440462E680AF009FBD8F8AA
:101D58000030D8F80420B084D11A03290BDD40469E
:101D68000AF0FEFAF88140460AF0FAFAD8F800308C
:101D7800D8F804203882D21A002A06DD591C2A68AD
:101D8800C8F800101B7882F826300CF0F3FD1CF020
:101D98004DFF794B1B68002B00F04C842868012507
:101DA80012F0EAF82B46FEF78BBA3346721CC8F8D5
:101DB8000020704F13F8022BBA70C8F800306F4A31
:101DC80073781370F31CC8F800306D4DB3782B711D
:101DD800331DC8F80030F378092BA8BF0923404603
:101DE800AB700AF0BDFAD8F80030D8F80420288083
:101DF800D11A012907DD40460AF0B2FAD8F80030B6
:101E0800D8F80420E8819A4207D05A1CC8F8002064
:101E18001B78003318BF0123FB710CF0ABFDD8F819
:101E28000030D8F804209A423EF464AA5A1CC8F834
:101E380000201B78EB7001252B46FEF741BA33468C
:101E4800721C504DC8F8002013F8022B2A71C8F8EC
:101E5800003073786B7140460AF082FAD8F8003087
:101E680028805A1CC8F800201B78AB7140460AF03D
:101E780077FAD8F8003068805A1CC8F800201B7818
:101E8800EB7101252B46FEF71BBA731CC8F800300E
:101E98003D4B32783D4F1A7000233B6040460AF0B4
:101EA80047FAD8F800203B6839493A4D0343501C9B
:101EB8003B60C8F8000013780B7240460AF050FAED
:101EC800286040460AF04CFA686040460AF048FA32
:101ED800A86040460AF044FA40460AF041FAFEF784
:101EE80009BA2D4B1B78012B3EF604AA731C314608
:101EF800C8F80030294F11F8023BBB70F31CD21A06
:101F0800C8F80010012A7078C8F8003040F3F08350
:101F180040460AF025FA012538802B46FEF7D0B94D
:101F2800731CC8F800303778112F00F2C780B31C33
:101F3800C8F800301A4D737805F8173040460AF093
:101F48000FFA40F6CA039842A8BF184640F2EE239B
:101F5800984205EB4701B8BF18460125A0F2EE22CA
:101F68002B46192092FBF0F24A70FEF7A9B900BF80
:101F7800EC590020F04E0020643C0020303C00204A
:101F8800C04B00208C2F00207C3C00205C3C0020B3
:101F9800305300208C430020E9680020EC680020C2
:101FA800E034002040460AF0DBF9054625F02AF81F
:101FB800FF283EF49FA93F2D00F225830DF1380933
:101FC800002309F8243DEE08494603A88DF80C3093
:101FD80001361EF047FF9DF80C30F6B205F00705F4
:101FE800B34205F1010503D19DF81430AB4203D08B
:101FF8002946304624F0F2FFD8F80030D8F80420FB
:10200800D21A012A7EF776A95A1C0EA8C8F8002011
:1020180000221D7800F82C2D1EF018FF9DF80C30BA
:10202800AB420AD0C44B1B683BB19A79AA4204D38D
:102038001B681B690BB128469847D8F800305A1C12
:10204800C8F80020484600221D788DF814201EF09C
:10205800F1FE9DF81430AB423EF44CA9B64B1B6818
:10206800002B3EF447A91B685B69002B3EF442A98C
:1020780028469847FEF73EB90722B3FBF2F2C2EBB7
:10208800C2055B1B1AD1D2B2571EFFB2002A3EF41A
:1020980031A9DFF8A89201371D46731CC8F8003033
:1020A800A64B96F90010002693F902208A4203F104
:1020B800080300F05D820136062EF5D14FF0FF359A
:1020C8002B46FEF7FDB8731CC8F8003033780E2B8A
:1020D800F4D8B21CC8F8002070780328EED89849C4
:1020E800062202FB03F28B18F51C5871C8F8005041
:1020F800B0788854321DC8F80020F2785A70721DE2
:10210800C8F8002032799A70B21DC8F80020727998
:10211800DA70F21DC8F80020B2791A7101252B4631
:10212800FEF7CEB8731CC8F80030864B32785A7563
:10213800FEF7E0B8731C834DC8F8003033782B7273
:1021480040460AF00DF9A88340460AF009F92883A9
:1021580040460AF005F9D8F800206883531CC8F8EF
:1021680000301278EA74D8F80420D31A032B00F34D
:102178006F82D8F80030D11A052913DD5A1CC8F827
:1021880000201B78EB7240460AF0D2F8D8F80030ED
:10219800E8605A1CC8F800201B782B74D8F8003067
:1021A800D8F80420D21A002A7EF7A4A85A1CC8F826
:1021B80000201B7885F8213001252B46FEF780B8D2
:1021C800614B06F108020136C8F8006016F8011CD8
:1021D80003F8011FB242F6D1FEF78CB83346721CE1
:1021E800C8F80020594A13F8021B9170C8F800304B
:1021F8007378537001252B46FEF762B8544BFEF7EF
:1022080088BC3388FF2BA8BFFF23DBB2FDF7F4BFE0
:102218001FF022FE00283DF4EEAF03780A2B28D8E1
:10222800B0F9023087FB0312DB17C3EBA2039BB2A2
:10223800FF2BA8BFFF23DBB2FDF7DEBF97E8220024
:10224800FEF769BC1FF008FE00283EF44BAC03788B
:102258000A2B3EF647ACB0F90430B0F9061003EB90
:10226800830383F3500521EAE171ADB289B2FEF729
:102278003BBC0023DFE723685A1C226019702988B9
:1022880020460AF0AFF82368EA78591C21601A70D2
:1022980023682A79591C21601A702368AA79591C65
:1022A80021601A7023686A79591C21601A70FEF738
:1022B80027BFDFF8A8B04FF000084FF0080A08F170
:1022C8000108C8F120020AFA02F2A8F120032BFA49
:1022D80008F616432AFA03F31E43B8F1250F06F051
:1022E80001024FF000030CD01343E8D05FFA88F0E6
:1022F8000FF09CFF0028E2D0414648460AF048FA11
:10230800DDE7144B1B78DA0700F1E8800026124F4E
:10231800B04602E00136252E22D0314638460AF072
:1023280047FA0028F6D0314648460AF041FA002814
:1023380074D108F10108EDE78853002008590020FE
:10234800B0430020305300202F530020583C002079
:1023580068230020D05A0020A856002090E33FF4BC
:10236800D34BD44EB3F8501020460AF03BF8D24B6A
:102378001988204689B20AF035F8D04B1A685301FB
:1023880003F02001C2F340030B43C2F3800143EA88
:102398004103C2F3C00143EA8103C2F3401143EA97
:1023A800C10102F01002114320460AF01BF803A9EC
:1023B8000422204609F0E6FF23683178C04A581CF9
:1023C8002060197011886429A8BF642120460AF08A
:1023D80009F8962D00F08780002120460AF002F8BF
:1023E8002168B8F1190348BFA8F11203A3F3C40385
:1023F8004A1C226020461A460B7004A909F0C2FF45
:102408002368B04A581C1021206019701188204692
:10241800012509F0CFFF2B46FDF752BF414603A81F
:102428000AF0B6F985E73346721CC8F80020A64DB5
:1024380013F8022B6A70C8F8003073782B70F31CFD
:10244800C8F80030B378AB70404609F089FFD8F877
:1024580000302881591C1A46C8F8001012F8021BCF
:102468006971C8F800205B78AB7101252B46FDF730
:1024780027BF731CC8F8003033780A2B47D0404672
:1024880009F07AFF404609F077FF0125404609F038
:1024980073FF2B46FDF714BFF4EEC87AF1EE10FA7D
:1024A80080F290804FF47A71FFF704B80827FFF79D
:1024B800A8B82368B978854A581C20601970236821
:1024C8001278591C21601A70FEF7F4BE22680125A3
:1024D800531923602B461070FDF7F2BE059B43F09D
:1024E8000103059312E723680322591C21601A701F
:1024F80023687278591C21601A7071E7404609F008
:102508002FFF734EFEF78DBB0427FFF77AB8B31C75
:10251800C8F800306F4B72781A70F21CC8F80020A7
:10252800B2785A70321DC8F80020F2789A70FDF718
:10253800E1BEF4EEC87AF1EE10FA3EF5D8AF9FEDA1
:10254800667AF4EEC77AFDEEE77AF1EE10FA17EE46
:10255800901A49D86FF4F973303903FB01F140F24E
:10256800E73391FBF3F101F2DB5189B2FEF7A2BF29
:1025780009EBC60A40468AF8021009F0F1FED8F8BD
:10258800003029F836001A46591CC8F8001012F80D
:10259800021B8AF80310C8F800205A788AF8042029
:1025A800DA1CC8F800209A788AF806201E1DC8F898
:1025B80000600135DB788AF80530AF427FF46DADF5
:1025C800FDF798BEFDEEE77A40F2E73317EE901A72
:1025D800303903FB01F140F2CF7391FBF3F101F2C3
:1025E800E93189B2FEF766BF40F2F313A1F58361C2
:1025F80003FB01F140F2E73391FBF3F101F2DD5106
:1026080089B2FEF757BF0DF11409484624F0DAFCE9
:10261800BDF81430AB423FF4EFAC304B1B68002BD5
:102628003FF4EAAC1B689B69002B3FF4E5AC2846F5
:102638009847E1E42A482B492B4A2C4B0360012593
:102648000B6013602B46FDF73BBE0023FFF76DB808
:10265800404609F085FEA884404609F081FED8F876
:102668000030D8F80420E884D11A03297FF783AD15
:102678001A46591CC8F8001012F8021BA977C8F8A6
:1026880000205B7885F82030404609F069FED8F8CC
:102698000030D8F8042068846DE500F07F00032836
:1026A80028BF0020012522F07BFB2B46FDF708BE42
:1026B80010010020DE590020345700208C590020DA
:1026C8007C430020A25500206C5A0020303C00209A
:1026D8002C3C0020BD67002000E082448853002085
:1026E800882D0020DC2D0020442E0020B9B80008D9
:1026F800084BB1781A88012512FB00F22B4692FB91
:10270800F1F23A80FDF7DCBD012511F0C7FD2B463B
:10271800FDF7D6BD9C3A00202DE9F04F2DED028B38
:1027280093B083461BF0E8F9B64B1D7825B113B07A
:10273800BDEC028BBDE8F08FB34B1B685B05F6D58B
:10274800B24FB34E3B68002B57D0B24C3168D4F827
:1027580010218A1A7C2A50D994F81421DFF80083B2
:102768009FEDAD8AC4F81011013284F814214FF09E
:10277800240A5E20984750463B689847A74BF8ECD8
:10278800016A9B8A07EE103AF8EEE66AB8EEC77A55
:102798000AF1010AC6EE877A5FFA8AFA67EE887A42
:1027A800FDEEE77ACDED027ABDF908905FFA89F07F
:1027B8001BF010F9C9F307201BF00CF9BAF1270F29
:1027C8003B68D6D15E2098473B6830209847002068
:1027D8001BF000F900201BF0FDF83B685E209847CD
:1027E80094F8143113F0030800F0868113F00708F9
:1027F80001F03782282B01F02183894B1B78002BAD
:1028080072D0844C874AD4F81831ABEB0303934257
:1028180000F27C8794F82091B9F1000F35D1DFF8E8
:102828004482D8F800000AF08FFEC0B201280FD900
:1028380002287D4F41F081833B78002B41F0FF85D2
:10284800D4F82431ABEB0303B3F57A6F81F07087CA
:10285800D4F82831002B47D094F82031C3B9734BF2
:102868001B689B7801211E3B00228B4284F82011B3
:1028780084F8342141F20387D8F80000022104309B
:102888001BF020F894F82C3111E0D4F828315BB310
:10289800D4F8303140F6B732ABEB0303934223D977
:1028A80094F82C31002B01F0B282DFF8B881013B9B
:1028B800DBB284F82C31002B00F08387D4F8287120
:1028C80094F8342117F8011B94F83531D8F8000032
:1028D800C4F828710A44013384F8342184F8353166
:1028E8000AF036FEC4F830B1514BD6F800801B7898
:1028F80043B1504F386828B14F4B1B78013B012B2F
:1029080040F26F874D4B1B7863B14D4F3B684BB11D
:10291800404CD6F80090D4F84C31A9EB0303632B54
:1029280000F21D81DFF8408198F80030022B01F099
:1029380036823D4F97F87430032B00F02C87414BBB
:102948001B7873B1404D2B685BB1324C0AF080FCA8
:10295800D4F85831029044F61F62C31A934200F229
:1029680059813A4B1B78002B40F08080384B1B78FC
:1029780043B1284CD4F8A83203F5C333A0339B45A0
:1029880080F07286334B1B78002B3FF4D0AE214E7B
:10299800314C324D06F2C92720680AF0D5FD0028CF
:1029A8003FF4C5AE20680AF0CBFD2B7880465A1E4E
:1029B80033B120682A700AF0C7FD0028F2D1B6E6C4
:1029C80003223946781E29F0B5FC96F8C83296F8E5
:1029D800C92286F8CB8283F47F4383F0FF039B1AD6
:1029E8001FFA88F89BB2B8EB132FD5D196F8CA22F4
:1029F800DBB29A42D0D1781E1FF0A8FA2B7818447F
:102A08002870C9E73C45002098510020F046002076
:102A18006C5700201C1D002000007A4490590020AB
:102A2800824700203F0D030000000020EC460020F4
:102A380084470020344500208C470020944700201C
:102A4800E85300209C470020A0470020E0470020D2
:102A5800F1470020A6470020AC470020B0470020DF
:102A6800C8590020E8460020D23000205B4C22786C
:102A7800A2B15B4B9B7A53B10AF0EAFB594B1B6836
:102A8800C31AA3F57A73B3F5FA6F07D82278564BB1
:102A9800564918680AF02CFD00232370544CD4F8CA
:102AA800A03203F5C333A0339B45FFF45FAF514D0C
:102AB800C4F8A0B22B78002B41F004834E4D2B783C
:102AC800002B41F00B824D4994F8A4228D5CE90754
:102AD80001F1BB84AA0701F175846B0701F16D83CD
:102AE800474A94F8A4321178013393FBF1F201FBC1
:102AF800123384F8A43239E7D4F8102141F288332C
:102B08009A4201F2F2813B685E2098473B681420A4
:102B180098473C4B3C4AB3F9043082FB03124FEA16
:102B2800E378C8EBA2080FFA88F85FFA88F01AF081
:102B380051FFC8F307201AF04DFF3B685E20984705
:102B48003B681C20984700201AF044FF00201AF028
:102B580041FF3B685E20984794F8143146E6DFF859
:102B6800A4A0DFF8A48041201AF05AFEBAF9023076
:102B780088FB0320DB17C3EBA00080B21AF036FEF7
:102B8800BAF9003088FB0320DB17C3EBA00080B242
:102B98001AF02CFEBAF9043088FB0320DB17C3EBCC
:102BA800A00080B21AF022FE184B386819780AF093
:102BB800CFFC94F8503113F0010801F0CF81144A8A
:102BC800C4F84C910133DBB2A2FB0312D20802EB2A
:102BD8008202A3EB420384F85031A3E67447002035
:102BE80030530020783F0020E4470020344700207D
:102BF8001C1D0020E8470020E9470020EC47002082
:102C0800F0470020D8590020676666664D540020BA
:102C1800CDCCCCCC94F85E31002B41F05A81DB4B03
:102C28001A6802F00803002B48F603414AF60B40E5
:102C38004BF60F4349F6074704BF03460F4612F009
:102C4800040F4FF0190118BF1F46920684F85E1151
:102C580003D547F4804747F02007CD4B5A79C7F38F
:102C68000909002A41F091859B79002B41F077866C
:102C7800984664204FF0FF3A4FF0000C0A970B97E4
:102C8800ADF834C0CDF83AC0CDF83EC0CDF842C05A
:102C9800CDF83090ADF83680ADF838A08DF8460004
:102CA8000AAF0FCFDFF800E384F805C0AEE80F00E5
:102CB80097E80F00AEE807002EF8023B71464FF088
:102CC800010C1B0CFE271F20C82201F81E39A77013
:102CD800A27184F807C0E07094F86E01207180F04A
:102CE800F10383EA0313DAB2130983F0E70343EA33
:102CF800022383EAC2031BB283EA0312D2B2C3F3EC
:102D0800072383EA121343EA022383EAC2031BB2AE
:102D180083F0C80282EA0212D2B2C3F3072383EA1D
:102D2800121343EA022383EAC2031BB283EA0C07A5
:102D380087EA0717FFB2C3F3072282EA171242EAAB
:102D4800072200EB0C0382EAC7070EEB0C0084F89D
:102D58006E31278011F8013B7B4083EA0313DBB215
:102D68001A0982EA172242EA032282EAC3031BB243
:102D78009FB281422780EDD183F07C0383EA03135D
:102D8800DBB24FEA131E8EEA172E8EEA032E8EEA66
:102D9800C30E0FFA8EFE1FFA8EFADFF810C2A4F8DF
:102DA80000A05FFA8EFE4FEA1A2A84F828A084F859
:102DB80027E00CF5CB7804F12209DCF80000DCF8F8
:102DC8000410DCF80820DCF80C3047460FC70CF17B
:102DD800100CCC45B846F0D1DCF8000038606D4FD7
:102DE8009CF8043088F8043007F1270884F8BDE11E
:102DF80084F8BEA117F8011F28680AF0A9FBB84596
:102E0800F8D194F85F31002B41F05E806249326856
:102E180009780A2084F85F01002901F0C4815F4F16
:102E280001293888069041F2A8850229B7F802E0FE
:102E380001F0C684B8880590032901F09785F888C1
:102E48000490042901F0AE850529388901F0A5858B
:102E58000629B7F80A9001F09C850729B7F80C8075
:102E680001F09485FB89039394F86E110A920B463E
:102E780083F0300282EA0212D2B217094849079356
:102E880087F07A0747EA02270988237187EAC2028E
:102E9800444FC1EB012187FB013A069B4FF0000C20
:102EA80063F30F0C059B6EF31F4C4FF0000E63F39A
:102EB8000F0E049BCDF82CC012B28A440027C91704
:102EC80063F31F4EC1EB6A2A039BCDF830E082EA18
:102ED800021160F30F070020C9B268F30F00C2F3B4
:102EE800072269F31F4782EA111263F31F404FF06C
:102EF80000090D978DF83DA00E908DF83C9042EAA0
:102F080001220DF1280C82EAC107BCE80F003FB28C
:102F180087F0C80888EA0818DFF88CE084F805907C
:102F28005FFA88F8C7F30727AEE80F0087EA181793
:102F380047EA08239CE8030083EAC8031BB283F02E
:102F480023024EF8040B82EA0212D2B2C3F307231B
:102F5800079F83EA1213704643EA022383EAC202F8
:102F680007F1010C20F814194FF023081621FE2749
:102F7800C82384F86EC1228084F807800EF1020EFF
:102F8800A770E170A371114612E000BF8C590020B0
:102F98006C5A0020B31E0020605A002002670020EF
:102FA800583A002003082080241D00201E1D002000
:102FB80010F8013B4B4083EA0313DBB21A0982EA9B
:102FC800112242EA032282EAC3031BB299B2704576
:102FD8002180EDD183F0F40383EA0313DBB24FEAD7
:102FE800131E8EEA112E8EEA032E8EEAC30E0FFAF6
:102FF8008EFE1FFA8EF8E64FA4F800804FEA182CD0
:103008005FFA8EFE84F81EE084F81FC07968BA68FB
:103018003868FB6807F5CB78A8E80F003869796944
:10302800BA6904F29717A8E8070004F2B51884F8FB
:10303800B5C184F8B4E117F8011F28680AF088FAC6
:10304800B845F8D194F866C1BCF1000F40F0368756
:10305800D04B94F86E71B3F90010B3F90220B3F9AC
:1030680004309FEDCD6ADFF840E384F805C007EE31
:10307800103A33680A9387F06A0383EA031306EE6B
:10308800901AD9B20B0983F0D50343EA012383EAE6
:10309800C1031BB283EA03115242C9B207EE902A58
:1030A800C3F3072383EA111343EA0123F8EEE77A0F
:1030B800F8EEE66AB8EEC77A83EAC1031BB267EE98
:1030C800867A66EE866A27EE067A002083F0C808BC
:1030D800CDED0C7ACDED0B6A8DED0D7A0E900F903B
:1030E800109088EA08160DF12809F6B2C3F30728EC
:1030F800B9E80F0088EA161848EA062888EAC608D8
:103108000FFA88F8AEE80F0088F01E0699E8070065
:1031180086EA0616F6B2C8F3072383EA161343EACB
:1031280006238EE8070083EAC6061C20C8214FF054
:1031380005084FF01E0CFE237A1CE070A17184F87C
:10314800668184F807C0A370AEF1100127710EF1F3
:103158000C00268084F86E2111F8013B734083EA45
:103168000313DBB21A0982EA162242EA032282EA30
:10317800C3031BB29EB281422680EDD183F02703A0
:1031880083EA0313DBB24FEA131E8EEA162E8EEA89
:10319800032E8EEAC30E0FFA8EFE1FFA8EFC7C4FAA
:1031A800A4F800C05FFA8EFE4FEA1C2C84F825C0F4
:1031B80084F824E007F5CB7804F1220938687968A7
:1031C800BA68FB6846460FC610374F45B046F5D17A
:1031D800724E3B88A8F8003006F1240784F8BAE15B
:1031E80084F8BBC116F8011F28680AF0B1F9B74284
:1031F800F8D194F867A1BAF1000F40F0598694F815
:103208006E81644B664AB3F90410B2F90620654E24
:10321800DFF898E1644F84F805A088F0220080EA7E
:103228000010C0B2030983F0590343EA002383EA7C
:10323800C0031BB2B2F5FA6F83EA0310C0B2A8BF8D
:103248004FF4FA62C3F30723B2F57A7F83EA1013C7
:1032580043EA0023B8BF4FF47A7283EAC000A2F5AC
:103268007A72642303FB02F28EFB023ED31786FBBD
:103278000162C9174FF0000CC3EBAE13C1EBA201FA
:10328800CDF828C006B2CDF82CC0CDF830C0CDF8A6
:1032980034C0ADF83A30ADF838100DF1280CBCE860
:1032A8000F0086F0C80E8EEA0E1E5FFA8EFEC6F379
:1032B800072686EA1E1646EA0E260FC786EACE06B7
:1032C80036B286F04A0383EA0313DBB2C6F307215A
:1032D80081EA13113A46DCF800E042F810E941EAC5
:1032E800032108F1010681EAC30305204A214FF0B2
:1032F800FE0C84F86E614FF0C80E142684F867013E
:1033080084F8048023800437E17184F802C0E670F1
:1033180084F806E0184612F8011B414081EA0111C1
:10332800C9B20B0983EA102343EA012383EAC101E6
:1033380009B288B2BA422080EDD181F0140181EA45
:103348000111C9B24FEA111E8EEA102E8EEA012E23
:103358008EEAC10E0FFA8EFE1FFA8EF60C4F2680EB
:103368004FEA16295FFA8EFE84F81D9084F81CE057
:1033780079683868BA68FB68B7F8188007F5CB7CB5
:10338800ACE80F0038697969ACE8030010E000BFC9
:103398001E1D0020D859002088C3E43AB31E00201F
:1033A8000267002067666666241D0020D34D621000
:1033B80004F29716ACF8008084F8B391B04684F80C
:1033C800B2E104F2B31918F8011F28680AF0C0F82E
:1033D800C145F8D1C44BC54A1B781278013B12F09D
:1033E8000100DBB214BFC0214021172B03D8C04A0B
:1033F800134493F830A0BF4B1A8893071ABF0023D1
:1034080041F01001012312F4027F18BF022312F0C9
:10341800100F18BF062312F0200F18BF1023002822
:1034280041F060814FF0030C94F86E910A9389F093
:10343800460383EA0313DAB2130983F0920343EADB
:10344800022383EAC2031BB283EA0310C0B2C3F3A8
:10345800072282EA101242EA002282EAC00212B26D
:1034680082F0C80E8EEA0E1E5FFA8EFEC2F30722A5
:10347800002382EA1E1203208DF82CA08DF82FC09D
:103488008DF82D3042EA0E2C8DF82E108DF8300074
:103498000AAA07CA8CEACE0E0FFA8EFEDFF868A2D7
:1034A800E3718EEA0E1CAAE803005FFA8CFCCEF3E7
:1034B800072E8EEA1C1E4EEA0C2181EACC0C94F8E9
:1034C80008E08AF800200FFA8CFC8EEA0C0E8EEACF
:1034D8000E1E5FFA8EFECCF3072282EA1E1242EA23
:1034E8000E22607AA17A94F80BC0637182EACE0248
:1034F80012B2504080EA001E5FFA8EFEC2F3072027
:1035080080EA1E1040EA0E2080EACE0000B2414058
:1035180081EA0111C9B2C0F3072282EA111242EA14
:10352800012282EAC10212B28CEA020C8CEA0C1C5B
:103538005FFA8CFCC2F3072282EA1C1242EA0C22D0
:1035480094F80CE0607BA17B94F8108084F80490D8
:1035580082EACC0212B28EEA020E8EEA0E1E5FFAE0
:103568008EFEC2F3072282EA1E1242EA0E2282EA85
:10357800CE0212B2504080EA0010C0B2C2F3072255
:1035880082EA101242EA002282EAC00212B25140D4
:1035980081EA0111C9B2C2F3072282EA111242EA92
:1035A800012282EAC102E17B13B281EA030282EAC4
:1035B8000212D2B2C3F3072383EA121343EA0223A7
:1035C80083EAC2031BB288EA030282EA0212D2B279
:1035D800C3F3072383EA121343EA022383EAC203ED
:1035E8001BB283F0320282EA0212D2B2C3F307237B
:1035F80083EA121343EA022383EAC2031BB29AB294
:103608004FF0FE0C4FF0090EC82009F10101DBB2A2
:1036180084F802C084F803E04FEA122CA07184F801
:103628006E11228084F812C0637438687968BA68A9
:10363800B7F80C900AF5C47EAEE807000AF5CC7A14
:103648008EF80280AEF8009084F8A8C184F8A731FB
:1036580016F8011F286809F07BFFB245F8D1029BD4
:10366800C4F85831FFF77DB994F8AC32204AC4F851
:10367800A8B202EB8302926C42B312AD04F2B323F8
:103688001D4E45F8203D002104F2C52331800B93DF
:1036980080211523A52784F8B232284684F8B11270
:1036A80084F8B07290472846318808F09BFE0A9D3E
:1036B800124804F52C716D1A152DA8BF15252A4638
:1036C80028F02DFE0E4A94F8AC3215700D4A0133DD
:1036D80082FB0312A2EBE37202EB42029B1A84F80C
:1036E800AC32FFF74FB900BF7C3C0020D05A002015
:1036F80034C502085A3200201C450020383E0020FC
:103708004D3E002056555555241D0020D34AD44B14
:1037180092F80BE03168D4F81C211B88D148891A2B
:103728004FF47A72DFB202FB0EF21B0A8777077535
:1037380091424FF00007C37743758770077180F097
:10374800EE83C94BC9491A689B68C4F818B181FB54
:1037580002E7D21781FB03E1C2EBA702DB17C3EB39
:10376800A10311124FEA232C4FF0F40E0277012720
:10377800417780F8203030217522782380F821C0E5
:1037880080F81AE0C77680F8221080F8232080F8A5
:103798002430FFF73FB8DFF8F492D9F8000009F0B9
:1037A800CBFE00283FF4CBA8D9F80000012109F08E
:1037B800BFFE0222002387F8742088F80030FFF744
:1037C800BEB894F8341194F83531D8F800004A1C82
:1037D800013384F8342184F8353109F0B9FEFFF754
:1037E80081B8A34CDFF8A8924FF0000A0AE01B2B1F
:1037F80000F002830D2B00F012824FF0010389F8CC
:103808000130386809F0A0FE002838D0386809F07F
:1038180097FE83B27E2B32682AD099F801100029CE
:10382800EFD194F83621002AE1D07D2B00F00C82EC
:1038380094F844E1BEF1000F04D080F02003DBB21D
:1038480084F84411511CC9B22244092984F836115C
:1038580082F8383100F0EC810829D2D8B4F8422136
:10386800134403EB132303F0FF03A4F84231C8E722
:1038780084F836A184F837A189F801A0C1E794F843
:10388800453133B194F8393184F84501302B00F0D3
:103898001D8794F83721774BDFF8F8C1DFF8F8E196
:1038A800DFF8F8A10127104600283FF42BA832685A
:1038B800A2EB0802012A00F2AD8194F84691B9F111
:1038C800000F40F0B08294F8471133F8112012B974
:1038D80084F84771E8E70131B2F5826F84F847113F
:1038E80000F002811FD9B2F5E26F00F09A8034D956
:1038F800B2F5046F00F0A480B2F5116F00F04781B3
:10390800B2F5E46FD0D110465B4A176C918A6423F4
:1039180003FB07F393FBF1F119F0BAFF002384F8D6
:103928003731FEF7EFBFB2F5007F00F0B9802CD831
:10393800B2F5807F00F04581B2F5887FB4D1DCF81C
:1039480000205207B0D500214FF4887019F0A0FF6D
:10395800002384F83731FEF7D5BFB2F5C06F00F009
:10396800B380B2F5E06F9FD1434A906B918A64238C
:1039780003FB00F34FF4E06093FBF1F119F088FFCB
:10398800002384F83731FEF7BDBFB2F5047F00F09D
:103998002781B2F5806F87D194F848310133DBB2C3
:1039A800032B00F2588142F2107184F8483101FB70
:1039B80003F1324B1B88002B40F04B810131304B17
:1039C8001B78DF072F4B1B8848BF0431D80748BF37
:1039D8000A319A0748BF14311F0648BF2831D80555
:1039E80048BF28315A0748BF64311F0748BFC8314C
:1039F800980548BF01F5C8719A0648BF01F57A7164
:103A0800DF0648BF01F5FA61580648BF01F57A613B
:103A18004FF4806019F03CFF002384F83731FEF73B
:103A280071BF1046144AD76B918A642303FB07F3CE
:103A380093FBF1F119F02CFF84F83791FEF762BF80
:103A4800114BB3F9041001EB81011046490019F03C
:103A58001FFF84F83791FEF755BF00BF4C55002073
:103A680044550020B447002020450020676666665C
:103A78001C1D002034C5020890590020A2550020C2
:103A8800D05A00205A320020D85900203031002066
:103A9800000000208C5900206C5A00205A55002044
:103AA8009EF8061000293FF4FFAEC84BC8491B68B2
:103AB800104681FB0321DB17C3EBA10119F0E8FED7
:103AC80084F83791FEF71EBF9EF80620002A3FF4BF
:103AD800EBAEBE4B4FF4C060996819F0D9FE0023D5
:103AE80084F83731FEF70EBFDCF8002012F0200909
:103AF8007FF4DAAEB74A1168090600F1C985B64AFB
:103B0800127B002A3FF4D0AE94F84911032900F241
:103B18006686DFE801F032281902B04B1B68597934
:103B28009A79DB7901F1407101EB022101EB034144
:103B3800002384F849314FF4826019F0A9FE00236C
:103B480084F83731FEF7DEBEA54B1A68137A507930
:103B580092781B0403EB002313444A1C84F8492180
:103B680003EB0161E7E79E4B1A68D3791079527825
:103B78001B0403EB00231344EFE7994B1A6893796E
:103B8800D07812781B0403EB00231344E5E79EF872
:103B98000520002A3FF488AE9AF8001000293FF467
:103BA80083AE904B1B8803EB83035B004FF41160DB
:103BB80093FBF1F119F06CFE002384F83731FEF71E
:103BC800A1BEDCF8002051077FF56EAE00214FF44E
:103BD800807019F05DFE002384F83731FEF792BE3D
:103BE8009EF80520002A3FF45FAE9AF800100029DD
:103BF8003FF45AAE784B5B7B002B00F06F85794B16
:103C08001B8893FBF1F101EB810149004FF404702B
:103C180019F03EFE002384F83731FEF773BE4FF0EB
:103C2800010184F8361184F83831A4F84221E8E516
:103C3800B4F84221C2F1FF0293427FF4DEAD4FF0A7
:103C4800010384F84531D8E54FF0010384F8443185
:103C5800D7E50231B3E6012384F8483142F2107106
:103C6800A7E63B685E2098473B6802209847FF20FC
:103C78001EF0F2F80378FF2B00F0258590F901304B
:103C88004FEAE3785FFA88F8D8B219F0A3FE404605
:103C980019F0A0FE3B685E2098473B6803209847D0
:103CA800FF201EF0D9F80378FF2B00F00785B0F944
:103CB8000830D8B2C3F30729DFF8348119F08AFE37
:103CC800484619F087FE98F80530002B40F0A78287
:103CD8000AA9454819F044FE3B685E2098473B68AE
:103CE80013209847BDF928805FFA88F019F072FE12
:103CF800C8F3072019F06EFE3B685E2098473B68C2
:103D08001B209847BDF92A805FFA88F019F062FEF7
:103D1800C8F3072019F05EFE3B685E2098473B68B1
:103D2800232098474E2019F055FE002019F052FE26
:103D38000AA92D4819F014FE3B685E2098473B6895
:103D480012209847BDF928805FFA88F019F042FEE2
:103D5800C8F3072019F03EFE3B685E2098473B6891
:103D68001A209847BDF92A805FFA88F019F032FEC8
:103D7800C8F3072019F02EFE3B685E2098473B6881
:103D880022209847452019F025FE002019F022FE30
:103D98003B685E20984794F81431FEF72BBD09F074
:103DA80057FA124B1B68C01A40F6B833984200F213
:103DB800CA80DFF840A09AF804303A2B00F08F83CD
:103DC800002388F80030FEF7BABD00BF2045002068
:103DD80067666666985100204C550020D02B00205D
:103DE800EC5900204455002080969800D8300020D7
:103DF8006C5A0020C0300020386809F0A5FB002864
:103E08007FF4FBAC4FF0010384F83731F9E4C4F8D0
:103E1800283184F82031DFF8A48219F087FD94F85E
:103E28002C31FEF744BD974906201EF019F90023EE
:103E380084F8460184F83731FEF764BD4FF0000975
:103E48003B6884F814915E203468DFF874829847E0
:103E58003B6817209847484619F0BCFD8A4BA3FBDE
:103E680004239B0BA8FB03125209C2EB0212A3EB1B
:103E78008203D8B219F0AEFD3B685E2098473B68D4
:103E880018209847814BA3FB04239B09A8FB031226
:103E98005209C2EB0212A3EB8203D8B219F09AFDC1
:103EA800484619F097FD3B685E209847FEF7A5BC89
:103EB8000AF1FF3A84F867A1FFF7D1BB0CF1FF3C88
:103EC80084F866C1FFF795B9013B84F85F31FFF7C5
:103ED800B9B8013B84F85E31FEF793BF6C493A20CC
:103EE8001EF0BEF82870FEF741BD3B685E2098477B
:103EF8003B6810209847404619F06CFD404619F081
:103F080069FD3B685E2098473B68212098474046FA
:103F180019F060FD404619F05DFDFEF7F4BD5D4BFC
:103F280032681B78C4F81C21013B012B3FF609AC11
:103F3800102202238270037103E419F0E7FC0123C5
:103F48003B70FEF785BC544AB2F852310021013368
:103F5800A2F8523188F80010FEF7F1BC4F4B1B88CD
:103F6800DA0515D4D80600F12784990600F13384C0
:103F78005A0600F13F84180700F14984D90700F177
:103F8800E38413F0020F0CBF4FF004084FF00C0845
:103F9800434B444A1B78D27803F001030AB143F03B
:103FA80002035320029319F03BFC3F4A128802EBAC
:103FB800820202EB8202900080B219F017FC002006
:103FC80019F014FC394A3A4912883868C2EBC2120F
:103FD800520081FB023111444FEAE27ACAEB612AAE
:103FE8005FFA8AFA514609F0B3FA324B38681A7800
:103FF800029B48EA03082F4B8AEA020A002183F849
:1040080000A009F0A5FA4146386809F0A1FA294B41
:10401800284A1B78386888EA0303DBB2194613700C
:1040280009F096FA94F85031002B7EF4C8AD4F2071
:1040380019F0F6FB1DF054F91DF052F91DF050F976
:104048000121386809F084FA1B4A1A4B92F800805B
:104058001B78184A386808F0010883F001034146C4
:10406800137009F075FA134B124A1B78386888EAFE
:1040780003031946137009F06BFA94F85031FEF7F0
:104088009EBD00BF91D8010873B2E745D34D6210B9
:1040980081DA0108784300201C1D00205A320020D4
:1040A800D05A0020385A002044550020583A0020A1
:1040B800030820804D540020CC3F0020E846002013
:1040C80089888888AE4EAF4B00930024A6F13F0143
:1040D800AD4BAE4A089106F8404CAD4909960AA87E
:1040E80008F058FA089E731C08933470089B29221C
:1040F800591C08911A70089BEA22591C08911A70D9
:10410800089BC822591C08910AA81A7025F0D8F8EB
:10411800471C0AA93A46089828F001F9089AD319C1
:1041280001330893D455089B5A1C08921C70089BAD
:104138005A1C08921C70089B5A1C08921C70089BF9
:104148005A1C08921C70089B5A1C08921C70089BE9
:104158005A1C08921C70089B5A1C08921C70089BD9
:104168005A1C08921C70089B5A1C08921C70089BC9
:104178005A1C08921C70089B5A1C08921C70089BB9
:10418800FF22591C08911A70089B0122991812A83D
:1041980008911A7050F8283D9B1B337019F03CFCAD
:1041A8002C70FEF7E3BB88468946084604910591C2
:1041B8008E4606910391FEF757BE764A704B1268F9
:1041C8000B93A3F1400500202121D70003F8400CF0
:1041D800A97040F1CE8270490326704B1B885805A0
:1041E80000F1C482DA0700F1F38203F002036C4A9B
:1041F800002B1CBF032611466A4F3246384628F06A
:104208008EF8F31912A80133B91E40F8203D002298
:104218005B1AF2556B7019F0FFFBFEF761BC624B3D
:1042280093F800A0BAF1000F3FF452AD5F4AB4F81A
:1042380016E111883B6802924FEA0E1E64201FFAAD
:104248008EFE00FB01A14FEA4A00B1FBF0F14EEAF5
:10425800012E1FFA8EFEC1F303215E204EEA0109EA
:1042680098473B68062098475FFA89F019F0B2FB37
:104278004FEA192019F0AEFBB4F81631029A4C49EE
:10428800B2F800904A7A01339BB2012A93FBFAF004
:104298000AFB1033A4F8163100F0BD826E2345489E
:1042A8004A7B03FB09F380FB03014FEAE379C9EB7F
:1042B800A1092AB13C4B1FFA89F91B7899FBF3F93C
:1042C8003B68DFF8FCA05E2098471FFA89F93B6835
:1042D8003A209847AAFB093A4FEA5A1A1FFA8AF372
:1042E800D8B2029319F076FB029B180A19F072FBF8
:1042F8003B685E2098473B683B209847642303FB54
:104308001A939BB22C48053380FB0320DB17C3EBC1
:10431800A000C0B219F05EFB002019F05BFB3B68FF
:10432800DFF898A0DFF890905E2098473B68282037
:104338009847DAF8003089FB0329DB17C3EBA90992
:104348005FFA89F019F046FBC9F3072019F042FB20
:104358003B685E2098473B6804209847B8F80830C7
:10436800002B40F04B82DAF8083083F310085FFA2C
:1043780088F019F02FFBC8F3072019F02BFBA7E4EE
:1043880034470020E359002014EC02081CEC020812
:1043980028EC0208043C002000EC02085A320020F5
:1043A80010EC0208F74600205A550020445500201A
:1043B8004C550020310CC3306766666620450020E6
:1043C8001F85EB51CC4ACD4B0B9212AEA2F13D00AA
:1043D80046F8200D1988CA4FA2F1400300204FF07B
:1043E8000A0E02F8400C082283F801E030469A7061
:1043F80007F0D2FF3B68C349DA1781FB0313C2EB0E
:10440800A30399B2304607F0C7FF0BF043FEBF681D
:104418000A9B3A0C591C0A911A700A9B3A0A591CB1
:104428000A911A700A9B5A1C0A921F700A9B5A1CFE
:104438000A921870304619F0EFFAFEF74EBBC4F82E
:1044480024B187F80090FEF703BAAF4F9FEDAF8A0B
:10445800B7F90220A8480B9007EE902AF8EEE77A01
:1044680012AE67EE887AA0F13D01FDEEE77A46F8D4
:10447800201D00F8403C0823CDED027A00F83F3CAF
:104488001E23BDF8081000F83E3C304607F084FFB4
:10449800B7F9003007EE903AF8EEE77A304667EE63
:1044A800887AFDEEE77ACDED027ABDF8081007F0BC
:1044B80073FFB7F9043007EE903AF8EEE77A304622
:1044C80067EE887AFDEEE77ACDED027ABDF808103E
:1044D80007F062FF304619F09FFAFEF7FBBA9AF828
:1044E8000240C4B1013CE4B20134544451460022B4
:1044F80011F8013B534083EA0313DBB2120ADF00D1
:1045080042EA03228C4287EA131382EA0302EFD1BC
:10451800002A7FF455AC794A7D4F794B12887D4C3F
:10452800FA61DFF804921A68FA629B68B4F85221BB
:10453800F8660021FB64D9F80000F963FA6508F011
:10454800D7FC029000287EF4F5A90221D9F80000D2
:1045580008F0EEFF94F854319AF803200392642B84
:104568004FF0040287F8742040F0648194F85531C4
:10457800072B04BF9DF8083084F8553194F855315D
:10458800069307EB031ADAF804100291084624F0A0
:1045980097FEDAF8081005915FFA80FA084624F0C9
:1045A8008FFEC0B204900AEB0002069B5A4802999B
:1045B80002900832C27123F00F0286468272049874
:1045C80003F00F0300EBCA008EF80D3052468EF848
:1045D8000E000EF10F0027F0A2FE504B049A059929
:1045E8000AF10900184427F09AFE0298C37903F1EA
:1045F800010ACBB1013B5FFA83FC0CF1080CDFF830
:104608002CE184440023073010F8011B59408B002B
:10461800CA0883EA410302F018024B404EFA02F23C
:1046280053408445DBB2EFD13C4A03980AF8023084
:104638001CF024FE94F855310022013384F85531DA
:1046480084F85421029BDDF808A09B785BB11AF826
:104658000510D9F8000008F07BFF01359AF8023000
:10466800EDB2AB42F3D894F854310322013384F805
:10467800543187F8742088F80020FFF78EB802219B
:10468800D8F8000008F054FF94F82C31FEF70FB961
:104698001023042218460AA98DF82A908DF82B9029
:1046A8008DF82C908DF82D908DF828308DF82920D4
:1046B80019F0CEF884F83791FEF724B94FF00009C5
:1046C8004846FFF7F9BA4046FFF7DFBA1449881F92
:1046D80018F098FF84F84601FFF7DBB8074B1988F4
:1046E800FFF791BA0F4AD278002A0CBF4FF0040C9A
:1046F8004FF0050CFEF798BE3447002044550020C3
:104708002045002067666666D859002058A08B416E
:10471800000000201C1D0020C0530020C6530020AC
:104728005C1E0020385A0020303100200007090E96
:104738000123D8F800003B7008F002FF0746D8F8BC
:10474800000008F0FDFE7F067EF482A88E287EF425
:104758007FA894F82031002B7EF497A8944BC4F8D6
:1047680028312D2384F82C31FEF779B80326914996
:1047780042E5914B914A1B68914903F480038342B7
:1047880016BF11460426032627E58E499A790B8819
:1047980003EB830303EB83034FEA83081FFA88F8CC
:1047A800002A00F0D580884B1B680FFA83FA0BF0BB
:1047B80071FC40B2FEF760BA4FF03408FFF7E8BB6F
:1047C800984699461846049305930393FEF74CBB05
:1047D8007E49042610E54FF02408FFF7D9BB4B1C8F
:1047E800DBB2042B84F849314FEA01617FF4A3A9B5
:1047F800FFF79EB94FF01008FFF7CABB0BF04AFC51
:1048080019F0E8F8002019F0E5F8FFF761BA4FF061
:104818002008FFF7BDBB3B685E2098473B683920FE
:1048280098475FFA89F019F0D5F84FEA192019F07E
:10483800D1F874E597F875A0654904951AF00F0F3B
:1048480004BF0AF1010A5FFA8AFABAF1070F28BF12
:104858004FF0010A4FEA0A1C07EB0C03187C5D4B6A
:1048680002930A18002392F824105A4A93725FFAA6
:104878008CF31A46584B964607EB0C024EEA00009A
:1048880001291870D26803F101000CD90239C9B2A4
:104898008D1C1D44034603F8012BAB424FEA12223C
:1048A800F9D101310844BC4422F060030AF1010A3D
:1048B8009CF811205FFA8AFA1343BAF1080F0370C3
:1048C80000F1010347D04FEA0A1C07EB0C01424AEA
:1048D800087C3F4901449A1A91F8241055180EF1A2
:1048E800100E132D5FFA8EFEC6DD049D0298DFF8C8
:1048F800F0E0D1B28B1DDBB243F04002C27103F18C
:10490800010CCBB14B1DDBB20833C31804930EF175
:104918000100002310F8011B59408B0083EA410372
:10492800CA084B402D4902F0180241FA02F25340DE
:10493800049A8242DBB2EDD103980CF80E3087F866
:1049480075A01CF09BFC7DE64FF00808FFF720BB24
:104958004FF0FF3329E7204A049D9A1AC6E71A4BFD
:104968009046B3F900A06420FEF786B998469946A8
:10497800184604930393FEF777BA98469946184663
:10498800049305939E460393FEF76EBA0393FEF7CE
:104998006BBA98460393FEF767BA9846994603930D
:1049A800FEF762BA9846994618460393FEF75CBA32
:1049B800B447002004EC02089851002000EC0208DB
:1049C800F8EB0208445500202045002008EC0208B6
:1049D80034C50208C0530020CD5300200007090E3B
:1049E800C65300202DE9F04F2DED0C8B3C4B1B7866
:1049F80095B0012B099001F06D863A4C94F800218E
:104A0800002A41F0C180072B374D01F05E86002354
:104A180005936B6834489847002800F06981B5F819
:104A2800B470002285F85520002F40F04387B5F96F
:104A38003E00AA6AB5F93C60696AB5F94030DFF80A
:104A4800B4B0821AE86A6A63711A1B1A2963274884
:104A580095F85610AB6317F021F8DBF80030990091
:104A680040F1F080D5ED0D5AD5ED0C7A204A94ED41
:104A7800656AD4ED666A94ED677AD4F8A031126855
:104A8800B8EEE58AD5ED0E5AF8EEE77AF8EEE58A43
:104A9800013377EE867A38EE268A78EE878A934253
:104AA800C4ED657A84ED668AC4ED678AC4F8A031DE
:104AB80001F0D0830A4B1F78142F02F011870023CE
:104AC800D4F8A8610693062E00F2AF80DFE816F04E
:104AD800D81535156A149D1614004915CE1400BF53
:104AE80094540020E81F0020044F0020344F002079
:104AF800D03F002098510020D84B1A78D4F8ACE168
:104B0800DFF8D0C39FEDD67A4FEACE000CEB000356
:104B180083ED007A002A7DD0D249B0EE476AF0EEE4
:104B2800476A0023F1EC017A013367EEA77A05EEB4
:104B3800903AB4EEE77AF1EE10FAF8EEE55AB8BF1B
:104B4800B0EE677A934276EEA76AA7EEA56AE9D136
:104B5800F5EEC06A0CEB0003F1EE10FA83ED007A73
:104B680058DDC6EE265AC04BC04A1288F7EE007AC6
:104B780075EEE75AD3ED007A65EEA77AFDEEE77A8F
:104B880017EE903A812B43F303859342A8BF13464F
:104B980007EE903AF8EEE77AB54B00EB0E0103EB1F
:104BA800810393ED057AD3ED003A93ED066A93ED10
:104BB800014AD3ED046AD3ED034A93ED025AA3EEFA
:104BC800A77AA4EE276A66EEC76AA7EE646ABDEE06
:104BD800C77AE5EE276A17EE101A812983ED056A70
:104BE800C3ED066A43F3D1848A42A8BF0A4607EE9A
:104BF800902AF8EEE77AFCEEE77ACDED077ABDF871
:104C08001C300CEB00029380BEF1000F02D1132F71
:104C180004F01E81152F42F01A846044DFF8B88230
:104C2800838828F81E30D4F8A861924B013683FB9C
:104C380006239A19F317C3EBA203C3EBC303F61AAF
:104C4800C4F8A8618C4B1B78002B01F0A3808B4E15
:104C5800DFF88892DFF880A206F5BC780027884B39
:104C6800D5ED087A1B78172B01F08E8396ED007A24
:104C7800B8EEC78A082B28EE278A07D1B0EE480A73
:104C8800069325F059FA069B2AF81700DBF800204E
:104C980092000BD5002F04F01E84B0EE480AD5F818
:104CA800143208F170009847B0EE408AB0EE480A16
:104CB800D5F83431A8F170009847D5F8A4314046AA
:104CC80098476F4B1B78032BB0EE408A01F0568350
:104CD800D6F8F800D5F8B830B0EE480A984701374A
:104CE800032F08F12408A9EC010A06F10406B6D13D
:104CF800634B93F80090B9F1070F00F0988694F889
:104D0800B831002B40F0A0865E4B5B79002B40F059
:104D1800CB8501235A4A84F8B8311278072A02F061
:104D2800238000230B93584B94ED709A93ED007AEF
:104D3800564BD4ED6FCAD3F800A0554B0693F7EE47
:104D4800007A37EEC9CA534B08932CEE07CA524B68
:104D58000A93B4EEE7CA514B07930025F1EE10FA17
:104D68004F4BDFF87C91DFF87CB1DFED4E8A9FED89
:104D78004EAADFED3BBADFED4D9A9FED4DBADFED60
:104D88004DAADFF864814C4F059388BFB0EE67CA1F
:104D98002E464A4B99ED008A2B44D3ED007AF5EE66
:104DA800407AF1EE10FA17D0454B2B44D3ED006A48
:104DB80038EE667AB0EEC76AF4EEC67AF1EE10FA0B
:104DC80008D5B5EEC07AF1EE10FACCBF37EEA68A58
:104DD80036EEE78A83ED008A069B1A88930700F06F
:104DE8008580022E00F082809AF82E10354B07EE4F
:104DF800901A2B4493ED007A4B42F8EEE76A07EEDF
:104E0800903A26EE877AF8EEE77AB4EEE77AF1EE92
:104E180010FA0AD407EE901AF8EE677AF4EEC77A19
:104E2800F1EE10FA88BFF0EE477A274B274903EBDB
:104E3800460331F91600B3F90C30C01A07EE100A10
:104E4800B8EEC77AD007E7EE687A40F10586204BBE
:104E580093ED008A27EE888A48E000BFD63F0020FD
:104E680000000000E81F0020D83F0020D43F0020A9
:104E78000C42002093244992CD3F0020344F00205B
:104E880094540020F04E0020982E0020EC59002069
:104E98005A32002078000020D05A00208851002083
:104EA800343A0020CDCCCC3DAE47813F0000C8420B
:104EB80000003443610BB63B403A00208C2E0020A2
:104EC800AC210020542100203C3C0020D85900206F
:104ED800742E0020F4410020985400208C510020AA
:104EE800EC200020842D00204C3A0020079B94F8E9
:104EF800D0212B44D3ED01DA38EE6DDA002A3DD00B
:104F0800D24BD4F8D42109991B688A1A9A4235DD04
:104F18009AF84830022B01F09B87022E04F0588241
:104F2800CB4B1B68990740F11C87CA4BCA49DFF86D
:104F380090E331F916C09EED008ADFF888E3C7EDEB
:104F480000BA03EB460028EE288AB0F90C00A0EB63
:104F58000C0007EE900AF8EEE77ADEF8000027EE7C
:104F6800888A904238EE6DDAC1F22681F7EE007A2F
:104F7800B4EEE79AF1EE10FA01F1F580B74B2B4445
:104F880093ED000A059B2CEE800A022E20EE0D0AF6
:104F9800A3EC010A059304F0A881089B9BED007A15
:104FA800D3ED007AAE4BD7ED006A93ED006AAD4BB6
:104FB80067EE277A2B4427EE8C7AD3ED007A67EEDA
:104FC800277AF0EE665AE7EE8D5AB1EE467AB4EEDD
:104FD800E57AF1EE10FA08DCB4EEE56AF1EE10FAC3
:104FE8008CBFB0EE657AB0EE467A94ED706AF7EE53
:104FF800007AB4EEE76AF1EE10FAACBF01230023A1
:1050080043B1F0EEE66AF0EEC77AF4EEE67AF1EE36
:1050180010FA01D587ED007A022E04F04081924AF9
:10502800924B52F826001B68B0EE6D0A9847904ADA
:10503800904B52F826001B6898479AF8373023B1EE
:10504800069B1B88002B00F06B85B0EE6B8A8A4BA1
:105058009BED007A38EE400A2B4493ED008A83EDED
:10506800000A9AF8483030EE480AC0EE077A2BB3A7
:105078000A9B1B78DB0721D5B7EE007AB4EEC79AF6
:10508800F1EE10FA04DB94F8D031002B00F05587CC
:10509800D4F8D431099AD31A6C4A12689A420DDDB1
:1050A800764B93ED007AB0EECDDAB4EEC7DAF1EED6
:1050B80010FA41F19D80002384F8D031704B94F8A8
:1050C800E0212B4493ED007A2CEE877A67EE277A5D
:1050D800C8ED007A32B9059BC7ED00BA43ED01BAB5
:1050E800C8ED00BA0136032E09F1040908F10408D5
:1050F80007F1040705F104057FF44BAE614B1B78FB
:10510800072B01F03383012B01F01B86002794F84D
:10511800E831002B40F0EF855B4A5C4B10681B6858
:1051280010F4805A93F82C3040F05E86584A59495A
:1051380092ED006A498B584A84ED7E6A92ED007AB6
:10514800564A84ED7F7A07EE901AF8EEE76AD2EDB8
:10515800037A534A84ED7C6A37EE467A77EEE67A2C
:10516800D2ED006A84ED7B7A012284F80022C7EE32
:10517800A65A4C494C4A91ED005A4C499FED4C6A4D
:1051880091ED004A4B49DFED4C6AD1ED004A92EDB2
:10519800007A35EE045AF7EE007AF4EEE75A35EE67
:1051A800245AF1EE10FA88BFF0EE675A25EE065A37
:1051B800F4EEE65AB1EE476AF1EE10FAB4EEC65ACA
:1051C800B8BFF0EE665AF1EE10FAC4ED815A01F15B
:1051D800CE80B4EEC75AF1EE10FA88BFB0EE475A47
:1051E800304ADFED336AD2ED017A304A92ED014A56
:1051F800304A77EE847AD2ED014A77EEA47A67EEE8
:10520800A67AB4EEE76AF1EE10FA08DCB4EEE77AB3
:10521800F1EE10FA8CBFB0EE676AB0EE476A214A29
:10522800DFED236AD2ED027A204AD2ED024A234A00
:1052380077EEA47A92ED007A67EEA67AB1EE473A55
:10524800F4EEC37AF1EE10FA47D43DE0A02E002028
:105258008C5900203C3C0020D8590020482E0020C2
:10526800BC2E0020542E00208C2D0020882D0020DC
:10527800E02D0020DC2D0020C0210020AC2E0020D5
:10528800602E00209454002098510020EC590020F2
:10529800AC3A0020305300200C3C00205C55002024
:1052A8007C2F0020343A0020C02E0020403A0020F5
:1052B8006F12833A4C3A002000000000C42E0020F0
:1052C800742E00209C2E0020F4EEC77AF1EE10FA1E
:1052D8008CBFB0EE473AB0EE673AF04A52780AB956
:1052E800B1EE433A002B41F06283F7EE003AEC4D01
:1052F8002A78002A02F04486EA4BDFEDEB7AD3EDF8
:10530800024AD3ED016A93ED037A66EE244AE5EE8C
:10531800264AE3EE074A63EEA44AF4EEE74AF1EEC2
:1053280010FAB4BFB0EE674AB0EE644A98BFF0EE28
:10533800647A012ACDED0C4A02F0478693ED067A8D
:10534800D3ED052AD3ED076A26EE077AA5EE227A71
:10535800A3EE267A23EE877AB4EEE77AF1EE10FA16
:10536800B4EEC47A8CBFF0EE676AF0EE476AF1EEED
:1053780010FA88BFF0EE676AB4BFF0EE447AF0EE38
:10538800477A022A8DED0D7A00F0DE8093ED0A7AD5
:10539800D3ED092A93ED0B4A26EE077AA5EE227A79
:1053A800A3EE047A23EE877AB4EEE67AF1EE10FAE9
:1053B800B4EEE77A8CBFB0EE664AB0EE474AF1EE3B
:1053C80010FA98BFF0EE446AA8BFF0EE477A032AB5
:1053D8008DED0E7A00F0B88093ED0E7AD3ED0D2A9C
:1053E80093ED0F4A26EE077AA5EE227AA3EE047A09
:1053F80023EE877AB4EEE67AF1EE10FAB4EEE77AA5
:105408008CBFB0EE664AB0EE474AF1EE10FA98BF8C
:10541800F0EE446AA8BFF0EE477A042A8DED0F7AC1
:1054280000F0928093ED124AD3ED112A93ED137A8E
:1054380026EE044AA5EE224AA3EE074A23EE844A42
:10544800B4EEE64AF1EE10FAB4EEE74A8CBFB0EEDD
:10545800667AB0EE447AF1EE10FA98BFF0EE476A39
:10546800A8BFF0EE447A052A8DED104A6CD093ED72
:10547800164AD3ED152A93ED177A26EE044AA5EEBF
:10548800224AA3EE074A23EE844AB4EEE64AF1EE36
:1054980010FAB4EEE74A8CBFB0EE667AB0EE447A02
:1054A800F1EE10FA98BFF0EE476AA8BFF0EE447A22
:1054B800062A8DED114A47D093ED1A4AD3ED192AE1
:1054C80093ED1B7A26EE044AA5EE224AA3EE074A7C
:1054D80023EE844AB4EEE64AF1EE10FAB4EEE74A57
:1054E8008CBFB0EE667AB0EE447AF1EE10FA98BF4F
:1054F800F0EE476AA8BFF0EE447A072A8DED124A0B
:1055080022D093ED1E7AD3ED1D2A93ED1F4A26EE85
:10551800077AA5EE227AA4EE037A27EE237AB4EE70
:10552800E67AF1EE10FAB4EEE77A8CBFB0EE666A6E
:10553800B0EE476AF1EE10FA8DED137A98BFF0EEEF
:10554800466AA8BFF0EE477A77EEE67AF7EE006A89
:10555800F4EEE67AF1EE10FAC4ED707A43F35D8466
:1055680086EEA77A022ADDED0D7A67EE244A67EE09
:10557800877ACDED0C4ACDED0D7A2DD0DDED0E7A82
:1055880067EE877A032ACDED0E7A25D0DDED0F7A06
:1055980067EE877A042ACDED0F7A1DD0DDED107AFB
:1055A80067EE877A052ACDED107A15D0DDED117AF0
:1055B80067EE877A062ACDED117A0DD0DDED127AE5
:1055C80067EE877A072ACDED127A05D0DDED137ADA
:1055D80027EE877A8DED137A344B1E6816F08056C5
:1055E80001F09180F6EE005AC4ED815A002A02F0CB
:1055F800BC842F4BD4ED7F4A93F8038094F9003292
:105608000A99D4ED7E6A91F800E0DFF8B0C0294924
:10561800DFF8AC90B1F906109CED007A059106EE22
:10562800103AFDEEE44A244B99F80090B3F81AB00A
:1056380094ED7B5AD4ED7C7A14EE903AFDEEE64A6E
:1056480000F0100C00F480000EF0010EB8EEC66AEF
:1056580014EE901A0690B8F1000F41F0EB81DFF8D4
:105668004480BCF1000F41F0968098ED007ADDEDA2
:105678000C6ADFF850C025EE877AA6EE267AF0EE9F
:10568800676AE5EE076ABDEEE67A17EE106A17EE6E
:10569800100A9E42A8BF184616E000BF7C3C0020B6
:1056A80075540020EC2E002000000000043C00206F
:1056B800385A00200267002030530020C82E0020EE
:1056C800E44B00206C3A0020B142C8BF084607EE00
:1056D800100AB8EEC77A012A8CED007A00F0DC8057
:1056E80098ED047ADDED0D6A25EE877AA6EE267A26
:1056F800F0EE676AE5EE076ABDEEE67A17EE106A25
:1057080017EE100A9E42A8BF1846B142C8BF084605
:1057180007EE100AB8EEC77A022A8CED017A00F07B
:10572800BB8098ED087ADDED0E6A25EE877AA6EE45
:10573800267AF0EE676AE5EE076ABDEEE67A17EEBE
:10574800106A17EE100A9E42A8BF1846B142C8BF99
:10575800084607EE100AB8EEC77A032A8CED027ADB
:1057680000F09A8098ED0C7ADDED0F6A25EE877AC5
:10577800A6EE267AF0EE676AE7EE056ABDEEE67AEF
:1057880017EE106A17EE100A9E42A8BF1846B142DB
:10579800C8BF084607EE100AB8EEC77A042A8CED8F
:1057A800037A79D098ED107ADDED106A25EE877AC4
:1057B800A6EE867AF0EE676AE7EE056ABDEEE67A4F
:1057C80017EE106A17EE100A9E42A8BF1846B1429B
:1057D800C8BF084607EE100AB8EEC77A052A8CED4E
:1057E800047A59D098ED147ADDED116A25EE877A9E
:1057F800A6EE867AF0EE676AE7EE056ABDEEE67A0F
:1058080017EE106A17EE100A9E42A8BF1846B1425A
:10581800C8BF084607EE100AB8EEC77A062A8CED0C
:10582800057A39D098ED187ADDED126A25EE877A77
:10583800A6EE867AF0EE676AE7EE056ABDEEE67ACE
:1058480017EE106A17EE100A9E42A8BF1846B1421A
:10585800C8BF084607EE100AB8EEC77A072A8CEDCB
:10586800067A19D098ED1C7ADDED136A65EE875A31
:10587800E6EE265AE5EE257AFDEEE77A17EE900A6F
:105888008342A8BF03468142C8BF0B4607EE903A41
:10589800F8EEE77ACCED077ABEF1000F40F03882D7
:1058A800002A40F0308233E2AB4B1B78013BDBB27D
:1058B800FFF730BAA94B07934FF47A761B68B6FB0B
:1058C800F3F3C3EB4316A649DFF8B88291F801A0B9
:1058D800A449B8F9060091F8009003EB8603DE00AE
:1058E800B6B2B74202F0E480D5F88810B5F93CE0CA
:1058F800EB6E4A1C07EE90EA7344012AC5F888202B
:10590800EB66F8EEE77A02F0DE80D5ED1E5AD5EDAB
:10591800206A07EE102A37EEE56AB8EEC75A012F5B
:1059280086EE057A37EE257A77EEC77A85ED1F7A07
:10593800E7EE866A85ED1E7AF0EE667AC5ED216A95
:10594800C5ED206A02F07C84D5F89C10B5F93EE0DC
:105958002B6F4A1C07EE90EA7344012AC5F89C2075
:105968002B67F8EEE77A02F0C780D5ED235AD5ED1C
:10597800256A07EE102A37EEE56AB8EEC75A012FF6
:1059880086EE057A37EE257A77EEC77A85ED247AA2
:10599800E7EE866A85ED237AF0EE667AC5ED266A2B
:1059A800C5ED256A02F08084D5F8B010B5F940E05D
:1059B8006B6F4A1C07EE90EA7344012AC5F8B020C1
:1059C8006B67F8EEE77A02F0B080D5ED285AD5ED8E
:1059D8002A6A07EE102A37EEE56AB8EEC75A012F91
:1059E80086EE057A37EE257A77EEC77A85ED297A3D
:1059F800E6EE276A85ED287AF0EE667AC5ED2B6A21
:105A0800C5ED2A6A02F04484A8F80600B5F8B43057
:105A1800544A013B92F80090A5F8B4300799002346
:105A2800B9F1070F4B608B60CB607FF468A907F072
:105A38000FFC059BDFF84C81C01A94F8B831A8F820
:105A48000000002B3FF460A9013B84F8B83115B081
:105A5800BDEC0C8BBDE8F08F94ED5E7AB1F90000D7
:105A6800D4ED5F6AB1F902E03F4AF4EEC76A80EA12
:105A7800E0738EEAEE71A3EBE073F1EE10FAA1EB9E
:105A8800EE71B8BFF0EE476A8B42B8BF0B4607EE1F
:105A9800103A1378B8EEC77A27EE287A002B40F030
:105AA8001D82324B93ED006AB4EECA6AF1EE10FA29
:105AB80041F1DC80F7EE005A75EEC65A3BEE477AA4
:105AC80065EEAA5A2A4BA7EE256A93ED007A26EED0
:105AD800076AB5EEC06AF1EE10FA40F21086C9EE18
:105AE800865AB7EE007AB0EE476AA6EEE56AF0EE9F
:105AF800466AF4EEC76AF1EE10FA88BFF0EE476A1C
:105B0800F5EEC06AF1EE10FAB8BFF0EE6B6A194B09
:105B180093ED007A67EE877AA7EEA68AFFF7E6B9D3
:105B2800154B164A2B4493ED007AD2ED007A144BAC
:105B380067EE277AF7EE006AF4EEE67AF1EE10FAED
:105B480093ED007A88BFF0EE667A67EE877A27EEE3
:105B5800888AFFF77CBA00BF303C002088510020BB
:105B6800F04E002094540020802E0020882E002023
:105B78007C2E0020782E002060210020702E00202E
:105B88006C2E002098540020072B02F01982002662
:105B9800DFF83CB3B64DDBF80030590501F16B80F6
:105BA800B44B1B78002B40F0F381B34F94F81231BB
:105BB80023B1B24A1288920742F0988194F81821CA
:105BC800002A41F06280BB7F002B00F0F383022B98
:105BD80002F01680032B01F0BE82A94B5B88F97F87
:105BE8000231C9B2002A01F0FC87002B01F0F987C5
:105BF800A4480068B3FBF0F30FFA83F9A4F84891BE
:105C0800002903F0128107EE909AF8EEE77AF7EE92
:105C1800006A86EEA77A9C4B0129D4ED576AD3ED2A
:105C2800007A77EEE67A67EE877AC4ED537A21D068
:105C3800D3ED017AD4ED586A77EEE67A022967EE59
:105C4800877AC4ED547A15D0D3ED027AD4ED596A27
:105C580077EEE67A032967EE877AC4ED557A09D09C
:105C6800D3ED037AD4ED5A6A77EEE67A67EE877A4F
:105C7800C4ED567A85480078092803F00E81B9F1F9
:105C8800000F40F39E8391B394ED577AD4ED537A85
:105C980077EE877A0129C4ED577AC3ED007A21D0CF
:105CA80094ED587AD4ED547A77EE877A0229C4EDC8
:105CB800587AC3ED017A15D094ED597AD4ED557A16
:105CC80077EE877A0329C4ED597AC3ED027A09D0B1
:105CD800D4ED5A7A94ED567A77EE877AC4ED5A7AEB
:105CE800C3ED037A01390229B8BF0221C9B2002ADB
:105CF80018BF022166E30A9B654D1B78DE0700F199
:105D080063812A7822B192006249634826F007FB32
:105D1800624B1B68002B40F02E83614B1B789BB1B4
:105D2800287870B1DFF87081DFF8A8910026F0B20A
:105D3800D9F80030B8EC010A98472878013686422D
:105D4800F5DB584B1B689847504B1B78072B00F026
:105D5800DF84012384F8003115B0BDEC0C8BBDE85D
:105D6800F08F514BC7ED00BA1B689342BFF6FEA8EF
:105D78004E4B1A88002384F8D031002A41F08E86D1
:105D88004B4A4C4B1178186881F0010108F0D6FB9A
:105D9800FFF7F4B8484EDFF8409106F5F47806F5B9
:105DA8001577F6EC017A95ED080AD5F81432F8EE75
:105DB800E77A404627EE800A9847A8F1E000D5F830
:105DC80034319847A8F17000D5F8A4319847D6F82F
:105DD800F400D5F8B830984708F124084745A9ECED
:105DE800010ADED1FEF784BF0A9A1278D50703D4D8
:105DF800214A128BA4F8F421304A2349128891EDE4
:105E0800037A07EE902AF8EEE77AB4EEE77AF1EE35
:105E180010FA41F281802A49098807EE901AF8EEB3
:105E2800E77AB4EEE77AF1EE10FAC0F2E78725498F
:105E3800254AD1ED006A92ED006A2449C4ED7E6AD4
:105E4800BCEEC75A76EE665A15EE102AC4ED7C6A87
:105E5800C4ED7B5A84ED7F6AA4F8F4210122D1EDC8
:105E6800006A84F8002277EE677AFFF780B900BFEE
:105E7800044F0020441B0020305300205A320020D9
:105E8800605A0020643C00205C5500209454002097
:105E980075540020CC2E00206C3A0020C43300201A
:105EA800EC4E0020E04B00209C2E002044570020A0
:105EB8004657002048570020344F0020802F0020EC
:105EC800822F00206C2F00200C3C0020882F0020FF
:105ED80098510020D84B00208C510020CC4B93EDDA
:105EE800005AB5EEC05AF1EE10FA40F30884C94BD7
:105EF800D3ED004AF5EEC04AF1EE10FA40F3FF8305
:105F080034EEC77A66EEE95A87EE246AC5EE856AEA
:105F1800B7EE007AB4EEC76AF1EE10FA88BFB0EEB9
:105F2800476AB5EEC06AF1EE10FA76EE876AB8BF36
:105F3800B0EE6B6A66EE266ADBE5B74A92ED007A48
:105F4800F0EEE76AF4EEC76AF1EE10FA7FF7A0A860
:105F5800B24A92ED007AF0EECD6AF4EEC76AF1EE3D
:105F680010FA7FF795A8AE4A99ED007AD2ED006A4B
:105F7800B0EEC77AB4EEE67AF1EE10FA7FF588A8AB
:105F880001220999C4F8D41184F8D021FFF784B804
:105F9800A44BA54FB3F906207B8B9A423FF706AE78
:105FA800A24B1B78012B01F00786192B01F0048600
:105FB8000E2B3FF4FBAD082B3FF4F8AD9C4B0022B1
:105FC8009A60C4F80C21F1E52B78002B3FF4A0AEC1
:105FD800D4ED5F3A94ED5E6AD4ED7C7A954A94EDFF
:105FE8007B7AD2ED005A94ED5C4AD4ED5B4ADFF837
:105FF8005C82DFF85CC2F4EEC63AF3EE046AF1EEB6
:1060080010FA37EEA65A00F1F78798ED026A26EEE5
:10601800446AF0EE674AE6EE074AF4EEC54A34EE03
:10602800E66AF1EE10FA48BFB0EE656A012B8CED16
:10603800006A3FF46DAE98ED066A26EE446AF0EE0B
:10604800674AE6EE074AB4EEE45A34EEE66AF1EE41
:1060580010FA88BFB0EE656A022B8CED016A3FF436
:1060680057AE98ED0A6A26EE446AF0EE674AE6EE05
:10607800074AF4EEC54A34EEE66AF1EE10FA48BF74
:10608800B0EE656A032B8CED026A3FF441AE98EDE1
:106098000E6A26EE446AF0EE674AE6EE074AB4EE68
:1060A800E45A34EEE66AF1EE10FAC8BFB0EE656A5B
:1060B800042B8CED036A3FF42BAE98ED126A26EEA2
:1060C800446AF0EE674AE6EE074AB4EEE45A34EE64
:1060D800E66AF1EE10FAC8BFB0EE656A052B8CEDE2
:1060E800046A3FF415AE98ED166A26EE446AF0EE9F
:1060F800674AE6EE074AF4EEC54A74EEE66AF1EE40
:1061080010FAB8BFF0EE656A062BCCED056A3FF4CD
:10611800FFADD8ED1A6A66EEC46AF0EE674AE6EE9D
:10612800874AB3EE046AB4EEE45A74EEC66AF1EE36
:1061380010FAC8BFF0EE656A072BCCED066A3FF48B
:10614800E7ADD8ED1E6A26EEC44AE4EE077AF4EE0F
:10615800C57A77EEC67AF1EE10FA48BFF0EE657AA6
:10616800CCED077AD4E50799334BD1ED017A93ED5D
:10617800007AF0EEE77AF4EEC77AF1EE10FA7EF5DF
:10618800FDAED1ED027AF0EEE77AB4EEE77AF1EE01
:1061980010FA7EF7F3AED1ED037AF0EEE77AB4EEBB
:1061A800E77AF1EE10FA7EF7E9AE244B1B689A07FE
:1061B8007FF5DEAD2249234BB3F90C20B1F900E09D
:1061C8002148AEEB020E00688EEAEE72A2EBEE7288
:1061D8008242BEF6D3AEB3F90E30B1F90220D21A1C
:1061E80082EAE273A3EBE27398427EF7C7AEBFE59B
:1061F8000B4B99ED007AD3ED006AB0EEC77AB4EE96
:10620800E67AF1EE10FA7EF759AFFEF754BF00BFF9
:106218007C2E0020842E0020B02E0020AC2E0020E2
:10622800B42E002002670020305300207C3C002060
:106238005C550020C82E0020A82E00208C59002074
:10624800D85900203C3C0020A42E0020EC2E002031
:106258006C3A002007EE103A524BDFF854811B7855
:10626800C4F8A071B8EEC77AF7EE006A132B86EE71
:10627800879AB8F90400B4F8A47195ED080A01F0FA
:106288007583494B494A93ED001A93ED053A93ED0E
:10629800122A93ED176AD3ED091A93ED0E4AD3ED3E
:1062A800015AD3ED063A93ED0A7A93ED0F5AD3EDDE
:1062B800132AD3ED186AD3ED044AD3ED030A67EE27
:1062C800897A69EE288A29EE088AA1EE273A02EB34
:1062D80087060021A2EE286AC4F89411C4F8981120
:1062E800A1EE884AE5EEA73AA7EE085A93ED167A8A
:1062F800D3ED0D5A93ED021AD3ED0C1A86ED003A40
:10630800E2EEA86A64EEC34A27EE467A93ED0B2ABA
:10631800D3ED152A86ED204AE0EEC33A65EEC45A5D
:1063280093ED143AC3ED053AE1EE274AF0EE477AC9
:10633800A1EEC45AE2EE085AE2EEC66AE3EE287A03
:10634800C3ED064A83ED0E5AC3ED0F5A86ED406A37
:10635800C3ED176AC3ED187AC4F89C117B1C03F0CF
:106368001F03A4F8A431A8F80400FEF7A3BBB0EEFD
:10637800465AFEF735BF0FF0F1FFCEE423F0DCFEFE
:106388002AF81700FEF7A4BC96ED007A05EB470241
:10639800B8EEC78A928F2AF8172028EE278AFEF7C8
:1063A80075BC00BF9454002078420020F43F0020C0
:1063B80098540020A4F848319946002A00F07281C8
:1063C800D74B0221D74ADFEDD86A1068D74A90F830
:1063D80002C092F800E0027807EE902AF8EEE77A19
:1063E800B0EE007A67EEA67AF4EEC77AF1EE10FA0C
:1063F80040F30E8337EEC77ADFEDCD6AB0EE676AF9
:10640800A7EE266AB0EE467A9FEDCA6AD3ED006A17
:1064180066EE866AB0EEE66AC4ED5B6A84ED5E6A93
:10642800BCF1000F13D005EE90CAB8EEE55ADFEDC7
:10643800BE5A66EEA64A25EE255AF7EE005A75EEC4
:10644800C55A64EE864AE4EE855A66EEA56ADFED23
:10645800BA5A427927EE257A27EE267ACAB1DFEDB5
:10646800B26ADFEDB65A26EE266A06EE902AF8EEF4
:10647800E66A26EE266AB4EEE56AF1EE10FA00F353
:106488007285F7EE005A35EEC66AC5EE866A27EEC3
:10649800267ABEF10C0F9FEDAA8ADFEDAA6A00F0FA
:1064A8001385B4EEC87AF1EE10FA98BFB0EE478AB9
:1064B800B4EEE68AF1EE10FAB8BFB0EE668A84ED63
:1064C800418A002900F0E280B0EE007AF4EEC77A43
:1064D800F1EE10FA05DD37EEC77ADFED956AE7EEE3
:1064E800267A93ED017ADFED936A27EE267AB0EEED
:1064F800C76A84ED5C7A84ED5F6ABCF1000F13D043
:1065080006EE90CADFED885AF8EEE66A27EE075ADB
:1065180066EEA56AF7EE005A75EEE65A25EE065ABB
:10652800E5EE265A27EE257ADFED836A827967EE53
:10653800A67A67EE877AAAB107EE102AB8EEC77A6C
:10654800DFED795ADFED7D6A27EE067A27EE257AA8
:10655800B4EEE67AF1EE10FA40F30985DFED7A6AD7
:1065680067EEA67ABEF10C0F00F08D84DFED746A39
:106578009FED747AF4EEE67AF1EE10FA88BFF0EE49
:10658800667AF4EEC77AF1EE10FAB8BFF0EE477A01
:106598000129C4ED427A79DD4278DFED636A07EEBE
:1065A800902AF8EEE77AB0EE007A67EEA67A427A99
:1065B800F4EEC77AF1EE10FA05DD37EEC77ADFEDB3
:1065C8005C6AE7EE267A93ED027ADFED5A6A27EEE7
:1065D800267AB0EEC76A84ED5D7A84ED606A9AB176
:1065E80006EE902ADFED505AF8EEE66A27EE075AD3
:1065F80066EEA56AF7EE005A75EEE65A25EE065ADB
:10660800E6EE855A27EE257ADFED4B6AC37967EE09
:10661800A67A67EE877A0BB307EE103AB8EEC77A18
:10662800DFED415ADFED456A27EE067A27EE257A37
:10663800B4EEE67AF1EE10FA0CDCB5EEC07AF1EEC3
:1066480010FA01F1C082B7EE006A36EE477AC6EE5C
:10665800076A01E0DFED3C6A67EEA67ABEF10C0F2F
:1066680000F00784DFED366A9FED367AF4EEE67ABD
:10667800F1EE10FA88BFF0EE667AF4EEC77AF1EE22
:1066880010FAB8BFF0EE477AC4ED437ABEF1090FAD
:1066980000F0D38397F82170002F40F06A8300231D
:1066A80084F81831294B1B7823B9294FBB78002B64
:1066B80041F0AD821D4B1B78072B00F0228400228D
:1066C800072B84F800217EF4A2A906F0C1FD0590ED
:1066D800FEF79FB91F4B204C1A68204BDFF88880C3
:1066E80094F80001D2691B88A8F80020A8F80230A5
:1066F80000287FF44CAA0590194DFEF78AB9DFED02
:10670800196AFFF704BA41023EF56CAFFEF76EBF97
:1067180006F09EFD144BC01BD880FFF71ABB00BFC4
:106728005C550020D02B00200AD7233C945400202D
:10673800D7A368416F12033B00004843A4707D3F14
:1067480000C0F94400C0F9C40000C8423C4500201C
:10675800EC68002024480020E81F00207C4300202B
:10676800044F0020000000009854002006F070FD3F
:10677800A94B0B9A1B78DFF8B482801A012BA8F872
:10678800020000F0E082072B7EF4C0AC06F060FD4A
:106798000746FEF7BCBCBEF1000F41F0438498EDFC
:1067A800007ADDED0C6ADFF888C225EE877AA6EE5E
:1067B800867AF0EE676AE7EE056ABDEEE67A17EECE
:1067C800106A17EE100A9E42A8BF1846B142C8BF09
:1067D800084607EE100AB8EEC77A012A8CED007A4F
:1067E8003FF491AA98ED047ADDED0D6A25EE877ADB
:1067F800A6EE867AF0EE676AE7EE056ABDEEE67AFF
:1068080017EE106A17EE100A9E42A8BF1846B1424A
:10681800C8BF084607EE100AB8EEC77A022A8CED00
:10682800017A3FF470AA98ED087ADDED0E6A25EE3C
:10683800877AA6EE867AF0EE676AE7EE056ABDEE1D
:10684800E67A17EE106A17EE100A9E42A8BF18469D
:10685800B142C8BF084607EE100AB8EEC77A032A45
:106868008CED027A3FF44FAA98ED0C7ADDED0F6AB1
:1068780025EE877AA6EE867AF0EE676AE7EE056A75
:10688800BDEEE67A17EE106A17EE100A9E42A8BF10
:106898001846B142C8BF084607EE100AB8EEC77AD4
:1068A800042A8CED037A3FF42EAA98ED107ADDEDD8
:1068B800106A25EE877AA6EE867AF0EE676AE7EE2A
:1068C800056ABDEEE67A17EE106A17EE100A9E42C8
:1068D800A8BF1846B142C8BF084607EE100AB8EE6E
:1068E800C77A052A8CED047A3FF40DAA98ED147A3C
:1068F800DDED116A25EE877AA6EE867AF0EE676AF4
:10690800E7EE056ABDEEE67A17EE106A17EE100A92
:106918009E42A8BF1846B142C8BF084607EE100AF3
:10692800B8EEC77A062A8CED057A3FF4ECA998ED03
:10693800187ADDED126A25EE877AA6EE867AF0EEF1
:10694800676AE7EE056ABDEEE67A17EE106A17EE9B
:10695800100A9E42A8BF1846B142C8BF084607EEB3
:10696800100AB8EEC77A072A8CED067A3FF4CBA94D
:1069780098ED1C7ADDED136A65EE875AE6EE265A25
:10698800E5EE257AFDEEE77A17EE900A8342A8BF76
:1069980003468142C8BF0B4607EE903AF8EEE77A05
:1069A800CCED077A002A7FF4AEA9FFF7B1B91B4BEB
:1069B8005A79002A3EF499AC194A1278002A3EF412
:1069C80094AC1B78DFED174A07EE903A164BB8EEF9
:1069D800677A1B8807EE902A06EE903AF8EEE77A77
:1069E800F8EE666A67EE277AB7EE007AC7EEA63A3F
:1069F800F4EEE43AF1EE10FA88BFF0EE643AF4EE01
:106A0800C73AF1EE10FAB8BFF0EE473AFEF76FBC9E
:106A1800B0EE677AF8E400BF945400206C5A002066
:106A28005A550020713DAA3F445500209854002033
:106A38006C3A0020BCF1000F00F09783BEF1000F04
:106A480041F07087DFF8A485B9F1000F41F0C885DF
:106A5800D8ED006ADDED0C4ADFF894C565EEA66A4C
:106A6800BDEEC77A17EE101AB0EE667AA4EE867AF3
:106A7800F0EE676AE7EE056ABDEEE67A17EE106A91
:106A880017EE100A9E42A8BF1846B142C8BF084672
:106A980007EE100AB8EEC77A012A8CED007A3FF4A7
:106AA80032A998ED047ADDED0D6A25EE877AA6EE17
:106AB800867AF0EE676AE7EE056ABDEEE67A17EECB
:106AC800106A17EE100A9E42A8BF18468E42B8BF39
:106AD800084607EE100AB8EEC77A022A8CED017A4A
:106AE8003FF411A998ED087ADDED0E6A25EE877A54
:106AF800A6EE867AF0EE676AE7EE056ABDEEE67AFC
:106B080017EE106A17EE100A9E42A8BF18468E426A
:106B1800B8BF084607EE100AB8EEC77A032A8CED0C
:106B2800027A3FF4F0A898ED0C7ADDED0F6A25EEB5
:106B3800877AA6EE867AF0EE676AE7EE056ABDEE1A
:106B4800E67A17EE106A17EE100A9E42A8BF18469A
:106B58008E42B8BF084607EE100AB8EEC77A042A74
:106B68008CED037A3FF4CFA898ED107ADDED106A2A
:106B780025EE877AA6EE867AF0EE676AE7EE056A72
:106B8800BDEEE67A17EE106A17EE100A9E42A8BF0D
:106B980018468E42B8BF084607EE100AB8EEC77A04
:106BA800052A8CED047A3FF4AEA898ED147ADDED51
:106BB800116A25EE877AA6EE867AF0EE676AE7EE26
:106BC800056ABDEEE67A17EE106A17EE100A9E42C5
:106BD800A8BF18468E42B8BF084607EE100AB8EE9E
:106BE800C77A062A8CED057A3FF48DA898ED187AB5
:106BF800DDED126A25EE877AA6EE867AF0EE676AF0
:106C0800E7EE056ABDEEE67A17EE106A17EE100A8F
:106C18009E42A8BF18468E42B8BF084607EE100A23
:106C2800B8EEC77A072A8CED067A3FF46CA898ED7F
:106C38001C7ADDED136A65EE875AE6EE265AE5EE14
:106C4800257AFDEEE77A17EE900A8342A8BF03463D
:106C58008142D8BF194607EE901AF8EEE77ACCEDD4
:106C6800077A002A7FF44FA8FFF752B8C74B93ED75
:106C7800006AFEF72EBFAB68002B3EF491AF05F11A
:106C8800500128469847FEF78BBFC14BC149D3F83E
:106C9800EC30086844F620618B42A8BF0B46B3F578
:106CA8007A7FB8BF4FF47A7399B2C006A4F81A1164
:106CB800DBF8003041F1BF82DB0400F16B83B64B97
:106CC800D3F800C0BCF932E0B44BB548D3ED037A31
:106CD800D4F81C31A0FB01018809642191FBF0F173
:106CE8001429BDEEE77A04EB4308A8BF1421013349
:106CF8008B42C4F81C3117EE109AA4BF0023C4F8C5
:106D08001C3104EB4303A8F82091B3F9203107EEB6
:106D1800103AB8EEC77A77EEC77AFDEEE77ACDED8E
:106D2800057ABDF9141081EAE173A3EBE1737345A9
:106D380002F364809B4B19464FF07E530B60FEF7BD
:106D480042BFDFF8B08206F083FA974AD4F8E431FC
:106D58001268C4F8E401C31A9A1A0746A8F804305E
:106D6800A8F80620FEF7D3B906F072FA0B90FDF7E3
:106D7800DABF1E21874805F01BFD00283FF48FACC1
:106D88008A4B1B885A063FF58AAC94F88431BB427B
:106D980042F0A980834BD4ED627A93ED010AD4EDD9
:106DA800435A9FED836ADFED836A27EEE57A68EE42
:106DB800277AA8EE007AE5EE807AB4EEC67AF1EE8C
:106DC80010FA88BFB0EE467AB4EEE67AF1EE10FA21
:106DD800F4EEC67AB8BFB0EE667AF1EE10FA88BF64
:106DE800F0EE467AF4EEE67AF1EE10FAB8BFF0EE7D
:106DF800667A84ED417AC4ED437A50E4B4F8F4112C
:106E0800914240F282856C496C4AD1ED007A92ED4C
:106E1800007A6B49C4ED7E7A77EE676AC4ED7C7AB6
:106E28000122C4ED7B6A84ED7F7AD1ED006ADFED43
:106E3800657A84F80022FEF79AB9FDEEC87ADFF881
:106E4800B48117EE903AA8F80490A8F8063021E427
:106E58005D4B1B88002B40F077855C4A5C4B1178B2
:106E6800186807F06BFBD4F8D421099B9A1AFEF72F
:106E780054B8BDEEE77ADFF87C8117EE103AA8F82F
:106E88000430FFF7EFBB9FED4A7ADFED4A6ADFF87F
:106E98006481F4EEC77AF1EE10FA98BFB0EE677A23
:106EA800FDEEE77AB4EEE67AF1EE10FA17EE902AE4
:106EB800B8BFB0EE667A012984ED427AA8F80220BC
:106EC8003FF76AABFFF7E6BBB4EEC87AF1EE10FA0B
:106ED80098BFB0EE478ABDEEC77AB4EEE68ADFF80F
:106EE8001481F1EE10FA17EE102AB8BFB0EE668AD8
:106EF80084ED418AA8F8002000297FF4E5AAFFF76D
:106F0800C9BB06F0A5F9DFF8EC80324B801B1B7873
:106F1800A8F80400FFF7D3BB2F4A3049D2ED006A26
:106F28002F4A91ED006A1278C4ED7E6A84ED7F6A7B
:106F3800002A40F0E68476EEC65AF0EE466ABCEEC9
:106F4800C76A2849C4ED7B5A16EE102AC4ED7C6A3C
:106F5800A4F8F421FF22D1ED006A84F8002277EE2C
:106F6800C77AFEF704B9DFED206AFFF790BAB5EEED
:106F7800C07AF1EE10FA00F12A86B7EE006A36EE12
:106F8800477AC6EE076AFFF7EBBA00BF7C2E0020EF
:106F980010010020043C0020EC5900205C55002022
:106FA800D34D621078000020643C00205A32002043
:106FB80000C0F94400C0F9C46C2F00200C3C00202C
:106FC800882F00200000000044570020465700206A
:106FD8004857002094540020AC3A0020702F00201D
:106FE800E44B0020842F00200000C842EC2E002033
:106FF8006C3A00209854002098ED016A26EE646AE5
:10700800B0EE674AA6EE074AB4EEC45A34EE666A92
:10701800F1EE10FAC8BFB0EE656A012B8CED006A7C
:107028003EF476AE98ED056A26EE646AB0EE674ADD
:10703800A6EE074AB4EEC45A34EE666AF1EE10FAC8
:10704800C8BFB0EE656A022B8CED016A3EF460AEF3
:1070580098ED096A26EE646AB0EE674AA6EE074A1A
:10706800B4EEC45A34EE666AF1EE10FAC8BFB0EE58
:10707800656A032B8CED026A3EF44AAE98ED0D6A00
:1070880026EE646AB0EE674AA6EE074AB4EEC45A22
:1070980034EE666AF1EE10FAC8BFB0EE656A042BEA
:1070A8008CED036A3EF434AE98ED116A26EE646AFC
:1070B800B0EE674AA6EE074AB4EEC45A34EE666AE2
:1070C800F1EE10FAC8BFB0EE656A052B8CED046AC4
:1070D8003EF41EAE98ED156A26EE646AB0EE674A75
:1070E800A6EE074AB4EEC45A74EE666AF1EE10FAD8
:1070F800C8BFF0EE656A062BCCED056A3EF408AE13
:10710800D8ED196A66EEE46AB0EE674AA6EE874AD9
:10711800B3EE046AB4EEC45A74EE466AF1EE10FA9D
:10712800C8BFF0EE656A072BCCED066A3EF4F0ADF9
:10713800D8ED1D6A66EEE44AE4EE877AF4EEC57A85
:1071480077EEC67AF1EE10FAB8BFF0EE657ACCEDBC
:10715800077AFEF7DDBD97F82030C3EB431103EB48
:107168008103DB009BB2FEF73ABDDFF80485B9F175
:10717800000F41F0CB80D8ED006ADDED0C4ADFF856
:10718800F4C465EEA66ABDEEC77A17EE101AB0EE23
:10719800667AA4EE867AF0EE676AE7EE056ABDEED7
:1071A800E67A17EE106A17EE100A9E42A8BF184634
:1071B800B142C8BF084607EE100AB8EEC77A012ADE
:1071C8008CED007A3EF468AB98ED047ADDED0D6A3B
:1071D80025EE877AA6EE867AF0EE676AE7EE056A0C
:1071E800BDEEE67A17EE106A17EE100A9E42A8BFA7
:1071F80018468E42B8BF084607EE100AB8EEC77A9E
:10720800022A8CED017A3EF447AB98ED087ADDED61
:107218000E6A25EE877AA6EE867AF0EE676AE7EEC2
:10722800056ABDEEE67A17EE106A17EE100A9E425E
:10723800A8BF18468E42B8BF084607EE100AB8EE37
:10724800C77A032A8CED027A3EF426AB98ED0C7AC5
:10725800DDED0F6A25EE877AA6EE867AF0EE676A8C
:10726800E7EE056ABDEEE67A17EE106A17EE100A29
:107278009E42A8BF18468E42B8BF084607EE100ABD
:10728800B8EEC77A042A8CED037A3EF405AB98ED84
:10729800107ADDED106A25EE877AA6EE867AF0EE92
:1072A800676AE7EE056ABDEEE67A17EE106A17EE32
:1072B800100A9E42A8BF18468E42B8BF084607EE7D
:1072C800100AB8EEC77A052A8CED047A3EF4E4AACF
:1072D80098ED147ADDED116A25EE877AA6EE867AA6
:1072E800F0EE676AE7EE056ABDEEE67A17EE106A19
:1072F80017EE100A9E42A8BF18468E42B8BF08462D
:1073080007EE100AB8EEC77A062A8CED057A3EF425
:10731800C3AA98ED187ADDED126A25EE877AA6EEF3
:10732800867AF0EE676AE7EE056ABDEEE67A17EE52
:10733800106A17EE100A9E42A8BF18468E42B8BFC0
:10734800084607EE100AB8EEC77A072A8CED067AC7
:107358003EF4A2AA98ED1C7ADDED136A65EE875A11
:10736800E6EE265AE5EE257AFDEEE77A17EE900A64
:107378008342A8BF03468142D8BF194607EE901A38
:10738800F8EEE77ACCED077ABEF1000F7EF4C0ACD8
:10739800FEF786BAAA4BD3F800C0BCF832E04FEA31
:1073A8005E0E91E4DFF8D092D4ED017A94ED006A94
:1073B800B9F80000D9F8143077EEA77AF0EE006A31
:1073C800B0EE677AA6EE267A013804EBC002D6EE54
:1073D800267A083A1033F6EE003A27EE237A67EE5B
:1073E800A37A84ED207AC4ED217A964CA64604F15E
:1073F800800192ED027A92ED036ADEED036ADEED1A
:10740800027A53ED014A13ED025A37EE674A76EED7
:10741800C65A77EE277AE4EE845A0138A2F10802B8
:10742800E5EE047A0EF1080E03F1080336EE267A2B
:1074380001F10801E4EE877AE5EE475A67EEA37A90
:1074480025EEA37AC1ED007A81ED017AD1D1142F0E
:107458007DF4EBAB05F0FCFE069BDFF82082C01A3A
:10746800A8F80200D4F8A861FDF7DFBBD4F8AC8116
:10747800B4F8A4A1744BCAF120095FFA89F90AEBA0
:10748800481E03EB8E0E5FEA990301F00185013374
:1074980018016E496E4A0EEB000C0EF1100313ED45
:1074A800024A13ED035A13ED016A13ED047A51ED04
:1074B800024A51ED035A51ED016A51ED047A64EE26
:1074C800244A65EE255A66EE266A67EE277A103357
:1074D8009C4542ED024A42ED035A42ED016A42EDF3
:1074E800047A01F1100102F11002D8D15949A0F132
:1074F8001002964401EB020C224419F0030309D050
:10750800BEEC017AFCEC017A67EE277A013BE2ECEB
:10751800017AF5D1BAF1000F41F0A581142F7DF45D
:1075280084AB05F095FE069BDFF85081D4F8A8617E
:10753800C01AA8F80200FDF778BBDFF83C91414873
:10754800D9F80820B9F80C1021F05AFE424B1F78E0
:10755800142F01F07385D4F8A8610136C4F8A86126
:1075680022E7D4F8AC913D4B3D4ADFED3E7AD2EDAF
:10757800008A3D4A4FEAC9010B44F8EE688A9B88A5
:1075880009EE103A643BC82BA8BFC82368EEA78A47
:10759800F8EE497A782BB8BF782368EEA78A07EE09
:1075A800903A4944B0EE680A02EB8108B8EEE78ADF
:1075B80022F00EFEB8EEC99AF0EE409AB0EE680AD4
:1075C80022F068FD38EE097A79EE487A28EE098AC1
:1075D80067EE877AB7EE006A88EE277A142FF8EEFE
:1075E800007A77EE076A60EE277A89EEA67A77EE58
:1075F800065A36EE477AC6EE256A67EEA67A27EE71
:10760800267AC8ED006A88ED047AC8ED026AC8EDEA
:10761800017AC8ED037A01F06385144B0E4A09F12B
:10762800010983FB0938A8EBE97808EB480801361B
:10763800A9EB08081778C4F8A861C4F8AC8117E763
:10764800EC590020E81F0020F43F0020844100206E
:10765800F81F00207441002094540020F4410020B9
:107668008851002027D4D2361C5100205655555534
:10767800EC2E00206C3A0020DC3F002098540020BB
:10768800DFF80494B9F800E0D9F804C04FEA5E08BE
:107698004FEA880204EB8E065FEADE0E04EB020373
:1076A80000F0A08010320EF1010EEB4803EB0E1E25
:1076B800324410330CF1100706F1100151ED032A82
:1076C80051ED043A10ED043A10ED032A51ED026A27
:1076D80011ED016A10ED020A10ED018A12ED044A5B
:1076E80012ED035A53ED044A53ED035A13ED027A8F
:1076F80053ED017A52ED020A12ED011A73EE238A54
:1077080072EE221A40ED048A40ED031A70EE268AC2
:1077180078EE061A40ED028A40ED011A74EE848A6A
:1077280075EE851A43ED048A43ED031A77EE208A35
:1077380077EE811A43ED028A43ED011A73EE633A3C
:1077480075EE655A17ED035A32EE623A74EE644AE2
:1077580065EE631A17ED044A23EE052A64EE652ADE
:10776800E3EE041A10339E4524EE843AA3EE842AED
:1077780000F1100007F11007A5EE853A01F110019C
:1077880002F11002E4EE852A41ED071A01ED082AFC
:1077980002ED073A42ED082A57ED055A17ED065A49
:1077A80070EE666A38EE466A30EEC77A71EE677A2E
:1077B80026EE253A65EEE63A25EE674A67EE054A73
:1077C800E6EE053AA6EE853AA7EE254AE7EEA54A83
:1077D80001ED063A41ED053A02ED064A42ED054A49
:1077E8007FF46CAF1FFA88F8624641469B481EF04A
:1077F80083F94146D9F8042030461EF07DF9984BAC
:107808001B78142B7FF42EAE24E6DFF8809299F8CB
:107818000020900801F0CB84DFF874C200F1010861
:107828004FEA48180CEB080E0CF12003ACF170017C
:1078380013ED076A53ED056A13ED037A53ED017AE8
:1078480053ED025A13ED084A53ED064A13ED045A54
:1078580026EE066A66EEA66A27EE077A67EEA77A2C
:10786800A4EE046A20339E45E4EEA46A01F11001F7
:10787800A5EE057AE5EEA57AF1EEC65AB1EEE66A0E
:10788800F1EEC76AB1EEE77A41ED085A01ED076AF1
:1078980041ED066A01ED057ACAD1A8F12008C44471
:1078A80004EB001012F0030318BF0CF1080C0FD002
:1078B8005CED017A1CED027A67EEA77A013BE7EEF0
:1078C800077A0CF1080CB1EEE77AA0EC017AEFD157
:1078D800142F01F013840136C4F8A861FDF70EB91E
:1078E80005F0B6FC5E4B06901F78142F05BFDFF835
:1078F800A481D4F8A861D4F8A861A8F80060FDF7BD
:10790800E2B876EE665AFFF71ABB564A5649D2EDE8
:10791800007A564A91ED007A1278C4ED7E7A84EDA9
:107928007F7A002A01F0648277EE676A5049C4EDD5
:107938007C7AC4ED7B6AFF22D1ED006ADFED4D7AD7
:1079480084F80022FDF713BC4B494B69002B3DF42A
:10795800E4AA4A484A4B008893FBF0F00B684FF0C2
:10796800010E186081F811E0FDF7D7BA454EDFF82F
:10797800289196ED004A96ED057AD6ED014A96EDE6
:10798800066AD6ED046A96ED035AD6ED025A67EEFA
:10799800897A09EB8703A4EE277AA4EEA76A66EE34
:1079A800C76AA5EE476AE5EEA76A20EE070A86EDE4
:1079B800056AC6ED066A83ED007A29EE088A22F088
:1079C800BBFB69EE288AD6ED0E5AD6ED176A96EDFE
:1079D800091AD6ED121A96ED0F5A96ED187A96ED09
:1079E8000A2AD6ED132A96ED0D6AD6ED167A96ED8B
:1079F8000C3AD6ED0B3A96ED154AD6ED144AE1EE5F
:107A0800085A002209EB8703E8EEA16A00B2C4F81D
:107A18009421A2EE085AC4F89821C4F89C21A8EE33
:107A2800A27A26EE656A67EEE67AA3EE655AA3EEB9
:107A3800886AA6EEC47AE8EEA47A86ED0E5AC3EDFB
:107A4800205A86ED0F6AC3ED406A86ED177AC6EDB7
:107A5800187AFEF783BC00BFF81F0020E81F00203B
:107A680094540020AC3A0020702F0020E44B0020F2
:107A7800842F0020000000004C570020645700208D
:107A880020A1070078420020DC3F0020D63F0020DC
:107A98006820002098540020F43F0020C6494A6915
:107AA800002A3DF46BAA0A6813604B74FDF766BAA6
:107AB800B5F93C306A6207EE903A0122F8EEE77AAF
:107AC800EB66C5F888200023012FC5ED1F7AC5EDA8
:107AD8001E7AC5F8803001F0B781B7427DF434AF23
:107AE800B5F93E302B6707EE903A00220123F8EEF5
:107AF800E77AAA62C5F89C300023012FC5ED247AE5
:107B0800C5ED237AC5F8943001F09A81B7427DF427
:107B18004BAFB5F940306B6707EE903A002201236E
:107B2800F8EEE77AEA62C5F8B0300023012FC5ED18
:107B3800297AC5ED287AC5F8A8307DF465AF9FEDA0
:107B48009F8AB9F1030F46D0BAF1000F09D007EEAA
:107B580090AAF8EEE77AF4EEC87AF1EE10FA01F19D
:107B68007183974A6B6F126894F8B011A8F80600F1
:107B780003EB560393FBF6F60023EE62936213635E
:107B8800D36231B18F4B1B8823F40063002B7DF443
:107B98003DAF8D4B1B6813F4003341F049818B498D
:107BA8001A46C85C012803F10C0300F0F584013281
:107BB800152AF6D1FDF72ABF854B9B7B002B3EF497
:107BC800FDA9FDF7F3BFF7EE006AFEF745BDF7EE36
:107BD800006AFEF7C5BCB0EE480A22F0ADFA00B262
:107BE800B2E7B4F8489109F1FF390FFA89F9B9F108
:107BF800000FA4F848917EF7E0AB764BFEF743B848
:107C0800B4F81A3103F57A739BB2FDF7E8BFDFF8D1
:107C1800E88198F80020013A0A2A1DD8DFE812F016
:107C2800A1005A0104013E011C001C00EE008F0057
:107C38006A0054000B00684A684952680968C832EB
:107C48008A4203D31BF014F830B1BB78032B01F040
:107C58002D83012388F80030FB78002B3EF42AADF1
:107C68005F4B1B78D80740F18580DFF87091D4F816
:107C78009021D9F800309A4200F2888098F80030B4
:107C8800012B3EF417AD94F88C21002A3EF412AD76
:107C98000B2B0DD801229A4040F6030112EA010786
:107CA8000DD112F4C06F03D0093B012B41F2E783D9
:107CB800494BD9F800205A600B2388F8003000237C
:107CC80084F88C31FEF7F6BC464B1B78002B01F08C
:107CD80025821A200AF0AAFA002841F01F8294F897
:107CE8008C31002B41F01A82092388F8003011F0FA
:107CF80089FCB1E71A200AF099FA0028F7D03A4B24
:107D08001B88002BF3D1394B4520D3F800901AF08B
:107D1800D3FF0E201AF0D0FF484611F067F9DDF8BE
:107D28002490484611F062F9314A324B12681A60C1
:107D380048460A2388F8003011F0C4F9D7E71AF04A
:107D480075FF11F091FC002886D01AF091FF0028E9
:107D580082D0274A274B12681A600A2388F8003015
:107D68007AE71F4B1B78DB0701F18F82FB78002B2A
:107D78003EF4A0AC0DF0F0F900283FF476AF174BB5
:107D88001B6803F59C530833C4F8903198F8003009
:107D9800012B7EF48FAC94F88C31002B7EF48AACE6
:107DA800BB78032B01F0798312F01AFA012384F8C7
:107DB8008C31FEF77FBC00BF4C570020000000004C
:107DC80024480020A2550020A4430020B8DE020861
:107DD800284800205C550020103C00206C570020EB
:107DE800D05A0020D03C0020903A00208C3A002045
:107DF800A03A0020983A0020E96800201AF016FFFF
:107E08007B4B002105208DE80300A3F108020291B5
:107E1800532012F01BF900287FF41EAF754A08237F
:107E2800106088F8003017E7DFF8C8911AF0FEFEF6
:107E3800714AD9F80430126864339342BFF40CAF26
:107E480040201AF0D7FE00287FF406AFD9F800309A
:107E5800DFF8CCB169494FF0400A0FE005911AF0FC
:107E68002BFF0599D9F800300A680133013ABAF1B5
:107E7800010A0A60C9F8003001F02A821BF80330B1
:107E88001846002BEAD100234FF0FF32C9F8003022
:107E98000423C9F8042088F80030DDE61AF0C6FE8D
:107EA800574A0292A2F10C03252101930091A2F1F5
:107EB8000A035021163A492012F0C8F800287FF426
:107EC800CBAE4C4B4FF0FF3107221860596088F851
:107ED8000020C1E6484B474A1B68536047490023C6
:107EE800136003220B6088F80020B5E6454ADFEDF1
:107EF800467A92ED080A0593B4EEE70AF1EE10FA15
:107F080040F2AD8422F0AEF9D4ED457A20EE270A8E
:107F180022F012F9B0F5617F059B00F33A8607EE6F
:107F2800900AF8EEE76ADFED397A66EEA76A07EE9F
:107F3800903AB8EEE77AFDEEE67A17EE903A2033FB
:107F4800402B41F2F0809FED320A22F0F5F800B2A2
:107F580007EE900AB8EEE77A2E4BD3ED037A77EE68
:107F6800877AC3ED037AFDF729BE0A9B93F800E0F0
:107F78000EF0010EBEF1000F7DF4CAAEFDF790BC05
:107F8800254BDFED267A1E68C4ED707A16F0805610
:107F980040F01A8310F4800600F0AE810026B6EE99
:107FA800007A67EE877AF4EEE75AF1EE10FA48BFE6
:107FB800F0EE675A40F10883C4ED815AFDF716BB0D
:107FC80005F046F90646FDF7E3BD74EE677AB7EEAD
:107FD800007AF4EEC77AF1EE10FAC4ED707A40F345
:107FE8001C8784EEA77A8DED0C7AFDF7F5BA00BFF1
:107FF800A0C70208103C00206C570020245600201F
:10800800F2C50208202D00208FC2753CD06D393A88
:10801800000000005C550020043C002000000080A7
:108028008CC50208BAF1000F00F0CD8598ED007AF2
:10803800DDED0C6ADFF8E8C825EE877AA6EE867AC9
:10804800F0EE676AE7EE056ABDEEE67A17EE106AAB
:1080580017EE100A9E42A8BF1846B142C8BF08468C
:1080680007EE100AB8EEC77A012A8CED007A3DF4C3
:108078004FAE98ED047ADDED0D6A25EE877AA6EE0F
:10808800867AF0EE676AE7EE056ABDEEE67A17EEE5
:10809800106A17EE100A9E42A8BF1846B142C8BF20
:1080A800084607EE100AB8EEC77A022A8CED017A64
:1080B8003DF42EAE98ED087ADDED0E6A25EE877A4E
:1080C800A6EE867AF0EE676AE7EE056ABDEEE67A16
:1080D80017EE106A17EE100A9E42A8BF1846B14262
:1080E800C8BF084607EE100AB8EEC77A032A8CED17
:1080F800027A3DF40DAE98ED0C7ADDED0F6A25EEAF
:10810800877AA6EE867AF0EE676AE7EE056ABDEE34
:10811800E67A17EE106A17EE100A9E42A8BF1846B4
:10812800B142C8BF084607EE100AB8EEC77A042A5B
:108138008CED037A3DF4ECAD98ED107ADDED106A24
:1081480025EE877AA6EE867AF0EE676AE7EE056A8C
:10815800BDEEE67A17EE106A17EE100A9E42A8BF27
:108168001846B142C8BF084607EE100AB8EEC77AEB
:10817800052A8CED047A3DF4CBAD98ED147ADDED4B
:10818800116A25EE877AA6EE867AF0EE676AE7EE40
:10819800056ABDEEE67A17EE106A17EE100A9E42DF
:1081A800A8BF1846B142C8BF084607EE100AB8EE85
:1081B800C77A062A8CED057A3DF4AAAD98ED187AAF
:1081C800DDED126A25EE877AA6EE867AF0EE676A0A
:1081D800E7EE056ABDEEE67A17EE106A17EE100AAA
:1081E8009E42A8BF1846B142C8BF084607EE100A0B
:1081F800B8EEC77A072A8CED067A3DF489AD98ED7A
:108208001C7ADDED136A65EE875AE6EE265AE5EE2E
:10821800257AFDEEE77A17EE902A9342A8BF134617
:108228008A42A8BF194607EE901AF8EEE77ACCED15
:10823800077AFDF76DBDD8003EF53EADFDF7C3BC2E
:10824800012A40F3018607EE101AB8EEC77AC7EE86
:10825800876AB1EEE68AB9F1030F13D0BAF1000FBD
:1082680009D007EE90AAF8EEE77AF4EEC87AF1EEB4
:1082780010FA00F1E787EB6E03EB560393FBF6F376
:108288006B622AE4B0EE480A21F056FF00B2E5E737
:10829800012A7FF754AC07EE101AB8EEC77AC7EE7A
:1082A800876AB1EEE68A4CE4012A40F3C98507EEF5
:1082B800101AB8EEC77AC7EE876AB1EEE68AB9F146
:1082C800030F13D0BAF1000F09D007EE90AAF8EE09
:1082D800E77AF4EEC87AF1EE10FA00F1B3872B6F63
:1082E80003EB560393FBF6F3AB620FE4B0EE480AD8
:1082F80021F022FF00B2E5E7B6EE007AF4EEC75AA5
:10830800F1EE10FA3FF74BAEFDF770B9D8ED004A21
:108318009DED0C4ADFF808C665EEA44AFDEEC73AA3
:10832800E4EE064AB0EE674AA4EE854A13EE901AC8
:10833800F4EEC46AF1EE10FAF0EE444A88BFF0EEAB
:10834800474AFDEEE44A14EE900A14EE906A984209
:10835800A8BF1E468142C8BF0E4604EE906AF8EEDA
:10836800E44A012ACCED004A3DF496AAD8ED044A25
:108378009DED0D4A65EEA44AE4EE064AB0EE674A62
:10838800A4EE854AF4EEC46AF1EE10FAF0EE444A1F
:1083980088BFF0EE474AFDEEE44A14EE900A14EE68
:1083A800906A9842A8BF1E468842B8BF0E4604EE9F
:1083B800906AF8EEE44A022ACCED014A3DF46CAA30
:1083C800D8ED084A9DED0E4A65EEA44AE4EE064A49
:1083D800B0EE674AA4EE854AF4EEC46AF1EE10FAEC
:1083E800F0EE444A88BFF0EE474AFDEEE44A14EE48
:1083F800900A14EE906A9842A8BF1E468842B8BFF9
:108408000E4604EE906AF8EEE44A032ACCED024ADE
:108418003DF442AAD8ED0C4A9DED0F4A65EEA44AF8
:10842800E4EE064AB0EE674AA4EE854AF4EEC46A62
:10843800F1EE10FAF0EE444A88BFF0EE474AFDEE3E
:10844800E44A14EE900A14EE906A9842A8BF1E46B9
:108458008842B8BF0E4604EE906AF8EEE44A042A51
:10846800CCED034A3DF418AAD8ED104A9DED104A08
:1084780065EEA44AE4EE064AB0EE674AA4EE854AE1
:10848800F4EEC46AF1EE10FAF0EE444A88BFF0EE5A
:10849800474AFDEEE44A14EE900A14EE906A9842B8
:1084A800A8BF1E468842B8BF0E4604EE906AF8EE92
:1084B800E44A052ACCED044A3DF4EEA9D8ED144A65
:1084C8009DED114A65EEA44AE4EE064AB0EE674A0D
:1084D800A4EE854AF4EEC46AF1EE10FAF0EE444ACE
:1084E80088BFF0EE474AFDEEE44A14EE900A14EE17
:1084F800906A9842A8BF1E468842B8BF0E4604EE4E
:10850800906AF8EEE44A062ACCED054A3DF4C4A97F
:10851800D8ED184A9DED124A65EEA44AE4EE064AE3
:10852800B0EE674AA4EE854AF4EEC46AF1EE10FA9A
:10853800F0EE444A88BFF0EE474AFDEEE44A14EEF6
:10854800900A14EE906A9842A8BF1E468842B8BFA7
:108558000E4604EE906AF8EEE44A072ACCED064A85
:108568003DF49AA9D8ED1C4A9DED134A65EEA45A2C
:10857800E6EE045AE5EE257AF4EEE76AF1EE10FA33
:10858800C8BFF0EE477AFEF7EFBE8223FCF739BB8F
:10859800DFEDE07AFCF700BBD4F8B46153003EB1DC
:1085A800981801EB800076784078B042BDF42EAA86
:1085B800134401EB83010023C4F8B411A4F8083272
:1085C800C4F80C32FDF722BAB7EE007A77EE677A74
:1085D800F4EEE75AF1EE10FA88BFF0EE675AEBE4D2
:1085E800D8ED004A9DED0C4ADFF834C365EEA44A85
:1085F800FDEEC73AE4EE064AB0EE674AA4EE854AB5
:1086080013EE901AF4EEC46AF1EE10FAF0EE444A52
:1086180088BFF0EE474AFDEEE44A14EE900A14EEE5
:10862800906A9842A8BF1E468142C8BF0E4604EE13
:10863800906AF8EEE44A012ACCED004A3DF463ABB7
:10864800D8ED044A9DED0D4A65EEA44AE4EE064ACB
:10865800B0EE674AA4EE854AF4EEC46AF1EE10FA69
:10866800F0EE444A88BFF0EE474AFDEEE44A14EEC5
:10867800900A14EE906A9842A8BF1E468842B8BF76
:108688000E4604EE906AF8EEE44A022ACCED014A5E
:108698003DF439ABD8ED084A9DED0E4A65EEA44A83
:1086A800E4EE064AB0EE674AA4EE854AF4EEC46AE0
:1086B800F1EE10FAF0EE444A88BFF0EE474AFDEEBC
:1086C800E44A14EE900A14EE906A9842A8BF1E4637
:1086D8008842B8BF0E4604EE906AF8EEE44A032AD0
:1086E800CCED024A3DF40FABD8ED0C4A9DED0F4A94
:1086F80065EEA44AE4EE064AB0EE674AA4EE854A5F
:10870800F4EEC46AF1EE10FAF0EE444A88BFF0EED7
:10871800474AFDEEE44A14EE900A14EE906A984235
:10872800A8BF1E468842B8BF0E4604EE906AF8EE0F
:10873800E44A042ACCED034A3DF4E5AAD8ED104AF0
:108748009DED104A65EEA44AE4EE064AB0EE674A8B
:10875800A4EE854AF4EEC46AF1EE10FAF0EE444A4B
:1087680088BFF0EE474AFDEEE44A14EE900A14EE94
:10877800906A9842A8BF1E468842B8BF0E4604EECB
:10878800906AF8EEE44A052ACCED044A3DF4BBAA07
:10879800D8ED144A9DED114A65EEA44AE4EE064A66
:1087A800B0EE674AA4EE854AF4EEC46AF1EE10FA18
:1087B800F0EE444A88BFF0EE474AFDEEE44A14EE74
:1087C800900A14EE906A9842A8BF1E468842B8BF25
:1087D8000E4604EE906AF8EEE44A062ACCED054A05
:1087E8003DF491AAD8ED184A9DED124A65EEA44AC7
:1087F800E4EE064AB0EE674AA4EE854AF4EEC46A8F
:10880800F1EE10FAF0EE444A88BFF0EE474AFDEE6A
:10881800E44A14EE900A14EE906A9842A8BF1E46E5
:108828008842B8BF0E4604EE906AF8EEE44A072A7A
:10883800CCED064A3DF467AAD8ED1C4A9DED134AD3
:1088480065EEA45AE6EE045AE5EE257AF4EEE76AF8
:10885800F1EE10FAC8BFF0EE477AFEF7F2B99FEDD5
:108868002E7AFFF779BB2D4B4FEA890E5FEA9A09FA
:1088780001EB0E0C03EBC818A64400F0FF8409F1C5
:1088880001094FEA091908EB090008F110030CF176
:1088980010010EF1100213ED024A13ED035A13ED05
:1088A800016A13ED047A51ED024A51ED035A51ED74
:1088B800016A51ED047A64EE244A65EE255A66EEA3
:1088C800266A67EE277A1033984242ED024A42ED53
:1088D800035A42ED016A42ED047A01F1100102F1F6
:1088E8001002D8D1A9F11009C8440CEB0901CE44F3
:1088F8001AF0030A3EF412AEB8EC017AF1EC017AF0
:1089080067EE277ABAF1010AEEEC017AF4D1FEF7A4
:1089180005BE00BF0000024300000000F43F002035
:108928006C3A0020BAF1000F00F09483DFF8548607
:108938009DED0C4AD8ED004A65EEA44AE4EE064ADD
:10894800B0EE674AA4EE854AF0EE444AB9F1000F4A
:1089580006D0F4EE446AF1EE10FAC8BFF0EE474ACA
:10896800BDEEC77A17EE101ABDEEE47A04EE901A3F
:1089780017EE100A814200F371849842A8BF184686
:1089880007EE100AB8EEC77ADFF8FCC5012A8CEDAD
:10899800007A3DF4BDA998ED047A9DED0D4A25EEC7
:1089A800877AA4EE067AB0EE674AA7EE054AB0EEDB
:1089B800447AB9F1000F00F03A84F4EEC46AF1EE9B
:1089C80010FA40F3348408469842A8BF184607EEC8
:1089D800100AB8EEC77A022A8CED017A3DF498A9FC
:1089E80098ED087A9DED0E4A25EE877AA4EE067A70
:1089F800B0EE674AA7EE054AB0EE447AB9F1000F27
:108A080000F00A84F4EEC46AF1EE10FA40F304842C
:108A180008469842A8BF184607EE100AB8EEC77A6B
:108A2800032A8CED027A3DF473A998ED0C7A9DED3A
:108A38000F4A25EE877AA4EE067AB0EE674AA7EECB
:108A4800054AB0EE447AB9F1000F00F0DB83F4EE8A
:108A5800C46AF1EE10FA40F3D58308469842A8BFDD
:108A6800184607EE100AB8EEC77A042A8CED037A86
:108A78003DF44EA998ED107A9DED104A25EE877ABF
:108A8800A4EE067AB0EE674AA7EE054AB0EE447A3D
:108A9800B9F1000F00F0AC83F4EEC46AF1EE10FAFD
:108AA80040F3A68308469842A8BF184607EE100A66
:108AB800B8EEC77A052A8CED047A3DF429A998ED19
:108AC800147A9DED114A25EE877AA4EE067AB0EE67
:108AD800674AA7EE054AB0EE447AB9F1000F00F0F4
:108AE8007D83F4EEC46AF1EE10FA40F3778308460A
:108AF8009842A8BF184607EE100AB8EEC77A062AA9
:108B08008CED057A3DF404A998ED187A9DED124A8A
:108B180025EE877AA4EE067AB0EE674AA7EE054AF4
:108B2800B0EE447AB9F1000F00F04E83F4EEC46A57
:108B3800F1EE10FA40F3488308469842A8BF184659
:108B480007EE100AB8EEC77A072A8CED067A3DF4CC
:108B5800DFA898ED1C7A9DED134A65EE875AE4EE7E
:108B6800065AE5EE857AB9F1000F00F02583F4EE98
:108B7800E67AF1EE10FA40F11F830A469A42A8BF3E
:108B88001A4604EE902AF8EEE44ACCED074AFDF7BF
:108B9800BFB807EE903ADFEDEC6AB8EEE77A66EE1A
:108BA800A65A9FEDEA5A9FEDEA6ADFEDEA7AA5EE4A
:108BB800856A26EEA55AE5EE867AE5EE276A26EE60
:108BC800870AFFF7C2B9D8ED006ADDED0C4A65EEF9
:108BD800A66AE4EE866AF0EE674AE6EE854AFDEE9E
:108BE800E46A16EE90EA714500F325829E45A8BF17
:108BF8009E4606EE90EAF8EEE66A002E00F034840F
:108C0800DFF884C3012ACCED006A3DF481A8D8EDD1
:108C1800046ADDED0D4A65EEA66AE4EE866AF0EEBA
:108C2800674AE6EE854AFDEEE46A16EE90EA71457B
:108C380000F31F819E45A8BF9E4606EE90EAF8EE17
:108C4800E66A002E00F03C84022ACCED016A3DF46D
:108C58005FA8D8ED086ADDED0E4A65EEA66AE4EE77
:108C6800866AF0EE674AE6EE854AFDEEE46A16EE9D
:108C780090EA714500F309819E45A8BF9E4606EE1D
:108C880090EAF8EEE66A002E00F00F84032ACCED95
:108C9800026A3DF43DA8D8ED0C6ADDED0F4A65EE99
:108CA800A66AE4EE866AF0EE674AE6EE854AFDEECD
:108CB800E46A16EE90EA714500F3E4809E45A8BF89
:108CC8009E4606EE90EAF8EEE66A002E00F0B883BB
:108CD800042ACCED036A3DF41BA8D8ED106ADDED3B
:108CE800104A65EEA66AE4EE866AF0EE674AE6EE9A
:108CF800854AFDEEE46A16EE90EA714500F3BF80FE
:108D08009E45A8BF9E4606EE90EAF8EEE66A002E5B
:108D180000F08C83052ACCED046A3CF4F9AFD8ED59
:108D2800146ADDED114A65EEA66AE4EE866AF0EE95
:108D3800674AE6EE854AFDEEE46A16EE90EA71456A
:108D480000F39A809E45A8BF9E4606EE90EAF8EE8C
:108D5800E66A002E00F07E83062ACCED056A3CF414
:108D6800D7AFD8ED186ADDED124A65EEA66AE4EED3
:108D7800866AF0EE674AE6EE854AFDEEE46A16EE8C
:108D880090EA714572DC9E45A8BF9E4606EE90EAC1
:108D9800F8EEE66A002E00F0BF83072ACCED066ADB
:108DA8003CF4B6AFD8ED1C6ADDED134A65EEA65A61
:108DB800E4EE865AE5EE257AFDEEE77A17EE902A7C
:108DC800914203DC9A42A8BF1A46114607EE901A50
:108DD800F8EEE77A002E7FF42AAA069B002B7FF490
:108DE80026AA059B5B45B8BFF0EE477AFFF71FBA86
:108DF80077EEC76AF0EE477AFEF798BDBCF83430D4
:108E08009FED557A07EE903AF8EEE77A534B67EE06
:108E1800877AC3ED007AFCF7D6BE514B1E6816F070
:108E280080567FF4BCA8FFF7B5B84E4BFCF722BFBD
:108E38004D4B1B78032B00F024820023FEF7AFBEB6
:108E48009FED4A8AFFF73BBA9FED488AFFF703BABE
:108E58009FED470ADFF8348125EE800A21F06CF98E
:108E6800D4F8A861A8F80600FBF7DFBE06EE901A52
:108E78008EE706EE901AE2E606EE901A67E706EE2F
:108E8800901A42E706EE901A1DE706EE901AF8E6E9
:108E98003849394A8C46FEF730BB93ED000A0593F2
:108EA8000791069221F048F9DFF8E4E0DFF8E4C022
:108EB800DEF8ECE0DFF8D480069AA8F800008CFB16
:108EC8000E3C4FEAEE7ECEEBAC1E07EE90EAF8EED3
:108ED800E77A059B0799FDEEE77A17EE900AA8F85E
:108EE8000200FCF7CCBE07EE907AF8EEE78ADFEDD9
:108EF800237A9FED2C0A84F8847168EEA78A38EEED
:108F0800800AFDEEC07A17EE903A2033402B40F2EB
:108F18009F819FED160A114BFDEEE87A83ED010A59
:108F280017EE903A2033402B00F29581DFED1E7A40
:108F3800F4EEE78AF1EE10FA40F3D481DFED176A18
:108F4800DFED0F7A3AE000BF84F9223F92E741B99A
:108F58009730083C15A82ABE6F12833A7800002083
:108F6800043C00205C5500207843002000000000ED
:108F78000000C84274410020E81F002035FA8E3CEA
:108F8800E4CB1641EC2E00206C3A002098540020C7
:108F980010010020D34D6210DB0F49C0DB0FC94020
:108FA800E4CB16C1DB0FC93FDB0F494092E741B95B
:108FB8009730083C15A82ABEF0EE478AF4EEE78AF7
:108FC800F1EE10FA38EEE67AF6DC5FED0D7AB4EEE3
:108FD800E77AF1EE10FA40F182811FED106A5FED39
:108FE800106A01E0B0EE677AB4EEE67AF1EE10FAB4
:108FF80077EE067AF6D41FED157AF4EEC77AF1EE1D
:1090080010FA40F32F811FED187A77EE677A27EE72
:10901800A76A5FED1A5A5FED1A6A1FED1A7AE6EE33
:10902800256A67EE865AA6EE267AE5EE877AC4EDBB
:10903800627AFDF7B4BE06EE901ADCE504F008F992
:10904800CB4BDFF874831F78069BC01AA8F8020080
:10905800FEF781BAFDEEC74A0DF1300E9A46DFF8E9
:109068005CC3DFF85C8314EE901A0EEB82024B4669
:1090780006E07245E8EC014A0CF1100C3CF448AEED
:10908800DCED004ABEEC014A65EEA44AE6EE044A6D
:10909800B0EE674AA5EE244AF0EE444A33B1F4EE46
:1090A800446AF1EE10FAC8BFF0EE474AFDEEE44A12
:1090B80014EE909A494504EE901A04DCD145A8BFF5
:1090C800D14604EE909AF8EEE44A002ED1D10698E3
:1090D8000028CED105985845B8BFF0EE474AC8E7F2
:1090E80004F0B6F8069BDFF8D082D4F8AC91D4F837
:1090F800A861C01AA8F80200FEF78FBA04F0A8F811
:109108009B4BDFF8B4821F78069B99F80020D4F8AF
:10911800A861C01AA8F80400FEF7DDBB09980FF093
:10912800D1FFFEF7E4BDDFED937AF4EEE76AF1EEE6
:1091380010FA40F3EE81DFED905A9FED906A01E05E
:10914800F0EE676AF4EEC66AF1EE10FA76EEE57AAA
:10915800F6DCDFED8B6AF4EEE67AF1EE10FA40F118
:10916800D581DFED855A9FED876A01E0F0EE667ADA
:10917800F4EEC67AF1EE10FA77EEA56AF6D4DFEDD2
:10918800827AF4EEE76AF1EE10FA04DDDFED797A1F
:1091980077EEE66A03E5DFED7D7AF4EEE76AF1EE55
:1091A80010FA44BFDFED767A77EEE66AF7E478489E
:1091B80000F1800CFEF776BBFDEEE77A17EE902AF9
:1091C8008A42FFF6E0ACD9E4BDEEC77A17EE100A82
:1091D8008842BFF6B2AC07EE101AB3E4BDEEC77A08
:1091E80017EE100A8842BFF683AC07EE101A84E423
:1091F800BDEEC77A17EE100A8842BFF654AC07EEE8
:10920800101A55E4BDEEC77A17EE100A8842BFF669
:1092180025AC07EE101A26E4BDEEC77A17EE100A41
:109228008842BFF6F6AB07EE101AFFF7F7BBBDEEA4
:10923800C77A17EE100A8842BFF6C6AB07EE101AB7
:10924800FFF7C7BBA8F80600A5F8B460FCF7E6BBB3
:1092580003F0D6F95FE6DFED4F7AE8E607EE101A7D
:10926800FFF790BB9FED497AF4EEC77AF1EE10FA5A
:1092780044BF9FED437A77EE677AC8E66146FFF709
:1092880037BB0EF0F3FBFCF7C1BB802017F054FE90
:1092980008B107F0F7F910F0A3FFFEF7DDBC94F86A
:1092A800E031002B7BF42AAFFBF715BFDFF81491F0
:1092B800D9F800000DF0EEFE374B1B780022022B88
:1092C800C9F800207EF4C5AC07F0F4F9FEF7C1BC7C
:1092D8001BF80330002B7EF4BFACFEF7D4BDF0EED4
:1092E800477A88E6B0EE687A6FE62C4A2C4B10680D
:1092F8001B689847089BDBED007A93ED007A294BB1
:10930800D7ED006A83ED020A274B67EE277A2B44D4
:1093180027EE8C7AD3ED007A244B67EE277AF0EEAD
:10932800665AEDEE275A93ED006AB1EE467AB4EE2E
:10933800E57AF1EE10FA08DCB4EEE56AF1EE10FA1F
:109348008CBFB0EE657AB0EE467A194B1B78012BCC
:1093580002D0192B7BF449AEDFED167AB4EEE7DACA
:10936800F1EE10FACCBF01230023FBF749BE00BF82
:1093780094540020DB0F4940DB0FC940E4CB164171
:10938800DB0F49C0E4CB16C1DB0FC93FDB0FC9BFF8
:10939800E81F002000000000613C0020302E002063
:1093A800442E0020343A0020542E0020BC2E0020E9
:1093B800583200200000964298540020EC2E0020DD
:1093C8006C3A00202856002000C0F84400C0F8C4B9
:1093D8005FED037AF4EEE7DAF1EE10FA20DC5FEDE8
:1093E800057AF4EEE7DAF1EE10FA19D44F4BD3ED23
:1093F800007AB1EE677AB4EEC7DAF1EE10FA12D459
:10940800B4EEE7DAF1EE10FA88BFB0EE67DA484B4F
:10941800C7ED00BA1B689342BBF6A8ADFCF7C5BE02
:109428009FED44DAF3E7B0EE47DAF0E70698002854
:109438007FF470AC05985845B8BFF0EE476A69E408
:10944800069800287FF444AC05985845B8BFF0EE5C
:10945800476A3DE4069800287FF47EAC0598584595
:10946800B8BFF0EE476A77E4069800287FF4C8ABE7
:1094780005985845B8BFF0EE476AFFF7C1BB4520CD
:1094880019F01AFCFF2019F017FC2B4819F000FC02
:10949800384619F011FCFEF70BBC802017F04CFD84
:1094A80000287DF407A9FEF77FBC069800287FF402
:1094B800EDAB05985845B8BFF0EE476AFFF7E6BB35
:1094C800069800287FF4C0AB05985845B8BFF0EE61
:1094D800476AFFF7B9BB132B05D1B0EE480A20F055
:1094E8002BFEAAF80000B0EE480AD5F8143213484B
:1094F8009847134B1B78132BB0EE408A7BF4D6ABFE
:1095080020F01AFEAAF80200FBF7D0BBF0EE676A5B
:1095180035E6F0EE667A1CE6069800287FF43DAC46
:1095280005985845B8BFF0EE476A36E4B82E0020D3
:109538009C2E00200000000094EC02081C51002022
:10954800945400202DE9F04F2DED028B984B994A49
:109558001C7893B000F59C4120318146069111603A
:10956800002C00F07C86944A1268904240F28A806F
:10957800924A93491768934DDFF888B20492013CE8
:1095880002911C7007F48057002F40F08880029BDE
:109598005B7D002B40F02D86049B1B681E0401F1A7
:1095A800FF80894B99459BF8023000F20085002B1B
:1095B80040F00185854B0593049B1F6817F480597B
:1095C80040F0BB85029BB5F906605B8B9E42B4BF39
:1095D800002601267E4B1B6813F0805369D0059A3C
:1095E800127812F001026AD002987A49408C91ED03
:1095F800037A039107EE900AF8EEE77AB4EEE77A79
:10960800F1EE10FA81F28081002E60D1724C94F84C
:10961800A01000295BD171487149006890F82D00AD
:1096280000240C604C608C606E49002850D1087092
:10963800002A51D0F8064FD56B4A1278D1064BD480
:10964800B9F1000F48D1002B46D17A0244D4674BB8
:109658001B78002B01F0FD86654B9B78002E41F0AE
:1096680030873BB1634A644B12681B689B1A002B16
:10967800C1F21F871020584C0EF016FA012384F807
:10968800A13029E04D4B4E4A1F68049307F48057D8
:1096980002924C4DDFF86CB1002F3FF478AF0021F7
:1096A8004B4803F085F800287FF471AF0FF06AF992
:1096B8006DE77C0293D4059A127802F00102464CB9
:1096C800002184F8A01043490391002EA3D04549F6
:1096D80001200870002AADD1484B1A78002A50D1D1
:1096E8000299B5F900E0488B898BB5F902407045BD
:1096F800B4BF8027002747F040037145D8BF3B46D9
:109708009B0843F08007A042B8BF3B4643F04007A0
:10971800A142C8BF3B469B08B5F90440B5F906709D
:1097280043F0800EA042B8BF734643F0400EA142FA
:10973800C8BF73469B0843F0800E274C8742C8BFBA
:10974800734643F0400E94F8A2C08F42B8BF7346E8
:109758009C4501F0BF82A4F8A42084F8A6202349E0
:1097680084F8A2300F78002F01F01F825F2B01F0E0
:109778008B826F2B01F02481059B1B78DE0741F15A
:10978800E880049B1B6803F00403002B40F020864C
:109798000DF140081A4C0022C8F8042004F15009C1
:1097A800109240F6330A192740F283362FE000BFA3
:1097B800E0300020DC2F0020DC3000209851002011
:1097C8003053002002670020404B4C00D05A002044
:1097D800043C00205C550020FC210020EC590020AE
:1097E800403A0020C8210020CC3F0020441B002024
:1097F800583C00206C570020203A0020A15500203A
:10980800803C0020385A002004344C4520D0A278EF
:10981800E3789A4217FB0261F6D26278043217FBAA
:10982800036335F912205245A8BF5246B2F5617F4D
:10983800B8BF4FF461728A42E6DD9A42E4DC2178CF
:109848002429E1D84046043402F0A2FF4C45DED179
:10985800624A634B177898E8030083E80300002FF7
:1098680000F03F855F4B07935D48012102F0A0FFA0
:10987800002840F0A9829BF80330002B40F0A48216
:10988800594B0693594C23881EB226F001061FFA3D
:1098980086F84345A4F8008000F0E187544E4FF065
:1098A80002090E2014274FF0FF0A86F800907770FF
:1098B80086F802A00EF0F8F849464948B4F8008046
:1098C80002F076FF002841F0AB8128F002039BB23A
:1098D800434523800BD0464B1421FF2202260E203D
:1098E8001E7059709A700EF0DFF8B4F80080414B82
:1098F800414A19785068089318F0030F08BF81F09F
:109908000201C1F34001099204F018FE24213448F1
:1099180002F04EFF30B9059A13785E0744BF23F072
:1099280004031370069B1B6813F00A0F1AD0062154
:109938002B4802F03DFF002800F0B4872388580622
:1099480041F1B2800721264802F032FF50B12B4B7B
:109958002B4AB3F904302B4982FB0302DB17C3EB14
:10996800A2030B800C211E4802F022FF2288002847
:1099780000F04A8242F480739A42238009D01C4B3B
:1099880002201421FF2218700E2059709A700EF0D0
:109998008BF81D4B1B78082B00F042820E2B00F031
:1099A8003F82049B1B68590561D5184B1B79002B16
:1099B80000F0258114210A4802F0FAFE002840F040
:1099C800238114F099F801200DF0AEFF00284ED045
:1099D800DFF83C9000264FF0CC0A1EE03C45002002
:1099E800043C0020D02B00208C5900205A32002043
:1099F800D84400203657002038570020D859002076
:109A0800676666661C3A00207C3C00204C550020A6
:109A1800885B0020DEB2022E29D80AFB06F8731CE8
:109A280059F80870002FF5D1C378D04A90F9020090
:109A380052F8233001970322009201213A460DF093
:109A480055FB034606EB460000EB0010069353B1A6
:109A5800394609EB8000CC2222F086FC069B49F8A7
:109A680008300136F6B21CF0B9FC0028D3D1059BAA
:109A78001E7816F0010600F02982BD4B01221A70EB
:109A8800079BB5F906101B68BA485A890127914205
:109A9800077080F20182B84B4FF07E521A60B74AC5
:109AA800029BB5F900E01F8B92F90430107892F808
:109AB80001C0002BAEEB070314BF01224FF0FF32A9
:109AC800002BB8BF5B42B3F5FA7FA8BF4FF4FA7317
:109AD800984280F2DE811B1A07EE903AF8EEE77A98
:109AE800039BBE45C3ED007A03DAF1EE677AC3ED56
:109AF800007AB5F902E0AEEB0703002BB8BF5B4272
:109B0800B3F5FA7FA8BF4FF4FA73984280F2BE818A
:109B18001B1A07EE903AF8EEE77A039B7745C3EDF8
:109B2800017A03DDF1EE677AC3ED017AB5F9040035
:109B3800C31B002BB8BF5B42B3F5FA7FA8BF4FF435
:109B4800FA736345CCBFA3EB0C03002302FB03F3BA
:109B580007EE903A039A049BF8EEE77AB842C2ED12
:109B6800027ABCBFF1EE677AC2ED027A1A6812F483
:109B7800805200F06881B1F5FA6F814BA8BF4FF4AD
:109B8800FA61B1F57A7F1878B8BF4FF47A71A1F508
:109B98007A71002840F070817A4D7B4885FB013E40
:109BA800CB17C3EB6E1303F1010E6FF0630C30F9A2
:109BB8001EE030F913000CFB0313AEEB000103FBAE
:109BC80001F385FB0315DB17C3EB651303441BB2D5
:109BD80007EE903A039BB8EEE78A83ED038A002AE2
:109BE80040F03C8423885B0624D4002E40F0B080EB
:109BF8001FF0E6F913B0BDEC028BBDE8F08F059BB2
:109C08001B78DA077FF5DDAE3C2017F095F90028C0
:109C18003FF42DAF06F036FD3C2017F02FF9002851
:109C28003FF425AF06F02EFD3C2017F027F9002859
:109C3800F0D11CE7554B564AB3F904305549DFEDCE
:109C4800566A09889FED557A82FB0302DB17C3EB3E
:109C5800A2035B1A1BB207EE903AF8EEE77A67EEBA
:109C6800A67A77EE876ABDEEE66A16EE103A2033DA
:109C7800402B40F22587DFED4A6ABDEEE77A17EE02
:109C8800103A2033402B00F217879FED467AF4EE06
:109C9800C77AF1EE10FA41F3AF82DFED435A9FED38
:109CA800436A01E0F0EE477AF4EEC67AF1EE10FA74
:109CB80037EEE57AF6DCDFED3E7AB4EEE77AF1EEE0
:109CC80010FA41F19D82DFED385A9FED3A6A01E0C2
:109CD800B0EE677AB4EEC67AF1EE10FA77EE257A2E
:109CE800F6D49FED2E7AF4EEC77AF1EE10FA00F36F
:109CF80023869FED317AF4EEC77AF1EE10FA44BF6D
:109D08009FED2B7A77EE677A67EEA75A9FED2B5A6D
:109D18009FED2B6A9FED2B7AA5EE856A27EEA55A53
:109D2800A5EE867AE5EE077A039A92ED016AD2EDFE
:109D3800005A27EEC67A65EEA77AA5EEA67AE6EE71
:109D4800267A82ED007AC2ED017A002E3FF450AFF8
:109D5800089B1978099B01F00101186804F0EEFBD3
:109D680013B0BDEC028BBDE8F08F00BF18E202080B
:109D7800D15A002000210020A4210020343C0020DA
:109D8800D42300201F85EB51D42B0020D859002064
:109D9800676666661C3A002035FA8E3CDB0FC93FC1
:109DA80000000000DB0F4940DB0FC940E4CB16413F
:109DB800DB0F49C0E4CB16C1DB0FC9BF92E741B93D
:109DC8009730083C15A82ABEB64B06931B689F0718
:109DD8007FF558ADB44CB4F8008018F0010F7FF44B
:109DE80074AD48F00103984523803FF46EADAF4B46
:109DF800022214211A700E20FF2259709A700DF059
:109E080053FEB4F8008060E522F480739BB29A4256
:109E180023807FF4B4ADA64B1B78082B7FF4BEAD2E
:109E2800228822F040039BB29A4223803FF4B9ADC6
:109E38009E4B02201421FF2218700E2059709A7030
:109E48000DF032FEADE5029B588B8142C0F21484BE
:109E5800B1F5FA6FD4BFC0EB0101C0F5FA614FF458
:109E68007A7303FB01F1934B1D78C0F5FA60B1FBDF
:109E7800F0F1002D3FF490AE5B788F4801FB03F3BF
:109E880080FB0301DB17C3EB611185E6DFED8B7AFD
:109E980043E6DFED8A7A23E6B1F5FA6F80F2EF83C5
:109EA800187A8B1A03FB00F3C2F5FA6293FBF2F3FC
:109EB800C3F1640307EE903AF8EEE77A9FED807AF3
:109EC800804B67EE877AC3ED007AE8E57E4B1B7816
:109ED8000693002B7FF4D4ADDFF81CA2DFF81C92A8
:109EE8001AF8030C99F800805146AAF1030708F004
:109EF80073F9002800F0C983069BB8F1000F53D10D
:109F080007F10801787908F067F9002841F0D9814C
:109F18006E49B87A08F060F9002800F0CA83B8F1F1
:109F2800020F41F0D1816A49F87B08F055F9002801
:109F380041F0A7816749387D08F04EF9002800F004
:109F4800CA83B8F1040F41F09F816349787E08F015
:109F580043F9002841F09B816049B87F08F03CF93B
:109F6800002800F0CA83B8F1060F41F093815C49DC
:109F780097F8230008F030F9002840F04487594941
:109F880097F8280008F028F9002800F0CA83B8F1EB
:109F9800080F40F04987544997F82D0008F01CF93C
:109FA80000283FF46DAD09231A4600F02EBF13B9FF
:109FB80001238BF802304D4B05931B201F789BF82B
:109FC800216008F033F9012E07F00109824600F0FC
:109FD800578607F0020303939BF82030DFF82081AF
:109FE800434C052B00F29C80DFE813F08C005000F6
:109FF8000600DD000101BF00012E04BF05238BF818
:10A008002030B9F1000F00F01581029B394FB3F9E8
:10A018001810B8F80030002261F30F0263F31F42F2
:10A02800002361F30F0361F31F436A603968DBF8AB
:10A0380014202B608A42C0F04E84012E41F07B82AE
:10A0480003229BF820300392CBE708F0F5F80128AB
:10A0580008D1284FB8F802303A68642101FB03237D
:10A06800CBF81030BAF1000F04D098F80630002B66
:10A0780040F09080012E53D01E4FDBF810203B6833
:10A088009A42C0F0788601238BF82030012E6CD0DC
:10A0980098F80730012B00F0D7800BF047F99BF8B0
:10A0A80020309EE78C5900205A320020D8440020E6
:10A0B8007C3C0020D42300201F85EB5100000000C9
:10A0C8000AD7233CA4210020D15A0020A444002010
:10A0D800A9440020AE440020B3440020B844002026
:10A0E800BD440020C2440020C7440020D05A0020AC
:10A0F800A25500206C5700209A44002080000020C0
:10A108008C2F0020B9F1000F9FD14FF48060BAF175
:10A11800000F00F0C4830DF0E5FD0023CBF81030EC
:10A12800039B002B3FF448AA03980DF0BDFC049B49
:10A138001F6817F480593FF445AA1D21B64802F05C
:10A1480037FB00287FF43EAAB44A029BD2881B8BB7
:10A15800B5F90660991A8E4240F3028613449E426E
:10A16800B4BF00260126FFF735BAAD4F3A68B8F8F4
:10A178000230642101FB03234FF480600022CBF8F6
:10A1880010308BF820208BF803200DF093FD9BF8FE
:10A19800203026E70BF0CAF803224FF47A738BF8C5
:10A1A8002020CBF81C309E4F238843F002032380E5
:10A1B8000EF0E8FB3A68DBF81C3013440422CBF8B5
:10A1C80018308BF82020012E40F0CD853B68DBF855
:10A1D80018209A42A4D2934B187818B908F026F898
:10A1E80000289DD1238823F002032380BEE78C4FEB
:10A1F800E9E7029A013BD27D35F91330002A40F095
:10A208006583A3F57A73B3F57A7FA8BF4FF47A73A1
:10A2180023EAE37307EE903A9FED837AF8EEE77A44
:10A2280067EE877A814AFCEEE77A17EE903A138058
:10A23800FFF7B7B97A4F3B6847F230520323CBF8A0
:10A248001C208BF82030AFE70BF070F8032240F6A3
:10A25800B8338BF82020CBF81C30714FA4E7744F2B
:10A268003B78002B00F0DC87724BDFF8DC81DFF8ED
:10A27800DCB1DFF8DCA1029345465E4603909946BF
:10A288000EE019F804109847032C28DC88B93B78AD
:10A298002AF8020F01349C4205F1040580F20C8172
:10A2A800072CE1B23046DBF80430EADD984700B20B
:10A2B800EDE738F824206B88801A4FF47A719B1ADE
:10A2C80001FB00F040F6CA0290FBF3F0084490420C
:10A2D80040F2EE23A8BF10469842B8BF184600B215
:10A2E800D5E7DFF870A1DFF87081534C0AF15A0600
:10A2F8004FF0010951461AF8010C07F06DFFF8B14B
:10A308009AF804009AF802309AF803E000EB40014A
:10A3180004EB8101013BD1F8B42003EB4303434430
:10A3280093420DD094F8E02081F8B0E009FA00F0EB
:10A3380022EA0000C1F8B430C1F8B87084F8E0002F
:10A348000AF1060AB245D5D13C4B07931946344A5F
:10A358003B4B3C4C09681B78D2F800900891069357
:10A36800A4F1B00A002663685BB31F784FB3A268F4
:10A37800A9EB0202002A0ADB9AF8E0200121B14089
:10A3880022EA010209F5FA718AF8E020A160069A2A
:10A39800BAB1227859780432D2B2002940F0BA8290
:10A3A800029935F91220098B01F1C800824240F365
:10A3B800A9849AF8E0109A7841FA06F3D90740F18F
:10A3C8001D850136042E04F10C04CCD1FFF74CBADC
:10A3D800194C94F8AA3053B1059B1B78D80706D5B9
:10A3E800029BB5F906205B8B9A4200F3DC841121AD
:10A3F800094802F0DDF9002800F0748294F8AE30C4
:10A408002BB994F8A83013B93223A4F8AC3001233F
:10A4180084F8AE30FFF7BCB9043C0020742F00204C
:10A428006C570020441B0020AAF1823F583A0020B4
:10A438003431002030530020FC210020D02B002094
:10A448005C5A0020AC220020AC340020605A002066
:10A45800FA210020B1430020C0C702081D21B748D7
:10A4680002F0A6F900283FF4BDAB9BF80330002B9F
:10A478007FF4B8ABDFEDB27AB24938EE678AC7F538
:10A48800FA63FDEEC87A1BB2CDED027ABDF9082059
:10A49800120381FB0201D217C2EBA11203FB02F3E4
:10A4A80043F30F333B4407EE903A039BF8EEE77A09
:10A4B800C3ED037AFFF796BBDDF80C90A24A04922D
:10A4C8001146A04A096842F2010AA2FB092B11EAC7
:10A4D8000A0A4FEA9B1B00F001829C4D9C489D4C48
:10A4E8009D4A95F800E0007884F800E01070BEF10D
:10A4F800000F04D0984A92F800E08EF0010E974CB5
:10A508000F2084F82400002B00F05C83944B0B93FD
:10A518001B780A931E463B78029F924AB7F824C0DC
:10A52800DFF8748209903D46FF8C08973746A2FBF6
:10A53800066252082D8B0E9502EB420294F82550C4
:10A548000C95BA1AD2B201F48051079204F1280688
:10A558000BF596726746844DCDF80CE0A446544638
:10A56800DDF830A00F9100200592CDF834909E467A
:10A57800039B002B00F03D823CF910101FFA81F973
:10A58800B9454FEA400203D3089B994540F27382CC
:10A5980058F820108B4580F03582A95E002C40F0D9
:10A5A800498201307045A95206F10606E0DB099898
:10A5B8006E4ADDF834908CF824000F286446514622
:10A5C8000CBF01210021734684F825A0117000F00A
:10A5D800FF82DFF8C8B1664E664F34883868DBF80A
:10A5E8000810DBF80420CBF80C0044F00404401AEF
:10A5F8009042574F3480584C4FF0010188BF0022D9
:10A608003970217088BF8BF82120002B00F0F5826B
:10A61800049A02991768584EB1F824C0B1F818E0A6
:10A62800514817F48057344640F00C8339460EE001
:10A63800627802EB820202EB820202F2EE2292B20E
:10A6480001318B4220F8022B04F102040ED016F8D7
:10A658001120002A00F01382022AE9D00131028871
:10A6680020F8022B8B4204F10204F0D10B9A1378E4
:10A6780001331370FEF788BF1146FFF7F4BB1B7A4E
:10A68800C3F1640307EE903A16E40AF105017879FC
:10A6980007F0A2FD00283FF43BACB8F1010F40F0F1
:10A6A800108607F10D01B87A07F096FD002840F0F2
:10A6B8000B863249F87B07F08FFD00283FF43AAC4F
:10A6C800B8F1030F40F0DD852D49387D07F084FD92
:10A6D800002840F0D9852B49787E07F07DFD0028B9
:10A6E8003FF43AACB8F1050F40F0D1852649B87F60
:10A6F80007F072FD002840F0CD85244997F8230023
:10A7080007F06AFD00283FF43AACB8F1070F40F0B3
:10A718007A831F4997F8280007F05EFD002840F06B
:10A7280083831C4997F82D0007F056FD00283FF455
:10A73800A7A9B8F1090F3FF4A3A934E4043C002009
:10A7480000007A44D34D621098510020B82F0020A1
:10A75800C00000205C5A0020C1000020FC2100201D
:10A76800E1300020ABAAAAAA026700205D5A0020A7
:10A77800A25500206C570020E0340020A944002096
:10A78800AE440020B3440020B8440020BD4400205B
:10A79800C2440020C7440020E4300020385A00207A
:10A7A800CD4CD4F88830A9EB0303002BFEF6F9AEA4
:10A7B800CA4A94F88C30517C069AC4F88820013330
:10A7C800C74A029E32F81120B17D03F00F0384F8C6
:10A7D8008C30234492B292FBF1F283F8902094F8E3
:10A7E800901094F8912094F8923094F89C000A44C0
:10A7F80094F89310134494F89420194494F89530DD
:10A808000A4494F89610134494F89720194494F83D
:10A8180098300A4494F89910134494F89A201944EB
:10A8280094F89B300A44134494F89D1094F89F20A0
:10A83800184494F89E3001440B441A4442F30B1216
:10A84800642AF17DA8BF642213B209B1C2F164037E
:10A8580007EE903A9FEDA37AF8EEE77AE0E402215A
:10A86800A14801F0A5FF00283FF42FA8268018F082
:10A87800020F7FF43CA848F00203434523803FF4CD
:10A8880036A89A4B022214211A700E20FF22597002
:10A898009A700DF009F9B4F80080FFF728B80DF0A8
:10A8A80009FA3AE4228822F040039BB29A422380B4
:10A8B8003FF448A88D4B02201421FF2218700E2067
:10A8C80059709A700DF0F0F8FFF73CB8C3F53B6388
:10A8D80008331BB295E403230393ADE4844A92F84A
:10A8E80000E004E694F8A830002B3EF451AF059B35
:10A8F8001B7813F001037EF44BAF012284F8A830D3
:10A9080084F8A920FEF744BF734C012184F8A010F5
:10A91800FEF7DDBE012900F032849AF8E020012319
:10A92800B34001361343042E8AF8E03004F10C04D6
:10A938007FF419ADFEF798BF9FED797A77EE677AC5
:10A94800FFF7E2B9059B6B4A1B781060DB0700F143
:10A95800388294F8A60000287EF413AFB4F9A43026
:10A96800322B7EF70EAF94F8A2200121572A84F8E3
:10A97800A61000F09284049B1B6813F0040302D015
:10A988005A2A00F04F855D2A00F0FB845B2A00F00C
:10A9980021855E2A00F02285562A00F03485972A00
:10A9A80000F02785A72A40F0B3845349049B0A780E
:10A9B8001B6842F004020A7003F00403FEF7E5BEC8
:10A9C800B2F5FA7FFEF6DDAE94F8A620002A7EF4F2
:10A9D800D8AE059B1B780121DF0784F8A61000F18B
:10A9E8008F840DF015FB049B1B6803F00403FEF72E
:10A9F800CCBE002F3DD058F820108B454FEA4002BE
:10AA0800FFF4CBAD3D4B995C03EB0209002900F044
:10AA1800F980022946D199F8011001EB810101EB77
:10AA2800810101F2EE2189B2032832DD09B2002C3E
:10AA38003FF4B7AD079B26F81310BAF1000F03D106
:10AA48000A9B022B7FF6ADADB6F800A07188B6F868
:10AA580004902B4B514489440FFA89F983FB09313F
:10AA6800284BA1EBE97123F8029009B24FF0010AD3
:10AA780097E539464200059B48F820308EE5CAB272
:10AA8800022A04D9032A7FF4E9AD6246D8E5724662
:10AA9800D6E5012303FA00F9099B23EA090309B261
:10AAA80009937BE5A95ABFE743F04002934222800D
:10AAB8007FF400AFFEF746BFDFED137AFFF734B936
:10AAC800F4EEC77AF1EE10FA40F3A783DFED115ADE
:10AAD8009FED0E6A2EE000BFFC210020E456002006
:10AAE8000057002014AE2341043C0020D844002025
:10AAF8005C5A0020243A0020CC3F0020E03400209B
:10AB0800565555556C22002000000000E4CB164134
:10AB1800DB0F49C0DB0FC940E4CB16C1DB0FC93FCF
:10AB2800DB0F494092E741B99730083C15A82ABE87
:10AB3800F0EE476AF4EEC66AF1EE10FA36EEE57A00
:10AB4800F6DC5FED0D6AB4EEE67AF1EE10FA40F14C
:10AB580087835FED105A1FED106A01E0B0EE667A48
:10AB6800B4EEC67AF1EE10FA77EE256AF6D41FED48
:10AB7800157AF4EEC76AF1EE10FA40F39F801FEDE4
:10AB8800187A77EE666A66EEA65A1FED1A5A1FED16
:10AB98001A6A1FED1A7AA5EE856A26EEA55AA5EE61
:10ABA800867AE5EE076AFFF768B83946C24801F0C9
:10ABB800FFFD00283FF4C6AE84F8A7700DF028FA10
:10ABC800FEF7DABDBD49BE4A0B91BE4D0121117099
:10ABD8001B21B948039301F0EBFD039B00287FF488
:10ABE800F8ACDFF800B3B84FDBF80C203B68CBF8C3
:10ABF80008309B1AC82B00F23683049B1F6807F4A1
:10AC0800805733E5C1B2022940F2B78203297FF4A5
:10AC180049AF0E9B19460F9B002B08BF394603E727
:10AC280028F0010292B2424522803FF420AE0E2065
:10AC380086F80090777086F802A00CF035FFB4F81B
:10AC4800008014E600210FE0627802EB820202EB3A
:10AC5800820202F2EE2292B20131994220F8022BCE
:10AC680004F102043FF402AD16F811201AB1022AC9
:10AC7800EAD00288F0E7CAB2032AFAD87246EBE7AC
:10AC880000230393FFF7A8B9B2F5FA7FFEF679AD72
:10AC980094F8A630002B7EF474AD059B1B78012137
:10ACA80013EA010084F8A61000F0BE820DF06AFED7
:10ACB800049B1B6803F00403FEF767BD9FED837ACE
:10ACC800F4EEC76AF1EE10FA44BF9FED817A77EE91
:10ACD800666A58E77F4A80491068B4F9A420C769B2
:10ACE80081FB07018911FF17781A00F5FF407F30B3
:10ACF80082423EF734ADC91B0A4412B2A4F8A4201C
:10AD0800FEF72DBDC8398A4240DA9AF8E0109A78E1
:10AD180041FA06F3DB073FF554AB52420120099292
:10AD28000CF0B0FF7B1E099A162B00F21B81DFE89E
:10AD380013F0BC01D201A301FB01E8010F02760167
:10AD480061014A0133011C011901FB0109010F02CC
:10AD580076016101F300DD00AC008B0194007E00F8
:10AD68000126FEF737BC3A68DBF81C301344CBF8F1
:10AD78001830FFF7D5B90AF0D9FA032240F6B833EC
:10AD88008BF82020CBF81C30FFF70EBA9AF8E03089
:10AD98000122B24023EA020309F5FA728AF8E03088
:10ADA800A260FFF70EBB0021434801F001FD002817
:10ADB8007FF41DAB322384F8AA00A4F8AC30FFF767
:10ADC80016BB464B1B78002B3EF4DBAC9BF80330DC
:10ADD800002B7EF4D6AC94F8A7300133DBB2032BFA
:10ADE80084F8A7307EF6CDAC3D4B5B7813B9002EC6
:10ADF8007EF4C7AC0DF0C6FDFEF7BEBC002A0CBF42
:10AE0800012002208BE707231A4602EB820217442F
:10AE180089F80030B97878781CF0E0F8059B1E783E
:10AE280006F00106FEF72CBE08231A46EDE7DAF80D
:10AE3800E400DFF8B48090F8361098F80230114436
:10AE48006429A8BF642121EAE17180F83610002B3B
:10AE580040F0658309F0AAFB5FE5DAF8E400DFF863
:10AE6800888090F8371098F802301144FE29A8BF5E
:10AE7800FE2121EAE17180F83710002BEAD0162074
:10AE880007F00CFADAF8E400E4E7DAF8E400DFF8AF
:10AE9800588081781144C829A8BFC82121EAE171E6
:10AEA800817098F80230002BD4D0142007F0F6F9FE
:10AEB800DAF8E400CEE700BF043C0020E1300020CF
:10AEC8005D5A0020026700206C570020DB0FC9BFC5
:10AED800DB0F49C024480020D34D62105C5A002083
:10AEE800583C0020385A0020EC680020DAF8E400CA
:10AEF800DFF8A48641781144C829A8BFC82121EAEF
:10AF0800E171417098F80230002BA3D0132007F0AC
:10AF1800C5F9DAF8E4009DE7DAF8E400DFF87886A6
:10AF280001781144C829A8BFC82121EAE17101703C
:10AF380098F80230002B8DD0122007F0AFF9DAF81C
:10AF4800E40087E7DFF85086089898F802304179DE
:10AF580011446429A8BF642121EAE1714171002BE1
:10AF680040F03E83DAF8E40074E7DAF8E400DFF84A
:10AF78002886017A98F802301144C829A8BFC82148
:10AF880021EAE1710172002B3FF464AF0B2007F056
:10AF980085F9DAF8E4005DE7DAF8E400DFF8F88527
:10AFA800C17998F802301144C829A8BFC82121EAFC
:10AFB800E171C171002B3FF44DAF0A2007F06EF923
:10AFC800DAF8E40046E7DAF8E400DFF8CC858179BE
:10AFD80098F802301144C829A8BFC82121EAE171B4
:10AFE8008171002B3FF436AF092007F057F9DAF8E2
:10AFF800E4002FE7DAF8E400DFF89C85417998F857
:10B0080002301144C829A8BFC82121EAE171417161
:10B01800002B40F0C882112F7FF43BAF1AE7DAF813
:10B02800E400DFF87485017998F802301144C829E2
:10B03800A8BFC82121EAE1710171002B40F0738299
:10B04800102F7FF457AF05E70898DFF84C85417853
:10B058001144B1F5967FA8BF4FF4967121EAE171CA
:10B06800417098F80230002B3FF47CAF152007F0B0
:10B0780015F9DAF8E400EDE60899DFF81C850F7990
:10B088001744642FA8BF642727EAE7770F7107F0F2
:10B098001FF998F80230002B3FF464AF03203946BB
:10B0A80007F0FCF8DAF8E400D4E60898DFF8E8845A
:10B0B80001781144FA29A8BFFA2121EAE171017047
:10B0C80098F80230002B3FF44DAF012007F0E6F866
:10B0D800DAF8E400BEE60898DFF8BC848178114409
:10B0E8006429A8BF642121EAE171817098F80230CF
:10B0F800002B3FF437AF022007F0D0F8DAF8E4006D
:10B10800A8E60898DFF89084C17998F802301144CD
:10B1180081F30801C171002B3FF424AF052007F02B
:10B12800BDF8DAF8E40095E6089BDFF86C849979B5
:10B1380098F8020011446429A8BF642121EAE1714A
:10B148009971002840F037820D2F7FF4FDAE09E792
:10B15800DAF8E400DFF84084C17898F80230114446
:10B16800C829A8BFC82121EAE171C170002B40F0AD
:10B17800B3810F2F7FF4D4AE6CE60E9954E435F901
:10B1880012209978B2F5617F4FF4966393FBF1F33F
:10B198003ADB40F633019142A8BF11460C2FA1F5C6
:10B1A800617191FBF3F100F0FB80182F7FF4B5ABD0
:10B1B800C9B2C8290B46A8BFC823DAF8E400C27D83
:10B1C800DFB297423FF4A9AB9A1ADFF8CC83C77570
:10B1D80048BF0732D71098F802300137FFB23BB9A1
:10B1E800002F3FF49AAB38460CF04CFDFFF795BBA7
:10B1F800182007F053F8F3E7B0EE677AFEF75BBD67
:10B20800F0EE477AFEF76DBD0C2F00F0E080182FA6
:10B218007FF483AB00210B46CFE7B0EE667A90E46B
:10B22800C74A0292FFF74AB9C64B1B6813F40033AA
:10B2380040F0D8801846C4490E5C0F2E00F10C006F
:10B2480045D00133152BF7D1049B1B68FA3A00212E
:10B25800A4F8A42003F0040384F8A610FEF795BA16
:10B26800F0EE476A83E4B94A049B1F68138823F009
:10B2780004031380012307F480578BF82130FFF76C
:10B28800F5B903231A46C0E504231A46BDE505238C
:10B298001A46BAE506231A46B7E5AD4BAD491A6812
:10B2A8004FF47A73B3FBF2F3C3EB431203EB82025E
:10B2B800049B1B68D200A1F8B42003F00403FEF736
:10B2C80064BA01231A46A0E502231A469DE5A24F57
:10B2D800D7F800E05800BEF1000F07D0C61801EB00
:10B2E80086069EF801E076787645ADD218449B4EE6
:10B2F8009B4B01EB80010020396030801860A3E788
:10B30800049B98491B680A6003F00403FEF73DBAE2
:10B318000021BB2A109100F0C980B72A00F0C28032
:10B32800BE2A00F0BD80BD2A00F0A380792A00F073
:10B33800EF807A2A00F0E5809E2A00F0DC809D2AC2
:10B3480000F0D280AE2A00F07681AD2A00F06C8140
:10B35800EF2A00F06381FD2A00F05A81FB2A00F0F1
:10B368005181FE2A00F04881F72A00F03F817B2AAC
:10B378007EF407AA4FF4FA61022019F045FCFEF7A3
:10B3880000BA794B002201207849794C0B60227071
:10B398000CF078FC049B1B6803F00403FEF7F5B976
:10B3A800CFB2734B09915B78BB423FF4B6AADFF882
:10B3B800E881384619F0F4FC98F8023009991BB175
:10B3C800C9B20C2006F06AFF0137FFB208E7002770
:10B3D8003946E6E7674B01220220D5E7664B022291
:10B3E8000320D1E7654B1B78032B00F0D780034679
:10B3F80021E7049B624A1B684FF4C871118003F06F
:10B408000403FEF7C2B90AF0C5FB00F0A1FD0AF07B
:10B41800A9FB04F0CFF801200CF034FC94F8A2202A
:10B42800FFF7BDBA94F8A820002A40F0D38094F81A
:10B43800AA3083F0010384F8AA30002B40F0C180C1
:10B448000C200CF031FB049B1B6803F00403FEF78F
:10B458009CB9002E3EF40EA94A4C94F8A130002B5A
:10B468003EF43AA90CF002FB002384F8A130FEF761
:10B4780033B94FF6FE73444AD08996890144334460
:10B488009381D1810AF086FB00F062FD0AF06AFB25
:10B4980004F090F801200CF0F5FBB4F8A420D3E6F2
:10B4A8000223E8E70B464FF6FE71E4E70B4602215C
:10B4B800E1E7344C0DF066FA002384F8A130FEF77A
:10B4C8000BB9002BC8D03149314A09684FF47A705A
:10B4D80000FB03131360BFE70F20099206F0DEFE9E
:10B4E800DAF8E400099A44E60021FF201EF072FC15
:10B4F80094F8A22026E701201EF06CFC94F8A22004
:10B508001DE7244A137A43F001031372FEF739B991
:10B51800204A137A23F001031372FEF732B9172079
:10B5280006F0BCFE1EE51020099206F0B7FEDAF818
:10B53800E400099A84E503230393FEF7F5BD00BFF1
:10B5480030530020A4430020B8DE0208A255002092
:10B5580088510020044F00209C210020F021002069
:10B56800F4210020243A0020D0670020EC59002064
:10B57800DE5900201E6800206C68002078430020F7
:10B58800666A0020FC2100203C3C00206C5700200B
:10B59800203A00201C5A0020EC6800200CF066FAC3
:10B5A800B4F9A42050E61120099206F077FEDAF8E3
:10B5B800E400099A2FE50D20099206F06FFE099A1A
:10B5C800C2E50B200CF070FA049B1B6803F004031F
:10B5D800FEF7DBB884F8A80084F8A910FEF7D5B800
:10B5E8000E2006F05BFEDAF8E40033E400210420C4
:10B5F80019F00AFBFEF7C5B80021032019F004FB77
:10B60800FEF7BFB80021022019F0FEFAFEF7B9B81C
:10B618000021012019F0F8FAFEF7B3B80021084616
:10B6280019F0F2FAFEF7ADB8FF2100201EF0D2FBA8
:10B6380094F8A2208CE6012100201EF0CBFB94F8A0
:10B64800A22082E6002870B51EDB0928044620DD0A
:10B65800012303EB83035B00B0FBF3F2092AF8D85C
:10B668007BB10E4EB4FBF3F00928CCBF5722302231
:10B67800A6FB03E5024403FB1044EB0801F8012B89
:10B68800F0D100230B7070BD2D230B7040420131A7
:10B69800DBE7303001F8010BF3E700BFCDCCCCCCB1
:10B6A800884230B44FF001042ED301FB04F4B0FB00
:10B6B800F4F58D42F9D284B1AAB901E0B0FBF4F5F2
:10B6C800092DCCBF572230222A4404FB150003F869
:10B6D800012BB4FBF1F4002CF0D100221A7030BC1D
:10B6E8007047B0FBF4F5092DCCBF372230222A442D
:10B6F80004FB150003F8012BB4FBF1F4002CF0D186
:10B7080000221A7030BC70470546002AEBD1D7E7F3
:10B7180003685A1C02601970704700BF2DE9F04792
:10B72800089C2578002B804689460CBF4FF0200ADC
:10B738004FF0300A661C35B3002A29DD334601E094
:10B74800024698B113F8011B501E0029F8D1971E24
:10B7580060B13D46013D51464046C8476B1C002B31
:10B76800F8DC257827EAE770013055B1041B294633
:10B778004046C847301916F8015B002DF7D1BDE8DF
:10B78800F087BDE8F087002A04DC2846BDE8F0878A
:10B798000020EBE7571EDCE783684268D0ED037AA8
:10B7A80000EB83010133934281ED040A836004BFF7
:10B7B8000023836000EB830393ED047A036870EE43
:10B7C800277A9A42C0ED037A77EEC77AC0ED037AFA
:10B7D8000CDA013307EE103AF8EEC76AB7EE007AD2
:10B7E80087EEA60A036030EE070A704707EE102AB4
:10B7F800B8EEC77A87EE870A704700BF90ED057AE2
:10B8080090ED004AD0ED066AD0ED014AD0ED047AF9
:10B8180090ED035AD0ED025AA4EE007AB0EE406AD9
:10B82800B0EE470AB0EE667AA6EE247A67EEC07AE2
:10B83800A0EE457AE6EE257A80ED057AC0ED067A27
:10B84800704700BFD0ED057A90ED013AD0ED003A8F
:10B85800D0ED064A90ED024A90ED077A90ED035A32
:10B8680090ED086AD0ED045AC0ED067AF0EE406A11
:10B8780027EE830AC0ED056AA3EEA60A80ED087AD2
:10B88800A4EE240AA5EE470AA5EEC60A80ED070A2B
:10B89800704700BFD0ED007A90ED017A30EE670A6C
:10B8A800E7EE007AB0EE670AC0ED007A704700BF95
:10B8B800704700BF0A44914214D030B40139551E74
:10B8C80041F2210211F8014F082380EA0420040400
:10B8D8004CBF82EA40004000013B80B2F7D18D4264
:10B8E800F0D130BC704700BF50F8043C012280F80A
:10B8F8004520103803B11847704700BF90F8203032
:10B9080033B1012B03D14FF4006383827047704732
:10B918004FF480638382704770B5044682B0143058
:10B92800E56D06236A464321A847B0B19DF8040097
:10B938009DF800609DF801109DF802509DF80320C5
:10B948009DF8053041EA062143EA002342EA052230
:10B95800A187E287A4F84030012002B070BD00BF83
:10B9680070B5044682B00830656A06236A463B21F2
:10B97800A847A8B19DF804009DF800609DF8011043
:10B988009DF802509DF803209DF8053041EA0621F4
:10B9980043EA002342EA0522E182228363830120ED
:10B9A80002B070BD70B40468037B2268022101FAFA
:10B9B80003F31A4213D042690A49582000FB0212C5
:10B9C8004FF6FE7650685289C5680068296831408C
:10B9D8002960C168D24392B20A40C260636070BCF9
:10B9E800704700BFE84B002030B4094B1C7864B1A5
:10B9F800084B002503EBC4041A6899885562D0687F
:10BA080008330143A342D160F6D130BC704700BF70
:10BA1800A84E0020AC4E0020F0B4334C00EB800060
:10BA280004EB80046468002C5BD0304E49004FF46E
:10BA38002040CDB23060A169090444D460682C4F1D
:10BA480045F08071384041F4903101434FF4204073
:10BA58006160306003E0411E002838D00846A169C3
:10BA68008F07F8D54FF42040A262306002E0421EF2
:10BA780068B31046A2691106F9D562681C4945F0F9
:10BA8800007545F480350A4015434FF42040656041
:10BA9800306002E0421ED0B11046A2699207F9D583
:10BAA800A362A3694FF420409B06306005D4431E6F
:10BAB80068B11846A3699B06F9D520233060E36175
:10BAC8000120F0BC7047411E08B10846B3E7094A97
:10BAD800138801339BB24FF0FF3131601380F0BC03
:10BAE80070472046F0BC70470857002030570020A8
:10BAF800009800FC34570020B0F1FF3F09D002281D
:10BB080010B402DC5DF8044B86E700205DF8044BB6
:10BB180070470020704700BF9AB170B505460C46C3
:10BB28008E1801E0B4420AD014F8013B697995F9FE
:10BB380004008022FFF7E0FF0028F3D170BD012048
:10BB480070BD0120704700BF134600200A466821D7
:10BB580062E70023262203600270272282700122F6
:10BB680043600271837170472DE9F3410569064608
:10BB78000F467DBBD0F80080C8F30A0323B3002327
:10BB8800D6F80080019314F0A3FD042819D1224CA3
:10BB9800236943F001032361BBB2A8F8003014F015
:10BBA80097FD04282ED108F102030193019B3F0C55
:10BBB8001F8014F08DFD2369042823F001032361FD
:10BBC80025D06FF0010505E014F082FD042805D0AA
:10BBD8004FF0FF35284602B0BDE8F0810E4C2369CE
:10BBE80043F002032361C4F81480236943F040033F
:10BBF800236114F06DFD2369042823F002032361F7
:10BC0800BDD0E5E7236923F001032361D9E7336851
:10BC180004333360DEE700BF00200240F8B5044675
:10BC28000D468E180027B54201D12069F8BDE3689A
:10BC3800591CE160234415F8012B1A720429F2D12A
:10BC4800A1682046FFF790FFE7602061EBE700BF9F
:10BC5800014B186801F07CBC3056002070B50446D2
:10BC680090F85900002833D104F11405236E80227E
:10BC78006B2128469847642001F04CFA236E284629
:10BC880003226B219847236E94F8542019212846E3
:10BC980098470F2001F03EFA236E94F85220284668
:10BCA8001A219847236E284618221B219847236E8D
:10BCB800284618221C219847236E2846022237213D
:10BCC80098472846236E01223821BDE8704018475E
:10BCD80001F0D6FF0546F0B1036881881B8A194038
:10BCE800C2D12023C171837102F060FA2146104B42
:10BCF80041F8103F284619F09FFEAB88B3FA83F34A
:10BD0800C3F11F035A1CAFD001229A4009490B689E
:10BD180013430B60A8E7014602F048FA2146044B9A
:10BD280041F8103F284619F087FE0122EEE700BFD0
:10BD3800F1B80008000401400846194619F0ECB9AA
:10BD480010B490E80600047B40690223A3404B60CE
:10BD580013685DF8044B4FF6FE710B40136001F059
:10BD680097BB00BF0B490C4A0C4808B58B6943F0D8
:10BD780001038B61136843F4805313600021402250
:10BD880020F0F2FA064B4FF0FF321A60C3F8032096
:10BD980008BD00BF00100240000001407C57002091
:10BDA800BC5700202DE9F041044618460D461646BA
:10BDB80098461DF085FA2768E6722844A07229463D
:10BDC8007D69434632462046AC46BDE8F0416047AF
:10BDD800036810B504461B689847236820469B688B
:10BDE8009847A37B0133A37310BD00BF427A02B901
:10BDF800704710B504460368406804F10A01984783
:10BE08000023637210BD00BF437A5A1C0344D2B2A8
:10BE180042729972037A934200D802B9704710B5FA
:10BE280004460368406804F10A01984700236372D6
:10BE380010BD00BF10B40B49002301E0272B0CD024
:10BE480011F8132082424FEA430403F10103F5D1AC
:10BE580021445DF8044B4878704700205DF8044B96
:10BE6800704700BF08C8020870B5448806460D46EA
:10BE7800C4F30B0422460021284620F075FA3369E2
:10BE8800094A934209D3094A934206D222462846D0
:10BE98001946BDE8704020F042BA23B12146284631
:10BEA800BDE87040184770BD08220308FC2203084B
:10BEB800064B07498B4202D30023184670471A885D
:10BEC800C2F30B029042F8D01433F3E7F81D0308CD
:10BED80008220308024A136823EA0000106070472A
:10BEE8005C3C0020F8B5174D2B78A32B28D16B7834
:10BEF800BE2B25D1022229464FF6FF70FFF7DAFC48
:10BF0800114FAC1C22884AB1A618BE4218D2052A85
:10BF180016D92146FFF7CEFC3446F3E72146022224
:10BF2800FFF7C8FC0222A118FFF7C4FC0634074B30
:10BF3800641B1C8041F60F53C31A58425841F8BD80
:10BF48000020F8BD00F00308000004087A43002030
:10BF58002DE9F04FDFF848914C4F8BB00326A7EB43
:10BF680009071822002104A820F0FEF9484BCDF853
:10BF7800109005971A69120604D5464A5A6002F1CC
:10BF880088325A6001228DF824203422DA60424B2C
:10BF9800424C1B88ADF800300222694604A8FFF71E
:10BFA8003DFE022269464FF6FF70FFF783FCDFF87B
:10BFB800F4A080464FF0000B544536D30AAC002558
:10BFC80024F8245D0222214604A8FFF727FE022256
:10BFD80021464046FFF76EFC40BAC043ADF8080062
:10BFE800022202A904A8FFF719FE079860B106AB60
:10BFF800C0F104022946184420F0B6F9069904A8AD
:10C00800FFF7B2FD079508909DF82430089A23B1F0
:10C018001F490B6943F080030B61013E2DD0002AB4
:10C028009FD1FFF75FFF50B32CE065888DF80DB006
:10C03800C5F30B05AB1DADF808302388C3F30B021D
:10C04800ADF80A201B0B062202A904A88DF80C30B3
:10C05800FFF7E4FD062202A94046FFF72BFC6168C2
:10C0680080462A4604A8FFF7D9FD616840462A465B
:10C07800FFF720FC143480469EE7002AD1D0052023
:10C0880003F064F90BB0BDE8F08F00BF00000408AE
:10C09800002002402301674556C80208F81D03081E
:10C0A80000F00308082203080378202B024600F159
:10C0B8000100F9D0092BF7D02D2B2CD02B2B03BF47
:10C0C8005378B7EE000A0246B7EE000AA3F1300132
:10C0D800C8B209289FED467A10D8F2EE046A07EE36
:10C0E800901AF8EEE77A12F8013FE7EE267AA3F104
:10C0F8003001C8B20928B0EE677AF0D92E2B4CD09F
:10C1080003F0DF03452B0BD0F7EE007A67EE276AC2
:10C1180020EE260A70475378BFEE000A0246D5E79C
:10C1280010B451782D2959D02B290ABF9178501C69
:10C13800901C0024A1F13003092B53D8002303EBF2
:10C14800830301EB430310F8011FA1F13002092A10
:10C15800A3F13003F3D9B3F59A7F28BF4FF49A734C
:10C16800072B42D9DFED236A1A46F7EE007A083A20
:10C17800072A67EEA67AFAD803F007032BB1F2EE86
:10C18800046A013B67EEA67AFBD124B3C7EE276A9F
:10C198005DF8044B20EE260A70475378A3F130016E
:10C1A800C8B2092802F10102AAD8F2EE046AF0EE38
:10C1B800665A07EE901AF8EEE77A12F8013F87EE12
:10C1C800A66AA3F13001C8B2092866EEA56A37EE5F
:10C1D800067AEED994E767EE276AD9E7901C91783A
:10C1E8000124A7E7F7EE007ACFE7F7EE007AC5E774
:10C1F8000000000020BCBE4CB5EEC00ADFED317A6D
:10C20800F1EE10FACCBF30EE270A30EE670ADFED08
:10C218002E7A20EE270A30B5FDEEC07A87B017EEE9
:10C22800904A054684EAE470002303A9A0EBE47071
:10C2380001930093029314F0ABFC002CACBF2023B5
:10C248002D2303A88DF800301DF03AF8012803A922
:10C2580024D002282DD0032805BF3023684668461D
:10C268008DF8013020F0A6F868461DF029F803384B
:10C27800C4B222466946284620F0FAF800232B5516
:10C2880028461DF01DF82E22431C2A540DEB0401EC
:10C29800E81820F0ACF8284607B030BD30236846CF
:10C2A8008DF801308DF802308DF8033020F082F8D7
:10C2B800DAE7302368468DF801308DF8023020F037
:10C2C80079F8D1E76F12033A00007A442DE9F0417A
:10C2D800064615460846B6FBF2F43CB905FB14645D
:10C2E800124B1B5D00F8013BBDE8F081B4FBF2F78F
:10C2F80067B90E4B05FB174705FB1464DA5D00F8B8
:10C30800012B1B5D00F8013BBDE8F081B7FBF2F89B
:10C31800B8F1000F02D04046FFF7D8FF05FB1878A8
:10C32800024B13F8082000F8012BE3E774ED02082C
:10C3380030B402681146531C036011F8024B0160C7
:10C34800D31C517803609378151D05601B0443EADC
:10C358000123D078234343EA006030BC704700BF14
:10C368000368591C1A46016012F8021B02605878CB
:10C3780041EA0020704700BF03685A1C0260187821
:10C38800704700BF38B50446006815461FF0C7FF60
:10C3980022682A44226038BD036810B40A0A5C1C6B
:10C3A80004601A7003685A1C026019705DF8044B27
:10C3B800704700BF03685A1C026010B41970036804
:10C3C8000A0A5C1C04601A7003680A0C5C1C04608E
:10C3D8001A700368090E5A1C026019705DF8044B44
:10C3E800704700BF03685A1C026019700368090A85
:10C3F8005A1C0260197070472DE9F047002488B074
:10C4080080460F461E46A14605AD531C039311787E
:10C4180039B3252933D1931CCDF810900393507864
:10C4280030284ED04FF0000AA0F13003DBB2092BC0
:10C4380042D96C2819D0642800F0938024D8252884
:10C448001CD063D9582876D063281BD13178404650
:10C45800B847039A531C0393117804360134002912
:10C46800D7D1204608B0BDE8F087039B5A1C039239
:10C478001B78642B7CD02AD8252B54D12521404603
:10C488000134B847039AC0E7732833D044D97528D4
:10C498004FD106F1040E30682B4600220A21764659
:10C4A800FFF7FEF8049A0095534639464046FFF7D1
:10C4B80035F9039A0444A8E704AA03A914F044FB35
:10C4C800B7E7D31C039390784FF0010AACE7732BBE
:10C4D80010D05BD9752B3AD0782B96D1A3F158029E
:10C4E800B2FA82F2306852092B4610210436FFF75F
:10C4F800D7F8D7E73368049A0093394600234046B3
:10C50800FFF70CF904360444039A7EE70028B9D1F2
:10C51800204608B0BDE8F0876E28B3D1039A336887
:10C5280004361C6071E72AD9582BD7D0632B8DD0DD
:10C538006BE77828A6D1A0F15802B2FA82F23068E7
:10C5480052092B461021FFF7ABF80436AAE706F18B
:10C55800040E30682B4600220A217646FFF7A0F821
:10C56800A0E7331D306829461E46FFF76BF899E7A8
:10C57800331D306829461E46FFF764F892E7002B02
:10C588007FF443AF204608B0BDE8F0876E2BC6D0D5
:10C598003BE700BF0EB400B584B005AB019053F87B
:10C5A800042B0649039301A8FFF726FF019B0022ED
:10C5B8001A7004B05DF804EB03B0704719B70008AF
:10C5C8000FB430B583B006AB0A490B4853F8042BB7
:10C5D800096800680193FFF70FFF084C05462068BB
:10C5E80000F0AAFF0028FAD0284603B0BDE8304082
:10C5F80004B07047582B00205C2B002030560020D8
:10C60800DFED2B7AB4EEE70AF1EE10FA4ADDDFED42
:10C61800296A9FED297A01E0B0EE670AB4EEC70AED
:10C62800F1EE10FA70EE667AF6DC9FED247AF4EEFD
:10C63800C77AF1EE10FA38D5DFED1E6A9FED207A41
:10C6480001E0F0EE407AF4EEC77AF1EE10FA37EE38
:10C65800A60AF6D4DFED1B7AB4EEE70AF1EE10FA7B
:10C6680014DDDFED137A37EEC00A60EE006A9FED45
:10C67800166A9FED167ADFED167AA6EE867A20EE18
:10C68800266AE6EE877AA6EE270A7047DFED117A6A
:10C69800B4EEE70AF1EE10FA44BFDFED087A37EEA0
:10C6A800C00AE2E7F0EE407ABFE7B0EE670AD1E7EA
:10C6B800DB0F4940DB0FC940E4CB1641DB0F49C013
:10C6C800E4CB16C1DB0FC93F92E741B99730083C6C
:10C6D80015A82ABEDB0FC9BF09B909E0194690FBA6
:10C6E800F1F301FB13030846002BF7D10846704706
:10C6F8000146FBE710B507EE901A2DED028BB8EE58
:10C70800678ADFED217A28EE008A044628EE278A18
:10C71800B0EE480A1DF05CFDF0EE408AB0EE480A23
:10C728001DF0B8FCF7EE007A9FED187AF0EE675A24
:10C73800E8EE875A0023A361B0EE676AC7EEA56AE0
:10C7480063612362E361A8EEC76ABDEC028B77EEF2
:10C75800C07AB6EE007AF8EE005A27EE877A20EE15
:10C76800250A27EE267A26EE266A67EEA67A20EEB6
:10C77800260A84ED046AC4ED017A84ED007A84ED1A
:10C78800027A84ED030A10BD27D4D236F304353F6C
:10C7980010B44C09012250F8243001F01F0102FAAC
:10C7A80001F10B4340F824305DF8044B704700BF9B
:10C7B8004B0901F01F0150F82320012303FA01F16E
:10C7C800114214BF18460020704700BF203970B5C9
:10C7D80001EB81010B4C4E1D264405460C4414F810
:10C7E800013B697995F904004022FFF785F9B442C5
:10C7F800F5D1697995F9040000234022BDE870401D
:10C80800FFF77AB958C8020838B50C46097839B123
:10C8180005462846FFF7DAFF14F8011F0029F8D16A
:10C8280038BD00BF30B583B0A1F1500510230024F6
:10C83800032201A98DF804508DF805408DF80630C3
:10C84800FFF76AF903B030BD30B501EB410421466A
:10C8580083B0C1F3C3036400A2F15005103304F0A0
:10C868000E04032201A98DF804508DF805408DF8B7
:10C878000630FFF751F903B030BD00BF38B50422C8
:10C8880008490546FFF748F94FF48064013C002346
:10C898004022697995F90400A4B2FFF72DF9002C1C
:10C8A800F4D138BDFCCA020838B580224179044663
:10C8B800AE2390F90400FFF71FF9054688B1162248
:10C8C80009492046FFF728F9042208492046FFF7BE
:10C8D80023F92046FFF7D2FF204603220449FFF739
:10C8E8001BF9284638BD00BF00CB020818CB020848
:10C8F8001CCB0208F0B55B4B5B4A97B019689142B4
:10C9080000AF00F0A3805949594A00234FF4700042
:10C91800C1F888003B607B60136843F48033136080
:10C9280003E03B68B3F5A04F09D0136803F4003364
:10C938007B603B6801333B607B68002BF1D04C4B3C
:10C948001B6813F4003318BF01237B607B68012B3D
:10C9580052D0464C464B474AE260474A596A1160F2
:10C968005A6A42F080725A625A6942F4FC025A6169
:10C978000025032207F10801012341F6FF764FF055
:10C988009040FD60BE603A73BB731AF05FFE4FF6CD
:10C99800FF7307F108013948BB601AF057FE07F129
:10C9A80008013748374E1AF051FE07F1080136489A
:10C9B8001AF04CFE07F1080134481AF047FE07F157
:10C9C800080133481AF042FE07F108001AF050FC3B
:10C9D800BB683049304AA1FB031330499B0CF02057
:10C9E8004FF0070E5C370B60566084F823009560A3
:10C9F800C2F800E0BD46F0BD294A1D4B1221116066
:10CA08005A685A605A685A605A6842F480625A6092
:10CA18005A6822F47C125A605A6842F4E8125A6042
:10CA28001A6842F080721A601A689201FCD5596837
:10CA38000F4A21F003015960596841F00201596019
:10CA4800536803F00C03082BFAD182E700221A601E
:10CA580062B6144B1B6883F30888134B1B6898470E
:10CA6800FEE700BFFC9F0020EFBEADDE00ED00E05A
:10CA7800001002400005FA055C530020000400483D
:10CA8800000800483F190100000C00480010004849
:10CA98000014004883DE1B4310E000E070570020BC
:10CAA8000020024000D8FF1F04D8FF1F2DE9F04FD7
:10CAB800714C54F8205083B0002D00F09A80D5F8BE
:10CAC80054901F46D9F80430EB64A9604FF4807382
:10CAD80005F15A019046064605F5AD72674828608B
:10CAE8006961AA61EB602B6199F8180018F06CF97C
:10CAF800D9F80C40F4B16248002103465A689442C0
:10CB080003F11C0303D001310C29F7D10021C1EB3B
:10CB1800C10100EB81015B480B6942694FF00C0EC3
:10CB28001A43731C426181F818E04B76EB6C2C6356
:10CB38002433AB64D9F80810002936D050480024B3
:10CB480003465A68914203F11C0303D001340C2CAC
:10CB5800F7D10024C4EBC40400EB8401494B0A69F3
:10CB68005869494C104358610B200876701C487668
:10CB78005869024399F81B005A618309002291F809
:10CB88000DE08DF805304D6101238C6001A88DF80A
:10CB980006208DF807308DF804E012F005FEEB6CE6
:10CBA800D9F808206A6328336B6495F8590001F0B6
:10CBB80067F8044695F8580001F062F83A0782468B
:10CBC80099F819B019D5C4B117F0110F4FF00B032C
:10CBD80006F1010614BF4E213E21A371E6715A46A3
:10CBE800204601F011F9FB0741D52B6B4BB36B6B5A
:10CBF8003BB3284603B0BDE8F08F17F0010F0CBF18
:10CC08002E274E2718F0020F09D044B10B22731CAF
:10CC1800A271E37120465A46394601F0F5F818F03A
:10CC2800010FE2D0BAF1000FDFD001360C238AF8E9
:10CC380007605A4639468AF80630504601F0E4F84B
:10CC4800D3E799F81A308DF8043099F81C30002190
:10CC58009B09012201A88DF805308DF806108DF882
:10CC6800072012F0A1FD284603B0BDE8F08F20464A
:10CC780001F058FCB9E700BF642B002020CB020864
:10CC8800F81200200010024049BD00080348D0F8FF
:10CC98003C3113B100F59A7018477047F81200201C
:10CCA8000348D0F8203113B100F58C70184770474D
:10CCB800F81200200348D0F804310BB1FC301847B3
:10CCC800704700BFF81200200348D0F8E8300BB1D5
:10CCD800E0301847704700BFF81200200348D0F82A
:10CCE800CC300BB1C4301847704700BFF812002091
:10CCF8000348D0F8B0300BB1A8301847704700BFD0
:10CD0800F81200200348D0F894300BB18C30184743
:10CD1800704700BFF81200200248836F0BB17030D3
:10CD280018477047F81200200248C36D0BB1543001
:10CD380018477047F81200200248036C0BB13830CE
:10CD480018477047F81200200248436A0BB11C309C
:10CD580018477047F81200200248836803B1184743
:10CD6800704700BFF81200201749184B184A194895
:10CD780010B4D1F8884044F47004C1F888401C68A5
:10CD880044F001041C605C6822405A601A6822F072
:10CD9800847222F480321A601A6822F480221A609F
:10CDA8005A6822F4FE025A60DA6A22F00F02DA6246
:10CDB8001A6B002410404FF0006218639C608A6070
:10CDC8005DF8044B704700BF00ED00E00010024022
:10CDD8000CC07FF8CCFC00FF436A8269D154436AD7
:10CDE8000169426B01338B4228BF00234362002A4A
:10CDF8002FD0EFF31181502383F31288436B1A6805
:10CE0800D2072CD470B45E686EB9456A826A9542BE
:10CE180017D084691444DC600ED9AA1A5A60856256
:10CE2800002280F850201A6842F00102C9B21A6044
:10CE380081F3118870BC70470469A21A5A6086622F
:10CE4800EEE7012380F85030C9B281F3118870BC35
:10CE58007047C26C136843F0800313607047C9B20F
:10CE680081F31188704700BF026B10B462B1036C84
:10CE7800C2684469D11A013B615C5DF8044B08BF84
:10CE880013460364C8B27047016A4369C4685B5CAF
:10CE98000131A14228BF114601625DF8044BD8B2A6
:10CEA800704700BF436B13B190F850007047836A16
:10CEB800406A181AB0FA80F040097047416A836ADC
:10CEC80099420AD3CB1A416B026961B14968501E75
:10CED8000B4483420AD2C01A704702691144CB1A24
:10CEE800416B0029F2D1501EC01A704700207047CC
:10CEF800036B43B1026C5B6893422FBF981AC068FA
:10CF08009B1AC0187047C269036A9A422FBFD01A89
:10CF1800C0688018C01A70470A4B30B503F1140472
:10CF280093F900205D78072AC8BF143A81180433A2
:10CF38000D7313F8025C855413F8012C0A76A3428A
:10CF4800EED130BD48CB020803682DE9F041DF6916
:10CF58001FB13B46BDE8F0411847002A164611DDCF
:10CF680004460D460E4400E023689B682046984717
:10CF78000028F9D0236815F8011B1B68204698473C
:10CF8800AE42F1D1BDE8F081002321220270437046
:10CF98008370C370704700BF30B50446C06C6171C0
:10CFA8000368A26823F00103036087B0A3790092A5
:10CFB80013F004023DD04FF4805213F002030192A3
:10CFC80044D102934FF480630022039311F00103CC
:10CFD800059237D1049308238D07694648BF049307
:10CFE80012F086FB6079E36CA17900F00202002A56
:10CFF80015BF4FF440324FF480324FF40034002410
:10D0080010F0010F586808BF2246CC074CBF0243F6
:10D0180020EA02025A609A6809074CBF42F00802E7
:10D0280022F008029A601A6842F001021A6007B0FA
:10D0380030BD13F0020301920BD04FF40055134694
:10D048000295C1E7042304930C23C5E74FF400536A
:10D05800B7E70293B8E700BF10B50446C06CA160FB
:10D06800036823F001030360A37986B013F0040278
:10D07800009141D04FF4805213F00203019244D141
:10D0880002934FF4806362790393D1074FF0000352
:10D098000493059345BF0423049308230C2369468E
:10D0A800920748BF049312F023FB6079E36CA179DF
:10D0B80000F00202002A15BF4FF440324FF48032CC
:10D0C8004FF40034002410F0010F586808BF2246BE
:10D0D800CC074CBF024320EA02025A609A6809074B
:10D0E8004CBF42F0080222F008029A601A6842F027
:10D0F80001021A6006B010BD13F00203019207D0B6
:10D108004FF4005113460291BDE74FF40053B7E7BF
:10D118000293B8E72DE9F04FDFF830C1474A484994
:10D12800484E494D8046102718F1FF38C0F08480DA
:10D13800DCF80430C3F30803002B5CD1EFF3118350
:10D14800002B58D10B68946800BF08688342F9D156
:10D15800D6F800904FF47A7000FB09FEAEEB040E8F
:10D16800BEFBF9FE00FB03EEDCF80430C3F3080352
:10D178004FF47A740120FBB9EFF31183E3B90B681C
:10D18800D2F808A000BFD1F800904B45F7D1D6F8E7
:10D1980000B004FB0BF9A9EB0A09B9FBFBF904FB86
:10D1A8000393A3EB0E03B3F57A7FBDD2DCF804300A
:10D1B800C3F30803002BDFD0EFF3118A87F312883B
:10D1C800D2F808B01368DB0344BF2860D2F808B06F
:10D1D8000B68D5F800905FFA8AFA8AF31188D6F8B6
:10D1E80000A0994404FB0AF3A3EB0B03B3FBFAF387
:10D1F80004FB0933D5E7EFF3118487F31288D2F8DB
:10D2080008901368D80303D501232B60D2F808903F
:10D218000B682868E4B284F31188D6F800A04FF4AC
:10D228007A7400EB030E04FB0AF3A3EB0903B3FBC8
:10D23800FAF304FB0E3E97E7BDE8F08F10E000E03C
:10D248006C570020705700206857002000ED00E060
:10D25800204B5B68C3F3080330B4BBB9EFF3118309
:10D26800A3B91D4B1D4C1868A16800BF1A689042ED
:10D27800F9D11B4B1C684FF47A7202FB04F3591A5C
:10D28800B1FBF4F130BC02FB00107047EFF31182E0
:10D29800102383F3128811498C680B6813F4803FBC
:10D2A800104B02D0012018608C680B49D2B20D686F
:10D2B800186882F311880A4B19684FF47A72284467
:10D2C80002FB01F31B1B30BCB3FBF1F302FB003084
:10D2D800704700BF00ED00E06C57002010E000E050
:10D2E800705700206857002030B4EFF311831022E4
:10D2F80082F312880649074C0A680748013200255C
:10D308000A602560DBB2026883F3118830BC70477D
:10D318006C5700206857002010E000E01D4B70B5E6
:10D328009C68E36C226BDD69C2B1636B2BB12B0780
:10D3380002D5E36C08221A6270BD2A06F7D5A26AE4
:10D34800616A8A421FD0511CA069A162825C20696F
:10D35800E66C81423285EAD3A362E8E7A906E4D500
:10D36800E26A1AB1988C80B29047DEE7E1699B8C3B
:10D378006069DBB24E1CE6614354E169E368994297
:10D3880028BFE261D1E7E26C136823F080031360E1
:10D39800CDE700BF642B00201D4B70B55C68E36CC3
:10D3A800226BDD69C2B1636B2BB12B0702D5E36C2D
:10D3B80008221A6270BD2A06F7D5A26A616A8A42F3
:10D3C8001FD0511CA069A162825C2069E66C814271
:10D3D8003285EAD3A362E8E7A906E4D5E26A1AB17E
:10D3E800988C80B29047DEE7E1699B8C6069DBB27C
:10D3F8004E1CE6614354E169E368994228BFE26143
:10D40800D1E7E26C136823F080031360CDE700BF17
:10D41800642B00201D4B70B51C68E36C226BDD6922
:10D42800C2B1636B2BB12B0702D5E36C08221A62D9
:10D4380070BD2A06F7D5A26A616A8A421FD0511CBC
:10D44800A069A162825C2069E66C81423285EAD3D8
:10D45800A362E8E7A906E4D5E26A1AB1988C80B21B
:10D468009047DEE7E1699B8C6069DBB24E1CE661A0
:10D478004354E169E368994228BFE261D1E7E26C6D
:10D48800136823F080031360CDE700BF642B0020EE
:10D4980070B4EFF31186502383F31288436B1A6834
:10D4A800D20720D45D686DB9446A826A944217D065
:10D4B80081691144D9600ED9A21A5A608462002287
:10D4C80080F850201A6842F00102F1B21A6081F324
:10D4D800118870BC704701698A1A5A608562EEE744
:10D4E800012380F85030F1B281F3118870BC704785
:10D4F80003682DE9F041DF691FB13B46BDE8F04103
:10D508001847002A164611DD04460D460E4400E071
:10D5180023689B68204698470028F9D0236815F8A7
:10D52800011B1B6820469847AE42F1D1BDE8F08147
:10D5380003689B69184700BF03685B69184700BF09
:10D548000368DB68184700BF03685B68184700BFBB
:10D5580003681B68184700BF054B53F8203033B1E8
:10D568001A689B88918A0B4218BF1B049361704705
:10D578003857002003682DE9F04F03F13845644E11
:10D58800AD0A0124755D05F01F066D09022D04FA28
:10D5980006F400F0A280032D00F0A480012D52D0E3
:10D5A8008088B0FA80F4C4F11F04A4B2E50803EB44
:10D5B800850504F007042E6AA4000F27A74026EA71
:10D5C80007062E622E6A01F0030702FA04F47A1E97
:10D5D8003443012AC1F3810CC1F300182C62C1F352
:10D5E800411135D9C60700F19780850700F1A3805E
:10D5F800440700F1B180020700F1BF80C60600F1C0
:10D60800CD80850600F1DB80440600F1E980020642
:10D6180000F1F780C60500F10581850500F1138149
:10D62800440500F12181020500F12F81C60400F1B3
:10D638003D81850400F14B81440400F159810204C5
:10D6480055D4BDE8F08F334D6E6934436C61A7E75C
:10D65800002422464FF0010E4FF0030904E0013286
:10D66800102A04F10204ECD00EFA02F636EA00059C
:10D67800F5D1D3F808A009FA04F5ED430AEA050A3A
:10D68800C3F808A0D3F808B00CFA04FA4AEA0B0A5F
:10D69800C3F808A0B3F804A01FFA8AFA2AEA060613
:10D6A8009E80B3F804A008FA02F646EA0A06B6B263
:10D6B8009E801E682E401E60D3F800A007FA04F66C
:10D6C80046EA0A061E60D3F80CA001FA04F605EA39
:10D6D8000A0A46EA0A05DD60C1E70E4DAE69344321
:10D6E800AC615DE70B4DEE693443EC6158E71A68AD
:10D6F80022F040421A601A6842EA87771F60DA68A7
:10D7080022F0404242EA8171D960BDE8F08F00BF43
:10D718006CE20208001002401A6822F003021A6044
:10D728001A683A431A60DA6822F003020A43850746
:10D73800DA607FF55DAF1A6822F00C021A601A6889
:10D7480042EA87021A60DA6822F00C0242EA810291
:10D758004407DA607FF54FAF1A6822F030021A608A
:10D768001A6842EA07121A60DA6822F0300242EABE
:10D778000112DA6002077FF541AF1A6822F0C00291
:10D788001A601A6842EA87121A60DA6822F0C00240
:10D7980042EA8112C606DA607FF533AF1A6822F4CE
:10D7A80040721A601A6842EA07221A60DA6822F49C
:10D7B800407242EA01228506DA607FF525AF1A68D1
:10D7C80022F440621A601A6842EA87221A60DA680C
:10D7D80022F4406242EA81224406DA607FF517AFFC
:10D7E8001A6822F440521A601A6842EA07321A602C
:10D7F800DA6822F4405242EA0132DA6002067FF522
:10D8080009AF1A6822F440421A601A6842EA87325D
:10D818001A60DA6822F4404242EA8132C605DA60C8
:10D828007FF5FBAE1A6822F440321A601A6842EAA1
:10D8380007421A60DA6822F4403242EA014285055A
:10D84800DA607FF5EDAE1A6822F440221A601A6891
:10D8580042EA87421A60DA6822F4402242EA8142A8
:10D868004405DA607FF5DFAE1A6822F440121A60C8
:10D878001A6842EA07521A60DA6822F4401242EA49
:10D888000152DA6002057FF5D1AE1A6822F440022F
:10D898001A601A6842EA87521A60DA6822F440026B
:10D8A80042EA8152C604DA607FF5C3AE1A6822F0F4
:10D8B80040721A601A6842EA07621A60DA6822F04F
:10D8C800407242EA01628504DA607FF5B5AE1A68F3
:10D8D80022F040621A601A6842EA87621A60DA68BF
:10D8E80022F0406242EA81624404DA607FF5A7AE22
:10D8F8001A6822F040521A601A6842EA07721A60DF
:10D90800DA6822F0405242EA0172DA6097E600BF14
:10D91800036803F138422DE9F04F920A584DAA5C8A
:10D9280002F01F0552090124022A04FA05F400F046
:10D938008C80032A00F08E80012A3CD001F0030776
:10D948007A1E012AC1F3810CC1F300188088C1F343
:10D95800411135D9C60700F19780850700F1A380EA
:10D96800440700F1B180020700F1BF80C60600F14C
:10D97800CD80850600F1DB80440600F1E9800206CF
:10D9880000F1F780C60500F10581850500F11381D6
:10D99800440500F12181020500F12F81C60400F140
:10D9A8003D81850400F14B81440400F15981020452
:10D9B80055D4BDE8F08F334A55692C435461BDE70F
:10D9C800002422464FF0010E4FF0030904E0013213
:10D9D800102A04F10204ECD00EFA02F636EA000529
:10D9E800F5D1D3F808A009FA04F5ED430AEA050AC7
:10D9F800C3F808A0D3F808B00CFA04FA4AEA0B0AEC
:10DA0800C3F808A0B3F804A01FFA8AFA2AEA06069F
:10DA18009E80B3F804A008FA02F646EA0A06B6B2EF
:10DA28009E801E682E401E60D3F800A007FA04F6F8
:10DA380046EA0A061E60D3F80CA001FA04F605EAC5
:10DA48000A0A46EA0A05DD60C1E70E4A95692C43D1
:10DA5800946173E70B4AD5692C43D4616EE71A6861
:10DA680022F040421A601A6842EA87771F60DA6833
:10DA780022F0404242EA8171D960BDE8F08F00BFD0
:10DA88006CE20208001002401A6822F003021A60D1
:10DA98001A683A431A60DA6822F003020A438507D3
:10DAA800DA607FF55DAF1A6822F00C021A601A6816
:10DAB80042EA87021A60DA6822F00C0242EA81021E
:10DAC8004407DA607FF54FAF1A6822F030021A6017
:10DAD8001A6842EA07121A60DA6822F0300242EA4B
:10DAE8000112DA6002077FF541AF1A6822F0C0021E
:10DAF8001A601A6842EA87121A60DA6822F0C002CD
:10DB080042EA8112C606DA607FF533AF1A6822F45A
:10DB180040721A601A6842EA07221A60DA6822F428
:10DB2800407242EA01228506DA607FF525AF1A685D
:10DB380022F440621A601A6842EA87221A60DA6898
:10DB480022F4406242EA81224406DA607FF517AF88
:10DB58001A6822F440521A601A6842EA07321A60B8
:10DB6800DA6822F4405242EA0132DA6002067FF5AE
:10DB780009AF1A6822F440421A601A6842EA8732EA
:10DB88001A60DA6822F4404242EA8132C605DA6055
:10DB98007FF5FBAE1A6822F440321A601A6842EA2E
:10DBA80007421A60DA6822F4403242EA01428505E7
:10DBB800DA607FF5EDAE1A6822F440221A601A681E
:10DBC80042EA87421A60DA6822F4402242EA814235
:10DBD8004405DA607FF5DFAE1A6822F440121A6055
:10DBE8001A6842EA07521A60DA6822F4401242EAD6
:10DBF8000152DA6002057FF5D1AE1A6822F44002BC
:10DC08001A601A6842EA87521A60DA6822F44002F7
:10DC180042EA8152C604DA607FF5C3AE1A6822F080
:10DC280040721A601A6842EA07621A60DA6822F0DB
:10DC3800407242EA01628504DA607FF5B5AE1A687F
:10DC480022F040621A601A6842EA87621A60DA684B
:10DC580022F0406242EA81624404DA607FF5A7AEAE
:10DC68001A6822F040521A601A6842EA07721A606B
:10DC7800DA6822F0405242EA0172DA6097E600BFA1
:10DC880010B50409013C052C17D80D4B33F81420A6
:10DC980000F00F0042FA00F313F001030DD0012346
:10DCA80003FA00F0013810401BF0B4FF054A064B98
:10DCB800125D104403EBC00010BD002010BD00BF72
:10DCC80058E2020864E20208F84800202DE9F04F03
:10DCD8004A484B4B4B4C4FF090414FF0010A4FF0E4
:10DCE80002094FF004084FF0080C4FF0100E2027DF
:10DCF8004026802530F8022B12F0010F03D019605E
:10DD0800A3F804A0083312F0020F03D01960A3F897
:10DD18000490083312F0040F03D01960A3F80480AC
:10DD2800083312F0080F03D01960A3F804C00833B1
:10DD380012F0100F03D01960A3F804E0083312F0B2
:10DD4800200F02D019609F80083312F0400F02D0D4
:10DD580019609E80083312F0800F02D019609D80F0
:10DD6800083312F4807F05D04FF4807B1960A3F844
:10DD780004B0083312F4007F05D04FF4007B19601B
:10DD8800A3F804B0083312F4806F05D04FF4806B09
:10DD98001960A3F804B0083312F4006F05D04FF4EB
:10DDA800006B1960A3F804B0083312F4805F05D043
:10DDB8004FF4805B1960A3F804B0083312F4005FD5
:10DDC80005D04FF4005B1960A3F804B0083312F4CF
:10DDD800804F05D04FF4804B1960A3F804B0083386
:10DDE800D20B04D04FF4004219609A80083301F531
:10DDF8008061A1427FF47EAFBDE8F08F58E202084F
:10DE0800F848002000180048002867D003682DE96A
:10DE1800F04F03F138445C4EA40A0125345D04F048
:10DE28001F066409022C05FA06F558D0032C00F0E9
:10DE3800A580012C58D08088B0FA80F4C4F11F0462
:10DE4800A4B2E50803EB850504F007042E6AA400D4
:10DE58000F27A74026EA07062E622E6A01F003075D
:10DE6800A2407C1E3243012CC1F3810CC1F300187F
:10DE78002A62C1F341113CD9C60700F189808507A0
:10DE880000F19580440700F1A380020700F1B180FA
:10DE9800C60600F1BF80850600F1CD80440600F17A
:10DEA800DB80020600F1E980C60500F1F7808505F0
:10DEB80000F10581440500F11381020500F121817B
:10DEC800C60400F12F81850400F13D81440400F16E
:10DED8004B81020400F15981BDE8F08F70472B4C4B
:10DEE800A6693543A561A6E7284C6669354365618F
:10DEF800A1E7002422464FF0010E4FF0030904E089
:10DF08000132102A04F10204E6D00EFA02F636EACB
:10DF18000005F5D1D3F808A009FA04F5ED430AEA9B
:10DF2800050AC3F808A0D3F808B00CFA04FA4AEABC
:10DF38000B0AC3F808A0B3F804A01FFA8AFA2AEA61
:10DF480006069E80B3F804A008FA02F646EA0A0616
:10DF5800B6B29E801E682E401E60D3F800A007FA55
:10DF680004F646EA0A061E60D3F80CA001FA04F685
:10DF780005EA0A0A46EA0A05DD60C1E7034CE669D4
:10DF88003543E56157E700BF6CE202080010024024
:10DF98001A6822F003021A601A683A431A60DA68AB
:10DFA80022F003020A438507DA607FF56BAF1A682F
:10DFB80022F00C021A601A6842EA87021A60DA68CC
:10DFC80022F00C0242EA81024407DA607FF55DAF75
:10DFD8001A6822F030021A601A6842EA07121A60B8
:10DFE800DA6822F0300242EA0112DA6002077FF5AD
:10DFF8004FAF1A6822F0C0021A601A6842EA871204
:10E008001A60DA6822F0C00242EA8112C606DA60B3
:10E018007FF541AF1A6822F440721A601A6842EA22
:10E0280007221A60DA6822F4407242EA0122850661
:10E03800DA607FF533AF1A6822F440621A601A6812
:10E0480042EA87221A60DA6822F4406242EA8122B0
:10E058004406DA607FF525AF1A6822F440521A6048
:10E068001A6842EA07321A60DA6822F4405242EA31
:10E078000132DA6002067FF517AF1A6822F44042CF
:10E088001A601A6842EA87321A60DA6822F4404253
:10E0980042EA8132C605DA607FF509AF1A6822F4D0
:10E0A80040321A601A6842EA07421A60DA6822F4B3
:10E0B800403242EA01428505DA607FF5FBAE1A6814
:10E0C80022F440221A601A6842EA87421A60DA6823
:10E0D80022F4402242EA81424405DA607FF5EDAE3F
:10E0E8001A6822F440121A601A6842EA07521A6043
:10E0F800DA6822F4401242EA0152DA6002057FF53A
:10E10800DFAE1A6822F440021A601A6842EA87529F
:10E118001A60DA6822F4400242EA8152C604DA60E0
:10E128007FF5D1AE1A6822F040721A601A6842EA86
:10E1380007621A60DA6822F0407242EA01628504D6
:10E14800DA607FF5C3AE1A6822F040621A601A6876
:10E1580042EA87621A60DA6822F0406242EA816223
:10E168004404DA607FF5B5AE1A6822F040521A60AE
:10E178001A6842EA07721A60DA6822F0405242EAE4
:10E188000172DA6002047FF5A7AE1A6822F04042F5
:10E198001A601A6842EA87771F60DA6822F04042FC
:10E1A80042EA8171D960BDE8F08F00BF002852D0E3
:10E1B800036803F138422DE9F04F920A504DAA5CEA
:10E1C80002F01F0552090124022A04FA05F443D07B
:10E1D800032A00F09080012A43D001F003077A1E39
:10E1E800012AC1F3810CC1F300188088C1F34111E1
:10E1F8003CD9C60700F18880850700F19480440760
:10E2080000F1A280020700F1B080C60600F1BE80CE
:10E21800850600F1CC80440600F1DA80020600F1A0
:10E22800E880C60500F1F680850500F10481440503
:10E2380000F11281020500F12081C60400F12E814F
:10E24800850400F13C81440400F14A81020400F194
:10E258005881BDE8F08F70472A4A95692C4394612C
:10E26800BBE7284A55692C435461B6E70024224687
:10E278004FF0010E4FF0030904E00132102A04F1B7
:10E288000204E6D00EFA02F636EA0005F5D1D3F814
:10E2980008A009FA04F5ED430AEA050AC3F808A03C
:10E2A800D3F808B00CFA04FA4AEA0B0AC3F808A033
:10E2B800B3F804A01FFA8AFA2AEA06069E80B3F881
:10E2C80004A008FA02F646EA0A06B6B29E801E685C
:10E2D8002E401E60D3F800A007FA04F646EA0A06A4
:10E2E8001E60D3F80CA001FA04F605EA0A0A46EA09
:10E2F8000A05DD60C1E7034AD5692C43D4616CE7A0
:10E308006CE20208001002401A6822F003021A6048
:10E318001A683A431A60DA6822F003020A4385074A
:10E32800DA607FF56CAF1A6822F00C021A601A687E
:10E3380042EA87021A60DA6822F00C0242EA810295
:10E348004407DA607FF55EAF1A6822F030021A607F
:10E358001A6842EA07121A60DA6822F0300242EAC2
:10E368000112DA6002077FF550AF1A6822F0C00286
:10E378001A601A6842EA87121A60DA6822F0C00244
:10E3880042EA8112C606DA607FF542AF1A6822F4C3
:10E3980040721A601A6842EA07221A60DA6822F4A0
:10E3A800407242EA01228506DA607FF534AF1A68C6
:10E3B80022F440621A601A6842EA87221A60DA6810
:10E3C80022F4406242EA81224406DA607FF526AFF1
:10E3D8001A6822F440521A601A6842EA07321A6030
:10E3E800DA6822F4405242EA0132DA6002067FF526
:10E3F80018AF1A6822F440421A601A6842EA873253
:10E408001A60DA6822F4404242EA8132C605DA60CC
:10E418007FF50AAF1A6822F440321A601A6842EA95
:10E4280007421A60DA6822F4403242EA014285055E
:10E43800DA607FF5FCAE1A6822F440221A601A6886
:10E4480042EA87421A60DA6822F4402242EA8142AC
:10E458004405DA607FF5EEAE1A6822F440121A60BD
:10E468001A6842EA07521A60DA6822F4401242EA4D
:10E478000152DA6002057FF5E0AE1A6822F4400224
:10E488001A601A6842EA87521A60DA6822F440026F
:10E4980042EA8152C604DA607FF5D2AE1A6822F0E9
:10E4A80040721A601A6842EA07621A60DA6822F053
:10E4B800407242EA01628504DA607FF5C4AE1A68E8
:10E4C80022F040621A601A6842EA87621A60DA68C3
:10E4D80022F0406242EA81624404DA607FF5B6AE17
:10E4E8001A6822F040521A601A6842EA07721A60E3
:10E4F800DA6822F0405242EA0172DA6002047FF5DB
:10E50800A8AE1A6822F040421A601A6842EA877771
:10E518001F60DA6822F0404242EA8171D960BDE8A2
:10E52800F08F00BF10B1036882881A85704700BF5A
:10E5380010B1036882889A61704700BF38B100291A
:10E548008388026814BF002110218B4093617047B3
:10E558000E4B1B8801463BB90D4B0E4A1B781068C1
:10E568000BB981F00101E9E70B4B5A691AB118B9E7
:10E578001A68106058747047084A18681188084A61
:10E5880092FBF1F201210260597470474457002050
:10E5980046570020485700204C5700206457002059
:10E5A80020A1070010B40A4B0A4A1C7801238340B3
:10E5B800234052F8200029B9B3FA83F149095DF8DC
:10E5C800044BBBE7191C18BF01215DF8044BB5E7E4
:10E5D80036570020385700202DE9F0410B4E34689B
:10E5E80073691C400FD0DFF828800127B4FA84F340
:10E5F800C3F11F0307FA03F558F823000368984787
:10E60800AC437561F2D1BDE8F08100BF0004014060
:10E618007C5700202DE9F0410B4E346873691C408B
:10E628000FD0DFF828800127B4FA84F3C3F11F0361
:10E6380007FA03F558F8230003689847AC43756157
:10E64800F2D1BDE8F08100BF000401407C570020F2
:10E658002DE9F0410B4E346873691C400FD0DFF888
:10E6680028800127B4FA84F3C3F11F0307FA03F5DE
:10E6780058F8230003689847AC437561F2D1BDE8A8
:10E68800F08100BF000401407C5700202DE9F041D3
:10E698000B4E346873691C400FD0DFF828800127BF
:10E6A800B4FA84F3C3F11F0307FA03F558F82300FB
:10E6B80003689847AC437561F2D1BDE8F08100BFAB
:10E6C800000401407C5700202DE9F0410B4E3468CE
:10E6D80073691C400FD0DFF828800127B4FA84F34F
:10E6E800C3F11F0307FA03F558F823000368984796
:10E6F800AC437561F2D1BDE8F08100BF0004014070
:10E708007C5700202DE9F0410B4E346873691C409A
:10E718000FD0DFF828800127B4FA84F3C3F11F0370
:10E7280007FA03F558F8230003689847AC43756166
:10E73800F2D1BDE8F08100BF000401407C57002001
:10E748002DE9F0410B4E346873691C400FD0DFF897
:10E7580028800127B4FA84F3C3F11F0307FA03F5ED
:10E7680058F8230003689847AC437561F2D1BDE8B7
:10E77800F08100BF000401407C57002038B50B4CE5
:10E7880023688BB15A68821A002A054604DA0CE01D
:10E798005A68AA1A002A07DB9A68226018461A687B
:10E7A80090472368002BF3D138BD38BD403F002087
:10E7B8000B4B002210B4027203F1C804042102E0DA
:10E7C800072A09DC9979890702D519798154013218
:10E7D8009C4203F11403F3D15DF8044B704700BF6A
:10E7E800A8E5020810B40D4C04232146002200E0DD
:10E7F8008B7913F0010301F1140106D101320B2AC0
:10E80800F6D103705DF8044B704702EB820204EB0B
:10E8180082025DF8044B137903707047A8E502087B
:10E828000123102112224170427103700371704755
:10E8380008B506F06DF8024B024ADA60FEE700BF41
:10E8480000ED00E00400FA052DE9F0470569C3680A
:10E858001D4028D00F4606464FF000484FF00009EB
:10E86800B5FA85F328FA03F2D2431B3B326115400F
:10E87800042B16D8DFE803F03129211903007B6A3D
:10E88800002B32D003F1FF3A1FFA8AFAC7F8249016
:10E898003C6A34B123682046514698476468002C86
:10E8A800F8D1002DDCD1BDE8F0873868716B0368BA
:10E8B80089B29847002DD3D1F5E77868B16B036822
:10E8C80089B29847002DCBD1EDE7B868F16B0368A2
:10E8D80089B29847002DC3D1E5E7F868316C036821
:10E8E80089B29847002DBBD1DDE7F36A1FFA83FA96
:10E8F800CEE700BF08B501210220FFF753FE094B00
:10E908001B7803F00503052B08D000210120FFF731
:10E9180049FE00210846FFF745FEFEE706F08AF8A3
:10E92800F3E700BF602B0020022828BF022010B4A4
:10E93800084C094B207000EB8002C0EBC20207496B
:10E948005DF8044B013003EB4203C0B20B6009F0E1
:10E9580099B900BFDE590020D0670020EC5900208B
:10E9680008B507F017F9FDF7F3FABDE8084007F016
:10E97800F9B800BF38B5434B5A899989914224BFE9
:10E9880000225A81198ADA89914224BF0022DA8149
:10E99800DA788AB3072A2FD03B493C4D91F85700C3
:10E9A800012400210A282C709C70D9713DD00C28B4
:10E9B80065D0DFED377A8ABB364C9FED370AA278EF
:10E9C800002918BFF0EE407A062A04D8334901EB33
:10E9D800820191ED000A217959B3013A032A4DD8F1
:10E9E800F7EE007A87EE800A1BF0A6FB2388984290
:10E9F80028BF1846208038BDD97921B198780428D5
:10EA0800B8BF04209870204890F857000A280CD006
:10EA18000C28CED1DFED227A002ACDD0072ACBD020
:10EA28000A282CD1DFED1F7AC6E70A20DFED1E7A0F
:10EA3800C1E79B78154A07EE103A1178B8EEC77A05
:10EA480027EE277A07EE901AF8EEE77A67EE877ACC
:10EA5800B4EEE70AF1EE10FA10DDC0EE077AFDEE2B
:10EA6800E77A17EE903A102BA8BF1023012BB8BFF6
:10EA78000123DBB28B4238BF0B46137038BDDFED84
:10EA88000B7A99E7F04E0020044F0020303C00201C
:10EA98006F120339C04B00206F1203385CCB020899
:10EAA8000AD7A3390F506E3A5304E9386F12833AE4
:10EAB80038B50D4C0D4DAC4206D261682046143471
:10EAC800FDF7D2F9AC42F8D3094B0A490A4D0B4A73
:10EAD8001D600B480B4C04600023B4250B704B7071
:10EAE80015605360936038BDF81D030808220308B9
:10EAF800EC590020DE590020D06700208C4300200C
:10EB0800D02B0020F059002008B5FFF7D1FF07F0FF
:10EB180041F8FDF71DFABDE8084007F023B800BF2B
:10EB2800F0B50C292BD8DFE801F06F2A2A2A4C2AE5
:10EB38002A2A2B2A2A2A0700046AB2F80CE09788A6
:10EB48001668674D24F480540462036A4468C169F6
:10EB580023F4005343EA0E3321F4E641A84243EA82
:10EB6800073341EA062100F0B58005F50065A842A3
:10EB780000F0B08092684460C16102640362F0BD35
:10EB8800046A96899588D2F800E0554F24F4807479
:10EB98000462036A4468C16923F4007343EA0623E4
:10EBA80021F07301B84243EA052341EA0E017ED001
:10EBB8004C4DA8427BD092684460C161C263036235
:10EBC800F0BD046A96899588D2F800E0444F24F095
:10EBD80010040462036A4468816923F0200321F069
:10EBE800807143EA061321F4E641B84243EA05136B
:10EBF80041EA0E2148D03B4DA84245D09268446076
:10EC0800816182630362F0BD046A9389B2F804E00B
:10EC18001768334E24F001040462056A4468816968
:10EC280043EA0E0321F4803125F002059BB221F05E
:10EC38007301B04243EA050341EA070114D0294DA4
:10EC4800A84211D005F54065A8420DD005F58065AC
:10EC5800A84209D005F58065A84205D092684460AD
:10EC6800816142630362F0BDD689158A578A23F011
:10EC7800080333433D43D68824F4407423F0040347
:10EC8800ADB233432C43E9E7D589178AD68823F0F8
:10EC9800800343EA051324F44064558A23F04003B3
:10ECA80044EA870443EA061344EA8504A6E7D589BB
:10ECB800178AD68823F4006343EA052324F44054D2
:10ECC800558A23F4806344EA071443EA062344EA96
:10ECD800051470E7158A24F4804444EA851449E74A
:10ECE800002C0140003401402DE9F04F4FF4A07290
:10ECF800002183B07848794CDFF80492784D794E3A
:10ED0800794FDFF800821DF02FFB78487849DFF84B
:10ED1800F8E1DFF8F8C100221359834200F0C180FE
:10ED2800B3F1804F00F0C980AB4200F0C880B34215
:10ED380000F0C780BB4200F0C680734500F0C58074
:10ED4800634500F0C480434500F0C380DFF8C0A1EC
:10ED580053457ED00AF5806A534508BF092379D008
:10ED68001432DC2AD8D15D4C624D634E604F04F1F9
:10ED7800DC0802E01434A04568D0A379002BF9D050
:10ED880023794FEA131909F1FF39B9F1050F03F097
:10ED98000F03EFD835F8190040FA03F2D207E9D586
:10EDA8004FF0010A0AFA03F3013B18401AF032FF48
:10EDB80016F809305149184411EBC002DAD051F85D
:10EDC8003000DFF850E1217A00F138439B0A1EF841
:10EDD800033003F01F0E5B09022B0AFA0EFA62D009
:10EDE800032B65D0012B03D17B694AEA03037B61BE
:10EDF80093880093B3FA83F3C3F11F039BB2DA0835
:10EE080000EB820203F00703D2F820E09B004FF0EA
:10EE18000F0C0CFA03FC2EEA0C0EC2F820E0D2F814
:10EE280020E001FA03F343EA0E0313626946002364
:10EE3800022214348DF804208DF805308DF8063040
:10EE48008DF8073018F002FCA04596D103B0BDE854
:10EE5800F08F082309EBC3034FF0010B93F820A0B0
:10EE68000AF01F034FEA5A1ABAF1020F0BFA03F31A
:10EE78000BD0BAF1030F0ED0DA457FF471AFD1F899
:10EE880014A043EA0A034B616AE7D1F818A043EAE1
:10EE98000A038B6164E7D1F81CA043EA0A03CB613B
:10EEA8005EE70023D6E7BB694AEA0303BB619FE735
:10EEB800FB694AEA0303FB619AE70123CAE70223D5
:10EEC800C8E70323C6E70423C4E70523C2E70623EC
:10EED800C0E70723BEE700BFC4570020A8E5020823
:10EEE800000400400008004000100040002C0140D1
:10EEF8000010024058E2020864E20208F8480020C4
:10EF08005CCB02080040014000140040003401407E
:10EF1800004401406CE202080149024894E400BF41
:10EF2800DC58002000480140014902488CE400BF39
:10EF38008C580020004001400149024884E400BF89
:10EF48006458002000340140014902487CE400BFB5
:10EF580064580020003401400149024874E400BFAD
:10EF68003C58002000080040014902486CE400BFFA
:10EF7800145800200004004001494FF0804063E429
:10EF8800EC57002010B5054C05482146FFF75CFCFE
:10EF980004F1F0010348BDE8104055E4C4570020CF
:10EFA800002C014000440140014902484CE400BFE4
:10EFB800C4570020002C01402DE9F0410468574D4A
:10EFC800A30AAB4200F085805CD9554DAB426CD0AA
:10EFD80078D9544DAB4264D00135AB4240F09A80A9
:10EFE8004FF49C7E072647794FEA970C00297CD07E
:10EFF800B000634685190227D4F80C809F400CEBBB
:10F008004503BFB2484D03F1040C47EA080745F829
:10F01800231045F82C20E760EFF31181502282F38A
:10F028001288821905EBC2021369002B41D01362C2
:10F038000433821905EBC202576917B11F6053697F
:10F048000433821905EBC202976917B11F609369EF
:10F058000433821905EBC202D76917B11F60D3695F
:10F0680004330027CAB21F6082F31188304405EBCD
:10F07800C000036A03BBE3684FF6FE721340E36007
:10F08800BDE8F0814A3DAB422BD00135AB4204D0FC
:10F09800B3F5801F21D0BDE8F0814FF0980E03260C
:10F0A800A1E74FF4887E06269DE74FF0E80E052677
:10F0B80099E705EB0E03BCE7E36843F00103E3605F
:10F0C800BDE8F081033DAB4226D14FF0C00E0426C7
:10F0D80089E74FF0200E002685E74FF0480E0126FD
:10F0E80081E74FF0700E02267DE7BF08022306FA7B
:10F0F80003F0BB40DB43E7680B4D9BB23B408719ED
:10F108000CEB470CE3600CF1040345F82C1045F8B0
:10F11800232081E7BDE8F081BDE8F0814B001000B5
:10F128005000100051001000C457002030B503688B
:10F138005C4D18885C4CB4FBF2F20139013AAB42E1
:10F1480094B283B089B282B266D05848834263D001
:10F15800B3F1804F60D0A0F5983083425CD000F5C1
:10F168008060834258D0524883425BD000F580606B
:10F1780083427DD022F4407200F58C3092B28342F3
:10F188001A80D9621C850ED0484A93420BD002F5EA
:10F198004062934207D002F58062934203D002F5A1
:10F1A8008062934201D100221A8601225A611A888C
:10F1B8003C4992B242F001028B421A8062D0B3F10C
:10F1C800804F61D03B4A934260D002F580629342FF
:10F1D8005ED002F5006293425CD002F580629342F1
:10F1E8005AD002F59032934258D002F540629342C9
:10F1F80056D002F5806293421ED002F58062934297
:10F2080008BF092219D002A84FF0012340F8043D95
:10F2180010F0CAFA03B030BD254822F070028342CC
:10F2280092B2A3D101201A80D9621C8558611A882C
:10F2380092B202431A80C5E708221F4B03EBC203B0
:10F2480001A893F821408DF80440012300228DF88D
:10F2580005308DF807308DF8062010F0A5FA1B2C24
:10F26800D8D1164B019301A810F09EFA03B030BD17
:10F2780001201A80D9621C8558611A8892B202430B
:10F288001A809CE70022D8E70122D6E70222D4E7B9
:10F298000322D2E70422D0E70522CEE70622CCE7F4
:10F2A8000722CAE7002C014000A24A0400340140AA
:10F2B80000100040000400405CCB02081901000166
:10F2C800204B98422DD0B0F1804F2CD0A3F5943329
:10F2D80098422AD003F58063984228D003F500634A
:10F2E800984226D003F58063984224D003F59033E2
:10F2F800984222D003F54063984220D003F58063FA
:10F30800984207D003F58063984208BF092202D0CB
:10F318000020704708220C4B03EBC20393F820002F
:10F3280070470022F7E70122F5E70222F3E70322FC
:10F33800F1E70422EFE70522EDE70622EBE70722D3
:10F34800E9E700BF002C01405CCB02082DE9F04F33
:10F35800013085B0C3B203938E4D8F4F8F4C904EC2
:10F368000A230293DFF8409216F060F94FF4FA7A14
:10F378004FF0100C4FF47A70D9F80430C3F3080337
:10F38800002B40F0C880EFF31183002B40F0C380BE
:10F398002968A26800BF2B689942F9D1D7F800E024
:10F3A80000FB0EF39B1AB3FBFEF300FB01314FF099
:10F3B800010E0191D9F80430C3F30803002B40F083
:10F3C8008E80EFF31183002B40F089802B68A168B1
:10F3D80000BF2A689342F9D1D7F800B000FB0BF2BE
:10F3E800521AB2FBFBF200FB0323019A9B1AB3F5F6
:10F3F8007A7FDFD3BAF1010ABED1039B002B40F01C
:10F40800C4804FF47A7ADFF8A09150464FF0100C80
:10F41800D9F80430C3F30803002B40F09980EFF3C8
:10F428001183002B40F094802968A26800BF2B68E4
:10F438009942F9D1D7F800E000FB0EF39B1AB3FB11
:10F44800FEF300FB01314FF0010E0191D9F80430B1
:10F45800C3F308033BBBEFF3118323BB2B68A168FD
:10F4680000BF2A689342F9D1D7F800B000FB0BF22D
:10F47800521AB2FBFBF200FB0323019A9B1AB3F565
:10F488007A7FE3D3BAF1010AC2D1029B013B02930E
:10F498007FF468AF4349444B4448454A0860DA6002
:10F4A80005B0BDE8F08FEFF311888CF31288A168DE
:10F4B8002368DB0344BFC6F800E0A1682B68326804
:10F4C8005FFA88F888F31188D7F800801A4400FB9F
:10F4D80008F35B1AB3FBF8F300FB0233CDE7EFF355
:10F4E80011888CF31288A1682368DB0344BFC6F82F
:10F4F80000E0A1682B6832685FFA88F888F3118801
:10F50800D7F800801A4400FB08F35B1AB3FBF8F342
:10F5180000FB023369E7EFF311828CF31288D4F809
:10F5280008E02368D90303D501233360D4F808E041
:10F538002B683168D2B282F311883A68194400FB0B
:10F5480002F3A3EB0E03B3FBF2F300FB01312EE74A
:10F55800EFF311828CF31288D4F808E02368D903FA
:10F5680003D501233360D4F808E02B683168D2B2A0
:10F5780082F311883A68194400FB02F3A3EB0E03E7
:10F58800B3FBF2F300FB01315DE7184615F0BEFE50
:10F5980037E700BF6C5700207057002010E000E0EC
:10F5A80068570020FC9F002000ED00E0EFBEADDEB4
:10F5B8000400FA052DE9F047B14FB24E06F0EAFA19
:10F5C800BE421ED2DFF84483DFF8449344462588C0
:10F5D80062197DB14A450DD2052D0BD93388618852
:10F5E800C3F30B03994200F0FA8014462588621988
:10F5F800002DEFD1716830461436FCF735FCBE4259
:10F60800E4D3A14A1378A3F1170102290FD99F491E
:10F6180011F83300002840F00481D80001444978EB
:10F6280029B19B4911F83330002B00F02281994C05
:10F638006378022B84BF002363702378022B84BF76
:10F6480000232370944B9A78042A00F0098132B978
:10F658001A88B2F5F07F84BF4FF4F0721A808F4D8C
:10F668008F4A2B681A40002A00F00681D80700F15B
:10F67800F280590400F1EA801A0700F1E2809B0445
:10F6880000F1D880874D2B685A8C998C914224BF01
:10F6980000225A84FFF76EF910F094FD10B98248E1
:10F6A80007F084FA8020FCF715FC4FF40070FCF793
:10F6B80011FC4FF48030FCF70DFC4FF48020FCF770
:10F6C80009FC4FF40010FCF705FC4FF00070FCF744
:10F6D80001FC4FF08060FCF7FDFB6378022B06D835
:10F6E800724A734903EB430302EB83030B602378ED
:10F6F800022B07D803EB83016E4AC3EBC10302EB6D
:10F7080043032B6002F0E4FD002130226A481CF01C
:10F718002BFE286804F0DEFD684B2E6803F15001CB
:10F7280002E0043399427AD01A78002AF9D19C78F9
:10F73800D8788442F5D26249624B91F804E0624875
:10F74800624D5C6B624B2860C827642111FB0E7107
:10F75800DFF8C0E159605F4F30F8061C5E4DAEF827
:10F76800001000219960D960196159619961D961C6
:10F7780083F8201083F821103A702E600CB10CF039
:10F788000BFA564B9FED565A1B88564A9FED566A00
:10F798005579564C56495748086006EE903AF8EEA7
:10F7A800E66A1388C5EE265A07EE103A538812798E
:10F7B800C4ED005A07EE903AB8EEC77A4E4BF8EE11
:10F7C800E77A1D725A7227EE067A67EE867ABDE8E6
:10F7D800F04783ED017AC3ED007A06F0C3B9637987
:10F7E8009B077FF402AF716894F804A03046FCF7D9
:10F7F8003BFB3388BAEB133F04D01436BE42FFF408
:10F80800E5AEFEE673887068AA1FC3F30B039A423D
:10F8180004F10601A8BF1A461CF081FDEDE701229C
:10F8280089E7D8000C186468002C7FF4F7AE172419
:10F838001470F3E63148FCF74DFB4020FCF74AFB17
:10F8480020E72F48FCF746FB2B6818E72D48FCF704
:10F8580041FB2B6810E72C48FCF73CFB2B6808E7BA
:10F868009A8AB2F57A7FBFF4FAAE4FF47A729A8226
:10F87800F5E618231370DAE643F008032B60F5E683
:10F8880008220308F81D03087C3C00207CE70208D6
:10F89800A8CE0208DE590020C04B00205C3C0020A6
:10F8A80009600002EC59002008590020F059002096
:10F8B800D02B0020D0670020AC220020803C002004
:10F8C8008C2F002090590020423C002080560020B8
:10F8D800385A0020441B0020E0220020F820002095
:10F8E800C0C9FB481423002017B7D138FC200020DA
:10F8F8006C2D00203661023D482D00200940000291
:10F9080001600002092000020860000202F00308FA
:10F91800000004080843002008B506F03BF9FCF78E
:10F9280017FB06F01FF9FFF745FE0120BDE8084068
:10F9380008F0A8B92DE9F04F013085B0C3B20393A0
:10F948000B4602918B4C8C4E002B00F099808B4D0E
:10F958008B4FDFF8309215F069FE4FF4FA7A4FF0CA
:10F96800100C4FF47A70D9F80430C3F30803002B55
:10F9780040F0DE80EFF31183002B40F0D980296836
:10F98800A26800BF2B689942F9D1D7F800E000FBC4
:10F998000EF39B1AB3FBFEF300FB01314FF0010E8F
:10F9A8000191D9F80430C3F30803002B40F0878095
:10F9B800EFF31183002B40F082802B68A16800BF11
:10F9C8002A689342F9D1D7F800B000FB0BF2521A1B
:10F9D800B2FBFBF200FB0323019A9B1AB3F57A7F73
:10F9E800DFD3BAF1010ABED1039B002B40F0BD80E2
:10F9F8004FF47A7ADFF88C9150464FF0100CD9F812
:10FA08000430C3F30803002B75D1EFF31183002BE7
:10FA180071D12968A26800BF2B689942F9D1D7F83B
:10FA280000E000FB0EF39B1AB3FBFEF300FB013171
:10FA38004FF0010E0191D9F80430C3F3080313BB4A
:10FA4800EFF31183FBB92B68A16800BF2A689342C2
:10FA5800F9D1D7F800B000FB0BF2521AB2FBFBF257
:10FA680000FB0323019A9B1AB3F57A7FE3D3BAF11B
:10FA7800010AC4D1029B013B0293002B7FF467AFBC
:10FA880005B0BDE8F08FEFF311888CF31288A168F8
:10FA98002368DB0344BFC6F800E0A1682B6832681E
:10FAA8005FFA88F888F31188D7F800801A4400FBB9
:10FAB80008F35B1AB3FBF8F300FB0233D2E7EFF36A
:10FAC80011888CF31288A1682368DB0344BFC6F849
:10FAD80000E0A1682B6832685FFA88F888F311881B
:10FAE800D7F800801A4400FB08F35B1AB3FBF8F35D
:10FAF80000FB023370E7EFF311828CF31288D4F81D
:10FB080008E02368D90303D501233360D4F808E05B
:10FB18002B683168D2B282F311883A68194400FB25
:10FB280002F3A3EB0E03B3FBF2F300FB01317FE713
:10FB3800EFF311828CF31288D4F808E02368D90314
:10FB480003D501233360D4F808E02B683168D2B2BA
:10FB580082F311883A68194400FB02F3A3EB0E0301
:10FB6800B3FBF2F300FB013118E7184615F0CEFBA2
:10FB78003EE700BF10E000E0685700206C57002007
:10FB88007057002000ED00E0024B1A889B78028035
:10FB980083707047C8CB0208084B196861B130B44C
:10FBA8005D68074C642202FB05F2B2FBF1F2228089
:10FBB80030BC002018605860704700BF2423002024
:10FBC8007C430020704700BF6F4B1B78002B3AD056
:10FBD8002DE9F0416D4B6E4D9B79AC68A860013BF7
:10FBE80082B0041B032B00F29C80DFE803F04A027A
:10FBF800312902F021FB002800F09B80654B664903
:10FC08001B78B5F84220D1ED037AEA64DB0700F1EE
:10FC1800AA8002FB04F007EE900ADFED606A604BF1
:10FC2800B8EEE77AD5ED127A5A60E7EE267A1A60CE
:10FC3800BDEEE77AC5ED127A85ED117A83ED027A89
:10FC480002B0BDE8F081564A136053609360704774
:10FC5800544B1B681801F3D5FF2012F0FDF8037808
:10FC68000A2B88BF00214E4B9CBFB0F90420B0F985
:10FC78000610296588BF0A466A655A601A60996045
:10FC8800DEE7494A494BD279DFF8308133F8122050
:10FC9800B8F902304648B8F9001092B207EE902A37
:10FCA80040F6E44707FB02F6C3EB1633B8EE670AE3
:10FCB8004FF47A7606FB03F393FBF1F3AB61FBF7A2
:10FCC8009DFDD5F818E0D5ED047ADFED346AB8F972
:10FCD8000220334BB8F900C0C3F804E00EFB04F06F
:10FCE80007EE100AB8EEC77ABCEEC06AE7EE267ACD
:10FCF8008DED016ABDF80410C5ED047ABDEEE77A12
:10FD080007FB01F7C2EB173706FB07F683ED027A0C
:10FD180096FBFCF685ED037A6E611E6002B0BDE8C5
:10FD2800F0811F4B00221A605A609A6002B0BDE849
:10FD3800F0811C4B1B68DE067FF560AF154BB5F8EC
:10FD480042201B78EA64D9077FF563AFB5F9401004
:10FD5800184B00FB01F083FB0013C017C0EBA31086
:10FD68000244EA6455E7FDEEE77A134E17EE900A6F
:10FD7800A0F57A7101FB01F386FB0306D817C0EBE7
:10FD880026100844E2E700BF5A5500206C5A0020AC
:10FD980024230020D05A00205C5500202FE33E3158
:10FDA8002045002098510020E456002000570020EC
:10FDB80040230020D34D62101F85EB512C3C0020BE
:10FDC800F0B53E4B5B79012B83B03DD0022B0FD0B1
:10FDD8003B4B00221A805A803A4B1B78022B05D1E4
:10FDE800374A394B5188128819805A8003B0F0BDC0
:10FDF800364B1B681B01EFD5FF2012F02DF8037856
:10FE08000A2B56D8B0F902203149D31781FB0212C8
:10FE1800C3EBA2039BB207EE903AB8EE670A2D4CEB
:10FE280004F15C00A4F85A30FBF7E8FCFCEEC07A59
:10FE3800234AB4F85A30CDED017A5380BDF8043026
:10FE4800A4F858301380C7E7234A244B9278214DF1
:10FE580033F81240A4B207EE904A05F18400B8EED8
:10FE6800670AFBF7CBFC1E4A154910789678537839
:10FE7800FCEEC07A00EB4010CDED017ABDF804200D
:10FE880044F6FB77C3EB033300FB027200FB0474F8
:10FE9800B2FBF3F2B4FBF3F3B2FBF6F2B3FBF6F307
:10FEA80092B29BB2A5F88020A5F882300A804B80D8
:10FEB80092E79FED0C0A0023B1E700BF6C5A0020BF
:10FEC8004455002094540020985400209851002054
:10FED8006766666624230020E45600200057002049
:10FEE800BD67002000000000F8B52D4D2D49687948
:10FEF8002D4C2E4B2E4E042264270A7001284FF0F9
:10FF0800000184F8A82084F8B170A4F8AA10A4F815
:10FF1800AC1084F8B010C4F8B4103170198059804E
:10FF280021D0022810D0A979224A00230129136080
:10FF380084F8B8305360936023D0022912D11E4A46
:10FF4800636453609360F8BD282204F158001CF0E4
:10FF58000BFA4CF250319FED190A04F15C00FCF7E2
:10FF6800C9FBE0E7F8BD282204F180001CF0FCF989
:10FF78004CF250319FED110A04F18400FCF7BAFBF2
:10FF8800D1E70F4AE36053609360D3609FED0D0A99
:10FF980002F110004CF25031BDE8F840FCF7AABB62
:10FFA8006C5A002078430020242300204455002068
:10FFB8005A5500202045002068230020CDCCCC3D98
:10FFC80030230020CDCCCC3E2DE9F0432F4DD5F881
:10FFD800BC3083B01BB195F8C030022B02D003B0FF
:10FFE800BDE8F0834FF020084046294C05F1C409CC
:08FFF8000126552702F01AF959
:020000040801F1
:10000000A0B199F800300BB9217891B908F1010835
:100010005FFA88F8B8F1230F04F1010409F101092E
:10002000E1D0404602F006F90028EAD189F8000044
:10003000ECE7D5F8BC0050B30DF1080EAA220EF87B
:10004000052D8DF802108DF800708DF801608DF887
:100050000430694655225340082213F0800F02F104
:10006000FF324FEA430318BF83F0310312F0FF025F
:10007000DBB2F2D1714502D011F8012FEBE7AA22D1
:1000800069468DF803308DF8042010F0BBFE89F826
:100090000060BBE724230020CCCB02081F4B18785C
:1000A000002839D01E4A1389FBB11E4A9FED1E6AF3
:1000B000D2ED026A07EE903AF8EEE66AF8EE677A59
:1000C00007EE103A77EEE66AB8EEC77A66EE866A11
:1000D000C6EE877AFDEEE77A17EE900A6428A8BF8D
:1000E000642020EAE070C0B2704710B40F4B54781F
:1000F0001B88117804FB1032091B642300FB01F0FC
:1001000003FB02F3B3FBF0F06428A8BF64205DF8A2
:10011000044B20EAE070C0B2704700BF5A5500207F
:100120006C5A0020204500200000C84244550020A1
:100130002DE9F04F794D81B0FDF78EF8D5F8CC4020
:100140000022C5F8C820002C00F0A580237D052BD7
:10015000074617D9216A23690B44C31A9342B8BFD3
:1001600005F1CC010ADBD5E0137D052B0AD9136A12
:1001700012691344FB1A002B80F2CC8051F8042F33
:10018000002AF1D14FF0010B0023B9461E46C5F8F5
:10019000C83098469A46274623E07A6A39693B7DFB
:1001A000A9EB0204B4FBF1F40134A4B213FB04F391
:1001B000013301369BB2B6B23C83FB82984506D22E
:1001C000BBF1000F01D1012C5FD99846BA46D5F892
:1001D000C830013305EB8302C5F8C830D2F8CC70C3
:1001E00047B3BB68C3B1FC8A002CD6D1396A4846F4
:1001F000A9EB01019847D0B195F81831002B52D1E5
:100200003B7DC7F82490013601334FF00102B6B2AE
:100210003A83FB820124D1E73B6A3A69A9EB0304E4
:10022000B4FBF2F4A4B23C8334BBFB8AC6E73C8344
:10023000FB8AC3E72B686A683949013316443C4698
:1002400085E848004F46C1F800A0BAF1000F27D05A
:10025000DAF8203095F81821AAF81640FB1ACAF8E7
:100260001C30CAF82090002A35D1DAF80C30484604
:1002700001B0BDE8F04F18473B7D13FB04F3013399
:1002800001369BB2B6B2FB8298E73A7D062A04BFDC
:100290009846BA469BE72B68214A01332B601460CD
:1002A00001B0BDE8F08FFCF7D7FF1E4B1E4A1F4C74
:1002B00011681A68A0EB090002EB000E2268C3F86F
:1002C00000E09042A1EB5111014438BF1046164A9C
:1002D0002060116094E7FCF7BFFFDAF80C300446A9
:1002E0009847FCF7B9FFDAF82C20DAF82830DAF86A
:1002F0003010001B9042A3EB53130344014438BF5A
:100300001046CAF82830CAF83010CAF82C0001B0DC
:10031000BDE8F08F4FF0000B36E700BF242300202C
:10032000244800208043002084430020884300208C
:10033000F0B43423184F194A03FB00F3D2F81C61C0
:10034000FC58FD18002E6B684B600C600DDDD2F878
:10035000CC309D421DD0CC32002303E052F8044F34
:10036000A54216D00133B342F8D10022342303FB57
:1003700000700A720369CB60037D4B72836AC56AA1
:10038000046BC2690A615B094D618C61CB61F0BC91
:1003900070470122EAE700BF10010020242300205B
:1003A0002DE9F0414E4ED6F81C41112C7ADC002C80
:1003B00040F39380D6F8CC30984273D0012C5DD0B6
:1003C000D6F8D03098426DD0022C57D0D6F8D43021
:1003D000984267D0032C51D0D6F8D830984261D0DB
:1003E000042C4BD0D6F8DC3098425BD0052C45D09D
:1003F000D6F8E030984255D0062C3FD0D6F8E430FD
:1004000098424FD0072C39D0D6F8E830984249D0DE
:10041000082C33D0D6F8EC30984243D0092C2DD09C
:10042000D6F8F03098423DD00A2C27D0D6F8F430D8
:10043000984237D00B2C21D0D6F8F830984231D0E2
:100440000C2C1BD0D6F8FC3098422BD00D2C15D09C
:10045000D6F80031984225D00E2C0FD0D6F80431B2
:1004600098421FD00F2C09D0D6F80831984219D0E5
:10047000112C03D1D6F80C31984213D0D6F8CC50B9
:100480004DB32B7D017D8B420FD3164F00253A468D
:1004900005E052F8043F53B11B7D8B4207D3013571
:1004A000AC42F6DA0020BDE8F0810E4F00256B1C4F
:1004B0009B00191F621B06EB850580463944F8181E
:1004C000920001341BF03AFFC5F8CC80C6F81C41FD
:1004D0000120BDE8F081034FE9E7CFD0E2E700BF9C
:1004E00024230020F0230020132830D0112807D81F
:1004F000184B342202FB003019B1C3680BB14FE72F
:10050000704770B5144DD5F81C41002C0FDDD5F89F
:10051000CC3098420CD005F1CC063346002203E0E3
:1005200053F8041F884206D00132A242F8D170BDB0
:10053000002205F1CC069000011DA21A9200314460
:100540003044013C1BF0FAFEC5F81C4170BD034B62
:100550001868D1E71001002024230020244800203F
:1005600010B54FF4804082B007F0E2F900B30022EA
:10057000032390F90200009301924FF4E1334FF40A
:10058000804106F0B7FD0C4BC3F8BC0070B10124EC
:1005900002221120214683F8C44083F8C54083F825
:1005A000C64083F8C020FFF79FFF204602B010BD71
:1005B000014BD3F8BC00E9E724230020F0B5064640
:1005C000006803681B6A85B00D4603B1984795E83B
:1005D0001800E41A0023039324238DF808304D23D8
:1005E0008DF80930B5F90A30FF2C2246A8BFFF224A
:1005F00001333FD02B7B002B0CBF3E233C238DF8D7
:100600000A30FE2C2B898DF80B208DF80C3033DD51
:1006100023128DF80D408DF80E3007273A4602A9B7
:100620003068FCF769FF02ABDA190DF10B0100230A
:10063000914223D1002C8DF807300CDD2246296829
:100640003068FCF759FF2B689DF8072019198B4279
:1006500018D18DF80720306801220DF10701FCF751
:100660004BFF306803685B6A03B1984704F10900E7
:1006700005B0F0BD2123C2E70527CFE711F8010B34
:100680004340D5E713F8010B4240E0E7F8B50A4EC6
:1006900005460024A359AB4204EB060707D12846C0
:1006A00006F0FCFCCC22002138461BF061FECC3465
:1006B000B4F5197FEED1F8BD885B00202DE9F34732
:1006C000012007F035F9174EDFF85CA00024CC2795
:1006D00008B1022C02D902B0BDE8F08707FB04F88C
:1006E00056F8085015B10134E4B2F1E7C37890F937
:1006F00002005AF8233001950322009201212A4674
:1007000006F0F8FC814648B104FB0760CC2229467C
:100710001BF02EFE013446F80890E4B215F062FE9C
:10072000D6E700BF885B002018E202082DE9F04FF1
:100730002DED088BB84CB94BC4F8343887B0002382
:10074000C4F83838FCF7DAF8FDF7C4FAFBF7CEFB4B
:1007500008B9FEF7DDF9FEF731FF0522B049B148CF
:100760001BF051FE08B1FEF7D3F994F83C38AE4DBA
:1007700043F0010384F83C38AC4B9A78AC4B1A70C8
:10078000AC4B1B682B6010F087F901210220FDF7AC
:100790000DFFFBF7EBFA2B6819070BD5A64B1A7A5E
:1007A0000A2A07D80123934040F20342134201D0A2
:1007B0000FF0A8FF6420A14EFCF7B0FCFEF798FAFA
:1007C0009F4ADFF8B8E20023B146995D03F10F00BC
:1007D00003F11307304437440EEB010A10F8018F80
:1007E000B8F1000F05D09AF80CC0C44508BF82F8D4
:1007F00058C090F80480B8F1000F05D01EF801C071
:10080000C44508BF82F859C08742E7D1B2F8580002
:1008100040B104EB810109EB03005065C1F84028A9
:1008200002F517722033602BCFD1286842F2010302
:1008300018420CBF4FF0FF310121C0F3801006F0C9
:10084000A9FA2B68DA0740F17F830FF055FCB4F862
:1008500058687C4B94F854081E80002E40F07A8330
:10086000FDF712FA784A7949106094F85528003259
:1008700018BF01220A7058B194F85638C671002B7F
:100880004FF02402827114BF11210121FDF792FC67
:100890000020FDF761FEDFF8E891DFF8E88159F804
:1008A000063C0293002B3AD019F90A6C142303FB7F
:1008B00006871A46002138461BF05AFDA219A9F1F5
:1008C000030A92F85A3892F85CB803931AF8011F99
:1008D000039B994203D11846FDF7D6F9B8609AF800
:1008E0000310594503D15846FDF7CEF9F860D145BC
:1008F000ECD1142303FB06F108EB0102906870B100
:10090000D06860B12644A9F10A0048F8010096F8C1
:100910005E18029B117496F86018536051744C4B2A
:1009200009F110099945BAD114F07AFC494B93F8B2
:1009300008909846B9F1000F2BD04846FDF7A4F96E
:10094000454E0746706018B12F2383710023C37191
:1009500098F80010002940F00183484615F0DAFCB1
:100960008046B0B127B1027A02213846FCF706FE74
:100970003A4F3B4A00230193009341468023384677
:1009800013F0A4FFB268802333611360012307F8DA
:10099000083C3449344A4B79581E43424341137052
:1009A0008B795E1E7342734113712B681F0400F133
:1009B000078313F0007305D01F4BDB7AA3F1080106
:1009C0004B424B41294E937014F020FA33682BB9F7
:1009D00072681AB9B268002A00F0D9801BB208EE1A
:1009E000103ADFED23AADFED238A234AB8EEC88A46
:1009F000002128EE2A8A117038EE280AFDEEC07A0E
:100A000017EE903A2033402B00F2DC82FBF7FCFD1E
:100A1000F0EE409A38E000BF2423002059BC0008C3
:100A200099ED0208E359002098510020DE5900207A
:100A3000945400205C3C002030530020D0CB0208AE
:100A400044240020445700204857002046570020E7
:100A50005ACC0208C8560020B4560020BC560020CC
:100A600000A24A046C5A0020F85600208C43002053
:100A700035FA8E3CDB0FC93F0C010020605300208B
:100A80003ACC020808570020FDEEC87A17EE903ADB
:100A90002033402B00F29982B0EE480AFBF7B4FDF8
:100AA000B0EE40AAB6F9043009EE103AB8EEC99A91
:100AB00029EE2A9A39EE280AFDEEC07A17EE903A0E
:100AC0002033402B00F28482FBF79EFDB0EE40BA4B
:100AD000FDEEC97A17EE903A2033402B00F27B826C
:100AE000B0EE490AFBF790FDB0EE409AB6F9083037
:100AF00008EE103AB8EEC88A28EE2A8A38EE280A9C
:100B0000FDEEC07A17EE903A2033402B00F2668259
:100B1000FBF77AFDF0EE408AFDEEC87A17EE903AC8
:100B20002033402B00F25D82B0EE480AFBF76CFDEB
:100B300069EE806A68EE8A7AF0EE665AE7EE895AC4
:100B4000C64B28EEA96A20EE0A7AC3ED035AF0EEEE
:100B5000465AE7EE495AE6EE897AA6EE497A68EEF9
:100B60008B8A2BEE400A2AEE4BAA69EE8B9AC3EDD4
:100B7000008A83ED010A83ED029AC3ED045A83EDE6
:100B800005AA83ED067AC3ED077AC3ED089A0AF049
:100B90008FFD002800F02882B14B18680BF0F0F8A8
:100BA00094F83C38AF4F012143F00203084684F823
:100BB0003C38FDF7FBFC00210846FDF7F7FC00215F
:100BC0000220FDF7F3FC0A260120FCF7C9FC0020F7
:100BD000FCF7C6FC1920FCF7A1FA3B68DB0302D442
:100BE0000120FDF7B9FC1920FCF798FA0020FDF769
:100BF000B3FC013EE8D131463046FDF7D7FC314623
:100C00000120FDF7D3FCFDF7B9FE974B974F18680D
:100C100003F064FB964B18880BF03AF8954B3A7842
:100C20001A7004F0F1F92A68934B12F4805F9E8ADF
:100C300018BF924A9B7818BF9688042BB84604D1F7
:100C40004FF48050FBF74AF9002603F0FFFF8C4B6E
:100C5000304619780DF0AAFB94F83C3843F00403B1
:100C600084F83C3803F064F905F02AFF854B1B68D3
:100C70000BB10DF0A9F905F059FB04F0D1FA12F00F
:100C8000DDFE4FF4197200217F48DFF84C927F4E51
:100C90001BF06EFBFFF712FD7D4B00271F809F703E
:100CA00004F094FF7B4B37604FF0FF3AC3F800A08D
:100CB0004846794BC4F864380CF07AFC774A84F8DB
:100CC0007278012384F87038537884F871A80D3352
:100CD00084F86C3813781E3384F86D383368042B2D
:100CE00004D05A1C32606E4A42F823902B689F034E
:100CF00052D594F880386B4FDFF8E0A1C7F800A018
:100D0000013B84F87838C82094F8813884F8793821
:100D1000FCF704FA3868DFF8C891FBF7C9FD89F8D9
:100D20000000C820FCF7FAF93B68C4F888380AF1DB
:100D300010075D4BC4F8843838460CF0E5FB0123FE
:100D400084F89038002384F89238FF2384F891388F
:100D5000082384F88C38152384F88D38534B1F6092
:100D600099F800303BB13368042B04D05A1C326030
:100D70004B4A42F823704E4C1022002120461BF0B3
:100D8000F7FA002015F08CFFFCF766FA064615F01E
:100D9000A1FF484B3344E3602B68580501D50DF0A3
:100DA00065F82B68190101D511F02EF808F034F917
:100DB00098F80030052B03D13F4B4FF4C8721A80CE
:100DC000274B3E4C1A684FF47A73B3FBF2F3C3EB34
:100DD000431203EB82033A4ADB00A2F8B4304FF42B
:100DE000006006F0A5FD98B1364B90F9020093F82B
:100DF0003230002B14BF18230023019303230093E8
:100E000000224FF496534FF4006106F073F920600E
:100E1000236813B12C4B2D4A1A604FF4005006F092
:100E200087FD2B4C98B1274B90F9020093F8323094
:100E3000002B14BF082300230193032300930022F7
:100E40004FF416534FF4005106F054F92060236814
:100E5000002B47D01C4B1F4A1A6043E0E44200209D
:100E600088510020A4430020EC5900207C3C002045
:100E70003C3C002058320020C04B0020742F002042
:100E800075540020C4330020885B0020F8550020F2
:100E9000385A00200405002050CC02082C450020C0
:100EA000FC550020885900207CCC02082C5A0020D8
:100EB0001C5A0020404B4C00666A0020CC66002083
:100EC000044F002097440020885300208400002015
:100ED000D85A0020A0000020882B0020982B00204A
:100EE000355A0020454A137843F008031370FEF783
:100EF000FFFF434B1A68920306D5424A07215172FD
:100F0000117A41F0010111723F4A12681A603F4B99
:100F10003F4A1B689B1A3F4A18BF012313703E4A81
:100F2000138843F08003138006F0F8FEFFF718FBE8
:100F30003A4A92F83C3863F07F0382F83C3807B0B5
:100F4000BDEC088BBDE8F08F9B047FF580AC0FF003
:100F50007FF87CE4314613F04FFE9CE401297FF4D6
:100F600018AD17B13846FCF7D7FC7068FDF7E4FA06
:100F700001274FF4E073336137703623002604A84D
:100F80008DF810308DF811708DF812608DF8137097
:100F900016F0C0F8372305A88DF814308DF81570B9
:100FA0008DF816608DF8177016F0B4F81C4AD369E6
:100FB00043F03003D3611B4B1E85A3F82864E8E49B
:100FC0000123FFE4DFED189A5EE59FED17AA69E5BE
:100FD0009FED15BA7CE59FED149A87E5DFED128A47
:100FE0009AE59FED110AA3E502210120FEF7A6FC78
:100FF000094A138843F001031380D1E5CC3F002058
:10100000985100201C5A00205C3C0020D84B002046
:101010008D440208EC4E0020A2550020242300201D
:1010200000100240001000400000000008B50E4B08
:101030001978012913D00DD3022902D10020FCF721
:101040008FFAFCF709F9094B00F5F42000F59070D0
:10105000186008BD00210846FDF7A8FAF1E7002056
:10106000FDF7A4FAEDE700BF686A00206C6A002073
:10107000037903F00C03042B05D0082B0FD0C3B960
:10108000B0F80B0070470C4BB0F80B001B7803EB6B
:101090008302C3EBC20300EB430080B27047064BF0
:1010A000B0F80B005B7803EB430300EB830080B2E6
:1010B00070470020704700BFDE590020FAF7A8BE35
:1010C00020B10078B0FA80F04009704701207047E5
:1010D00008B520211BF081F90346184623B1027898
:1010E000202A03F10103F8D008BD2DE9F8430D468D
:1010F00016468146002440F634074FF0190848464A
:10110000FFF7E6FF814690B118F08AFEB842A8BF0B
:101110003846B0F5617FB8BF4FF46170A0F56170DB
:1011200090FBF8F04CB928703378013333700134F8
:10113000022CE4D14846BDE8F8836870F4E710B5A6
:101140000446B0F80900FAF7B7FE01462046FFF75B
:101150008FFF4B68184410BD38B505460C46FFF7A5
:10116000EEFF2B7903F00303012B00D001D20470B2
:1011700038BD048038BD0FB413B5084C0849206849
:1011800004AB53F8042B0193FBF73AF92068FAF704
:1011900031FE02B0BDE8104004B07047082C0020BA
:1011A000BD100108024B01461868FAF731BE00BFB6
:1011B000082C002038B5064C451E15F8011F206884
:1011C00019B9BDE83840FAF715BEFAF721FEF4E781
:1011D000082C00202DE9F0410379054603F030008A
:1011E00020280E4614462BD1294FDFF8B08000246A
:1011F0006B799C4201DBBDE8F0812B7903F003039E
:10120000022B11D0032B15D0012B14BF315D3157A8
:101210003846FFF7B0FF6B79013B9C4202DA40464B
:10122000FFF7C8FF0134E3E736F814103846FFF73C
:10123000A2FFF0E736F914103846FFF79CFFEAE703
:1012400003F00303012B06D008D2097848B1102817
:1012500013D0BDE8F08191F90010F7E7B1F9001063
:10126000F4E70B48FFF787FF84B1B5F90720B5F91C
:1012700005100848BDE8F0417DE76A79064B53F850
:101280003230BDE8F04153F8210093E7BDE8F0812A
:10129000D1ED0208D2F1020894DD0208B0ED020897
:1012A00038B50D460446FFF74AFF2A460146204658
:1012B000BDE838408EE701487CE700BF3CEF0208FC
:1012C0002DE9F74F344C01F0100381468846002584
:1012D00027460093314B1868FAF78CFD94F804B058
:1012E0000BF00C034B453FD10D2303FB0573B3F803
:1012F0000900FAF7E1FD06462046FFF7B9FE0BF0BC
:101300000302012A82467168B06835D03CD211F8D8
:101310000A2010F80A00801A42424241009B03B1A1
:1013200012BB18F0200F10D07AB90D2101FB057106
:101330001B4809680192FFF71EFF7168019A51442A
:101340002046FFF747FFFFF7B6FF0D2202FB0572AD
:1013500014481168FFF70FFFB1680022514420467E
:10136000FFF738FFFFF7A7FF0135C22D04F10D0489
:10137000B0D103B0BDE8F08F11F90A2010F90A00CE
:10138000811A4A424A41C9E731F90A2030F90A0074
:10139000831A5A425A41C1E7B8D30208082C0020E8
:1013A000B2ED0208B3ED020810B5064C0B4602463A
:1013B00005492068FBF724F82068FAF71BFDBDE813
:1013C000104078E7082C0020BD1001080FB407B5C5
:1013D00004A951F8040B0191FFF7E6FF03B05DF893
:1013E00004EB04B07047F8B5037903F03003102B19
:1013F0000AD0202B23D03BBBB0F90720B0F9051051
:101400001248BDE8F840E1E74579114E1148FFF771
:10141000D1FE06EBC50300241F79BC4202D3BDE810
:10142000F84048E714B10C48FFF7C4FE56F83530D1
:101430000A4853F82410FFF79EFE0134EDE7417986
:101440000748BDE8F840C1E7F8BD00BFBDED0208A0
:1014500094DD0208D4ED0208B0ED0208C2F00208E3
:10146000E4ED02080CB407B510F0200009D069B90A
:101470002320FFF797FE05A904980191FFF794FF39
:10148000012003B05DF804EB02B070470020F8E7DC
:101490000CB4C30607B500D551B905A9049801914C
:1014A000FFF782FF012003B05DF804EB02B0704744
:1014B0000020F8E72DE9F04FDFF820B189B0804631
:1014C000894616460D4614464FF0000A002E71D08C
:1014D0006A6863689A426BD1AF68A368FB1A5F427F
:1014E0005F4194F90B30049394F90A300393B4F9F3
:1014F00008300293B4F906300193B4F90430009334
:101500005A46534639464046FFF7ACFF95F90B3033
:10151000049395F90A300393B5F908300293B5F9AD
:1015200006300193B5F9043000935A4653463946C4
:1015300040460AF1010AFFF7ABFFBAF1080F05F1C7
:101540000C0504F10C04C1D10024DFF894A0254659
:1015500096B30027012303FA07FB325959F80430E8
:1015600053403BEA030314BF0123002312EA0B0F8D
:10157000079306D000972B46524607994046FFF73F
:1015800071FF59F804301BEA030F06D000972B4671
:10159000524607994046FFF77BFF01370E2FD9D1FE
:1015A0000135082D04F10C04D2D109B0BDE8F08F4B
:1015B000002796E73746A9E73746012359F8042064
:1015C000BB40134206D000972B46524601214046AD
:1015D000FFF75EFF01370E2FEFD1E1E7F5ED0208CF
:1015E0000DEE02082DE9F347DFF868A081460F46AB
:1015F000904602260024B8F1000F28D037F82420A6
:1016000038F824309A4238F806201ED1BD5BA91A5A
:101610004D424D4101920093524623462946484689
:10162000FFF720FFBB5B019337F82430009352464D
:101630002346294648460134FFF72AFF042C06F1C9
:101640000406D8D102B0BDE8F0870025E2E74546A0
:10165000E8E700BF22EE02082DE9F04F2DED088BE0
:10166000DFF80C9193B0804692460D461446002652
:1016700095ED008AB5EE408AF1EE10FA71D0D5ED05
:10168000019A95ED029AD5ED038ABAF1000F3FD089
:1016900094ED000A94ED01BAD4ED02AA94ED03AAE8
:1016A000B4EE408AF1EE10FA60D1F4EE4B9AF1EE0E
:1016B00010FA5BD1B4EE6A9AF1EE10FA56D1F4EE5C
:1016C0004A8AF1EE10FA0CBF012700270FA8FAF79B
:1016D00097FDB0EE4B0A83460CA8FAF791FDB0EEE9
:1016E0006A0A059009A8FAF78BFDB0EE4A0A049041
:1016F00006A8FAF785FD049A059B039002920193D0
:10170000CDF800B033464A4639464046FFF7AAFEB8
:10171000B0EE480A0FA8FAF773FDB0EE690A074663
:101720000CA8FAF76DFDB0EE490A834609A8FAF74E
:1017300067FDB0EE680A049006A8FAF761FD049B05
:10174000039002938DE8800833464A4600214046C4
:101750000136FFF79DFE082E05F1100504F1100477
:1017600086D113B0BDEC088BBDE8F08F0027ADE744
:1017700033EE02082DE9F04F834687B092460C46BF
:10178000154600274FF019094FF46178BAF1000FA0
:101790004ED023782A7893422B7947D160786978A4
:1017A000884243D1A078A97888423FD1E078E9788F
:1017B00088423BD12179994238D166796979711A89
:1017C0004E424E410593EB780493AB7819FB0383AB
:1017D00003936B78019219FB038302936B79009357
:1017E000144A3B4631465846FFF73CFE23790593A1
:1017F000E3780493A3780F4A19FB03830393637878
:1018000019FB038302932378019363790093314694
:101810003B4658460137FFF73BFE0F2F04F1060405
:1018200005F10605B2D107B0BDE8F08F0026C9E783
:101830005646DBE747EE02082DE9F04F364FDFF85A
:10184000E0A087B0814690460C46164602F1300B68
:1018500094F9022000233149591891F90610914258
:1018600054D00833302BF6D108365E4504F1080415
:10187000EED107B0BDE8F08F96F9023071799A4247
:10188000328841D1208890423ED1E578F078854277
:101890003AD125793079854236D1A579B07985421A
:1018A00032D16579681A4542454157F821100491B3
:1018B000B17957F821100391317957F8211002912D
:1018C000F178009257F82110019152462946484676
:1018D000FFF7C8FD627994F9023057F8222004928C
:1018E000A27957F822200392227957F822200292F7
:1018F000E27857F822200192228800922946524627
:101900004846FFF7C5FDAFE70025CEE7B8F1000F69
:10191000B2D14546DEE700BF18E202088C53002032
:1019200065EE02082DE9F04FDFF8B4A085B08146DE
:1019300090460C46154600261927B8F1000F4CD0EA
:1019400028782378834246D162786B789A4242D1D4
:10195000A278AB789A423ED1E178EB78CB1A594223
:1019600059418B4612F04AF998B1EA784FF4617107
:1019700017FB02120392AB7817FB031302936B78E9
:101980000193037A00935246334659464846FFF77F
:1019900069FD207812F032F998B1E2784FF4617164
:1019A00017FB02120392A37817FB031302936378C9
:1019B0000193037A00935246334659464846FFF74F
:1019C00067FD0136142E04F1040405F10405B4D1B9
:1019D00005B0BDE8F08F0021C3E7C346D9E700BFDB
:1019E00082EE0208F7B50746FFF76AFB044630B1FE
:1019F000002224490120FFF795FF03B0F0BD3846CF
:101A000018F00EFA1328054635DC8600781C8DF890
:101A10000740FFF75DFB1B4C074668B118F000FA62
:101A2000C0B212F0D1F838B1037804F825309DF82F
:101A3000073001338DF807303846FFF749FB07467A
:101A400050B118F0EDF90D2806D8A31958709DF87B
:101A5000073001338DF80730B11C0DF10702214426
:101A60003846FFF742FB9DF80730042BC5D0002312
:101A700044F82530C1E71323224603490348FFF702
:101A8000A5FCBAE7803C002095EE02089BEE020818
:101A900008B5FFF78FFBBDE808400CE40048F7E706
:101AA000B4EE0208F0B585B00546FFF709FB002843
:101AB00038D104462B78002B3BD1062C41D1BDF9FF
:101AC00004309AB2072A3CD8BDF90610A1F2EE22E2
:101AD00092B240F2DC54A24233D8BDF90820A2F2FF
:101AE000EE2080B2A0422CD8BDF90A00814228DC49
:101AF000824226DB914224DCBDF90C5005F16404DE
:101B0000A4B2C82C1DD8BDF90E40112C19DC194EF9
:101B10000C2707FB03639980DA8018819D72DC72C1
:101B200005B0F0BD13490022012005B0BDE8F0402A
:101B3000C0E42D2B03D0A3F13002092A15D8052CBF
:101B400003DD05B0BDE8F040A8E7284618F068F9C5
:101B500004AB661C03EB440424F80C0C15F8013F9D
:101B6000303B092BFAD93446A4E7202BE9D10135C3
:101B70002646F8E7603200202DE9F0410546FFF7E0
:101B80009FFA064628B1002227490120BDE8F0410E
:101B900028E5264928461AF0F3FB70B9224B4FF48A
:101BA0007A714FF4FA6219805A809980DA8019812B
:101BB0005A819981DA81BDE8F081284618F030F920
:101BC0000328044628D82846FFF782FA064650B173
:101BD00018F026F9012705463046FFF779FA28B9AB
:101BE000BDE8F0415AE705460746F5E718F018F951
:101BF000002FF5D0A5F2EE2240F2DC539A42EFD846
